:020000040800F2
:100000000070012001000108D9820408DB82040885
:10001000DD820408DF820408E18204080000000099
:10002000000000000000000000000000E38204085F
:10003000E582040800000000E5960408FD96040827
:100040004500010845000108450001084500010878
:1000500007C8040845000108F9D30408FFD30408C1
:1000600005D404080BD4040811D40408FD9804082E
:100070000D9904081D9904082D9904085599040840
:10008000659904087599040845000108F982040877
:1000900005830408450001084500010817D4040839
:1000A0008F83040827830408398304083F830408E6
:1000B000458304084B830408518304084500010864
:1000C00045000108450001084500010845000108F8
:1000D00045000108098304080F83040815830408F8
:1000E0003BD4040845000108E9820408958304080C
:1000F0007D8304089B83040845000108450001082E
:10010000450001084500010859830408450001081D
:100110001B8304082183040871830408778304087F
:100120008599040895990408A5990408B5990408C7
:1001300000000000000000000000000000000000BF
:1001400000000000000000000000000000000000AF
:1001500045000108450001084500010800000000B5
:10016000000000000000000000000000000000008F
:10017000000000000000000000000000000000007F
:10018000000000000000000000000000000000006F
:10019000000000000000000000000000000000005F
:1001A000000000000000000000000000000000004F
:1001B000000000000000000000000000000000003F
:1001C000000000000000000000000000000000002F
:1001D000000000000000000000000000000000001F
:0401E0005FF8E0F1F3
:020000040801F1
:10000000002103E00A4B5B584350043109480A4B76
:1000100042189A42F6D3094A02E0002342F8043B10
:10002000074B9A42F9D337F0EDFC37F011FE7047D9
:10003000BF8E0608000000206C0300207003002023
:1000400090230020FEE7000040F8044B40F8045BDA
:1000500040F8046B40F8047B40F8048B40F8049BA4
:1000600040F804AB40F804BB40F804CB40F804DB94
:1000700068467047024B5A69026058610020704719
:1000800070030020024B5A6912685A61704700BF22
:1000900070030020024B9A69C0E900219861704703
:1000A00070030020044A93691968916110B11846E1
:1000B0005A681047704700BF7003002038B50446E7
:1000C000044DAB690BB1A34200D338BD0120FFF74B
:1000D000E9FFF6E770030020C460056146618761AF
:1000E000C0F81C80C0F82090C0F824A0C0F828B048
:1000F000C0F82CD0C0F808E0FFF7BCBF0F4D08B522
:100100006C690CB937F060FE60602046FFF7D6FFDF
:1001100023686B612046C468056946698769D0F821
:100120001C80D0F82090D0F824A0D0F828B0D0F8C7
:100130002CD0D0F808E00120704700BF70030020E9
:1001400010B50021044600F00FFA18B914B120468A
:100150000DF0B2FC10BD002100F006BA10B501216F
:10016000044600F001FA18B914B120460DF0A4FCC1
:1001700010BDFFF7E5BF10B501220C4600F00AFBE9
:1001800018B914B120460DF097FC10BD00F002BB69
:1001900000F094BA2DE9F04100210325274A0024FC
:1001A000D2F84472013403199E08BE5D03F00303C4
:1001B0005B0046FA03F303F00303022BF2D0D2F8FC
:1001C000503203EB001000EB0414A04206D191B3AF
:1001D000013902EB4103B3F86402E0E703681E074C
:1001E00027D1D2F850629E4223D8D2F854729F424F
:1001F0001FD99B1BD2F844C29F091CF807804FEA05
:10020000131EC3F301135B0048FA03F606F003065E
:10021000012E0ED105FA03F33F2943EA08030CF837
:1002200007309DBF02EB4103A3F864E20131C2F83D
:1002300060620430C9E7BDE8F08100BF70030020B0
:100240004FF4037221F00F0138B50B1A013BDB00AC
:10025000B3FBF2F305460F4C5A1C1544C4E9910355
:10026000C4F84C52A1EB83159B00073302EBD30279
:10027000C4E99451002131F0A0FB01220023A4F82D
:10028000E4224FF0FF32C4E99633C4E9BA32238145
:1002900038BD00BF70030020024A13890233138166
:1002A000704700BF70030020024A1389023B13818C
:1002B000704700BF70030020024B1889003818BF38
:1002C00001207047700300202DE9F04106460D46DD
:1002D00000244FF00308154FAC4201D1BDE8F08176
:1002E00056F824301A071FD1D7F850229A421BD84B
:1002F000D7F85412994217D99B1AD7F844C29909D2
:100300001CF801E01809C3F301135B004EFA03F275
:1003100002F00302012A07D108FA03F343EA0E03AD
:100320000CF80130FFF736FF0134D5E770030020E9
:100330000748662103890C3043F0010320F8043C90
:100340000023C0F85432C0F8DC32FFF7BDBF00BF55
:10035000700300202DE9F74300274C4CD4F860626D
:10036000002E3ED14FF00109D4F85C324FEAD30899
:10037000D4F84C32F7009D5D002D49D10136B045CF
:10038000F6D2A8462A4603274FF0020CD4F844625E
:100390009008315C02F003035B0041FA03FE0EF0AB
:1003A000030EBEF1020F65D0BEF1030F66D0BEF1A1
:1003B000010F05D1012507FA03F321EA03033354A2
:1003C000D4F85C3201329A42E0D90023C4F85832A2
:1003D0002389C4F85C8223F00103238103B0BDE8C4
:1003E000F0830025C4F86072D4E99123B5EB830F44
:1003F000B4D2AB08D35C05F003025200134103F002
:100400000303032B02D12846FFF7C4FE0135EBE7B7
:10041000EB072CD5D4F84422BB08D35C07F00302C9
:100420005200134103F00303012B20D1D4F85022D2
:100430003B01D35802EB071073B16A4640F22B21FF
:100440000CF09AFC009B3BB10DF082FDDDE9000150
:100450000DF04EFD0DF092FDD4F84C02FB0807F0B4
:10046000070209FA02F1C25C22EA0102C2546D08D5
:10047000013781E7002D9DD19046A1E70CFA03F3E7
:1004800021EA030390460025335499E770030020C6
:10049000044B1A8942F001021A810022C3F860223B
:1004A000FFF758BF7003002000232E4AF0B5D2E9B1
:1004B0009441D2E99176091B01601D4619461C46FC
:1004C000C0E90133C0E90333C0E90533B600A3082E
:1004D000FB5C04F003025200134103F00303012B01
:1004E00042682AD0022B2BD023B982680131013215
:1004F00082601D460134A6420AD0A308FA5C04F0CB
:1005000003035B001A4112F0030301D0012BDED17B
:10051000012D19D10269013202618269AA4238BFF4
:100520008561A64201D0012BD1D1C3688B4238BF6F
:10053000C160A6420ED00021C9E701324260D8E76F
:10054000013242600135D5E7022D02BF4269013216
:100550004261E2E743681B01436083681B018360DB
:10056000F0BD00BF700300202DE9F84300F10F0635
:1005700036090D4603D100231846BDE8F8834E4CDA
:100580002389002BF7D1B4F8E432002B0CBF0120F3
:10059000002006D0D4E9BA239A4202D339F06EF88B
:1005A0000120D4E991C70022D4F858329F4202D8E2
:1005B0000028E0D1F2E71CF8031011F0030F49D135
:1005C0000132964247D89B00012A02BF591C890874
:1005D000C4F85812981AD4F85C12471C99422CBFE0
:1005E000C4F85C12C4F85C3207F003014FEA41081A
:1005F00001214FEA970E01FA08F11CF80E80023033
:1006000041EA08014FF002080CF80E10834242D272
:10061000D4F8E812D4F85082314408EB0713184696
:10062000C4F8E8121201002131F0C7F9EA070346C5
:100630004FEA0719A0D5002248F809200122D4F872
:100640004C02F90807F0070702FA07F7425C174364
:10065000475491E7002211F00C0F05D10132964268
:1006600003D89B000133AFE7002211F0300F05D112
:100670000132964203D89B000233A5E7002211F015
:10068000C00F05D10132964203D89B0003339BE78C
:10069000002201338AE7D4F844E24FEA900C00F0DC
:1006A00003011EF80C90490008FA01F141EA090122
:1006B0000EF80C100130A9E7700300201C4B70B538
:1006C0001A8922F0010292BB88B30121D3F850228B
:1006D000D3F84C62801AC509C0F3021401FA04F47D
:1006E000715D020921EA040171550325D3F85842CE
:1006F0008109B4EB901F88BFC3F85812D3F8446245
:10070000940802F00301305D490005FA01F120EA86
:1007100001013155D3F8440201329108415C02F0E5
:1007200003004000014101F003010229E6D070BD41
:1007300070030020034610F00F0010B526D1144AB4
:10074000D2F85012994220D8D2F854429C421CD977
:100750005B1AD2F844129A098A5C1C09C3F301138C
:100760005B0042FA03F303F00303012B0DD10130C8
:1007700023189A088A5C03F003035B0042FA03F330
:1007800003F00303022BF2D0000110BD0020FCE7B0
:10079000700300202DE9F84F88461446064628B914
:1007A00001464046BDE8F84FFFF7DEBE19B9FFF736
:1007B00085FF002433E04C480589002DF9D1D0F89D
:1007C0004872D0F850124FEA87090127711A0B09B5
:1007D00008F10F02D0F844A2120903F1010ECE4530
:1007E0001AD24FEA9E0C1AF80CC00EF0030B4FEA17
:1007F0004B0B4CFA0BFC0CF0030CBCF1020F03D1B9
:1008000001370EF1010EEAE7BCF1000F04D101350A
:1008100007EB050C9445F4D3974203D134462046A8
:10082000BDE8F88F1ED91A4414463B440327D0F87C
:1008300044124FEA940E04F0030511F80EC06D0047
:1008400007FA05F501342CEA05059C4201F80E5023
:10085000EDD1D0F858129308B1EB920F88BFC0F8D1
:100860005832DBE73D44954225D34FF0020E9918EC
:100870003B448B420FD3D0F85C32D21B8B422CBF4F
:10088000C0F85C32C0F85C121201002106EB0710C0
:1008900031F093F8C2E7D0F844C29D0803F0030496
:1008A0001CF8058064000EFA04F444EA08040CF80D
:1008B00005400133DDE7002CB1D0D0F84C22C90946
:1008C000515C03F007031941404601F00101FFF7B5
:1008D0004BFE04460028A2D031463A0131F02FF8F1
:1008E0003046FFF7EBFE9AE77003002010B5044690
:1008F0008AB003A8FFF7D8FD059B2046009308495E
:10090000DDE9032300F0A8FF069B20460193099B25
:1009100004490093DDE9072300F09EFF0AB010BDF3
:10092000283305084A3305082DE9F047DFF8189108
:100930004649D9F850220546002400F08DFF444E68
:10094000444FDFF81481D9F84832B4EB830F4FEAF3
:10095000830121D2A2062AD1A246D9F844024FEA45
:100960009A03C35C0AF00302520013419B0703D1B0
:100970000AF1010A5145F2D1AAEB04027F2A11D9EA
:1009800039462846920900F067FFD9F848322AF024
:100990003F04B4EB830F05D32846BDE8F0472F4949
:1009A00000F0A5BB31462846220100F055FFD9F8DA
:1009B0004422A308D35C04F003025200134103F065
:1009C0000303022B2CD0032B2CD0012B2CD1D9F8D4
:1009D00050222301D258424528D0214B9A4227D099
:1009E000204B9A4226D0204B9A4225D01F4B9A4248
:1009F00022D01F4B9A4221D01E4B9A421ED01E4B32
:100A00009A421DD01D4B9A421CD01D4B9A420CBFDE
:100A10004D22682228461B4900F01EFF013492E750
:100A20003D22F7E76D22F5E72E22F3E75422F1E7A6
:100A30004C22EFE74422EDE75322EBE74122E9E7BE
:100A40004622E7E74222E5E77003002090330508DD
:100A5000C7330508AB330508C8A105080CBA05085B
:100A600078940508488B050874A00508009F0508C0
:100A7000808705083487050854900508A890050864
:100A80001C9605089D9B05080346064A506A1A688D
:100A90004168C1F31E018A4202D3521A1A6070479C
:100AA0000068F5E77003002041F2055301448842D5
:100AB00004D398B2012838BF0120704710F8012BE9
:100AC00003EB43135340F2E7034B044A5A620022FC
:100AD000C3F8A421704700BF700300203801060846
:100AE0002DE9F04781460F46002943D0FFF7DCFF90
:100AF0008246214B5C6A0CB9204637E094F90730F6
:100B0000E668002B4FF0000506F1FF3616DB0136D4
:100B100004F11808B54215D32468ECE706EB050884
:100B20004FEA580808F106033A46484654F823109D
:100B300030F094FF0028CCBF45464646731B012B7E
:100B4000ECD8E4E7236933F815309A4510D163698E
:100B50005B5D9F420CD13A46494658F8250030F07B
:100B60004EFF28B96068C0F31E002844BDE8F08736
:100B70000135CFE70120F9E7700300202DE9F843A4
:100B800080460E46FFF7ACFF0246002840F09280F8
:100B9000FF2E03D949494A480CF052F9494C751CBB
:100BA000D4F8A40190B1D4E96A132B448B4229D91B
:100BB0002944FFF7EBFA0746D8B90246D4F8AC113E
:100BC000D4F8A401FFF7E2FAC4F8A471802D2F46EF
:100BD00038BF80273846FFF7BEFAC4F8A401D0BB5F
:100BE0002846FFF7B8FAC4F8A40198BB28460CF0D1
:100BF00063FFD4F8A8312B44C4F8A831D4F8A43149
:100C0000002BE3D041464FF00008D4F8AC31D4F8C3
:100C1000A47132461F4438462B44C4F8AC3130F03E
:100C20008EFE3146384607F80680FFF73DFF636ABF
:100C30008146D3E90253AB422AD36D000A2D38BF57
:100C40000A25C5EBC5001830FFF785FA48B9C4F886
:100C5000A401CBE72F460023C4F8A871C4F8AC3137
:100C6000D0E700F1180303EB8503626A036103EB2D
:100C70004503436153680260D268C3F31E03134403
:100C80004268C0F80C8063F31E02C0E9012560626F
:100C9000636AD3E903025B6922F810901E54636A09
:100CA000821D43F82270DA680132DA605A68C2F3B2
:100CB0001E0202441046BDE8F88300BFCF3305088A
:100CC000A88E05087003002010B5044630F0A9FE78
:100CD00001462046BDE81040FFF750BF07B5019020
:100CE00001A8FFF7D1FE019A036933F8120003B09F
:100CF0005DF804FB07B5019001A8FFF7C5FE019B55
:100D00004269D05C03B05DF804FB07B5019001A80F
:100D1000FFF7BAFE019B063350F8230003B05DF8DD
:100D200004FB13B5019001A80C46FFF7ADFE019B33
:100D30004269D25C063350F82300226002B010BD35
:100D40002DE9F8431D4600230746884616460360F2
:100D50000B6013602B60154BDFF854905C6A0CB18C
:100D60004C4505D12B68326813442B60BDE8F883ED
:100D70003B6801333B60E268D8F800301344C8F8A0
:100D800000306269E368D1188A4207D32046FFF732
:100D9000D1FC2B68246803442B60E0E7336812F829
:100DA000010B013303443360EEE700BF7003002002
:100DB000380106082DE9F8430D4B0E4F5C6ADFF849
:100DC0003880DFF838900CB1BC4201D1BDE8F8831F
:100DD000E36804F1180505EB8306B54201D32468E6
:100DE000F1E74146484655F8042B00F035FDF4E79D
:100DF0007003002038010608D7330508B4710508D0
:100E000030B50023202411F8012F0AB9027030BD3B
:100E1000120600F101051FD50BB1047028460B78AE
:100E2000124A03F07F036BB9013A12F8013F0546FD
:100E300013F0800F00F101000BD003F07F032B7043
:100E40000123E0E712F9015B002DFBDA013BDBB285
:100E5000E9E700F8013CE8E7012B04BF04702846ED
:100E60000B7800F8013B0223CDE700BFDE33050815
:100E700038B54468036821449942054610D9037B7C
:100E80001BB1002107480BF0DBFF01F1100424F037
:100E90000704083421468068FFF76DF92C60A860CC
:100EA00038BD00BFA88E050870B5044615460E462D
:100EB0001146FFF7DDFFD4E901302A4631461844D8
:100EC00030F065FD62682A44626070BD70B54668A6
:100ED0000446B14228BF31460D460121FFF7C8FF45
:100EE000A368681C5919721B184430F050FD6368E0
:100EF000A06801336360284470BD012938BF012117
:100F000038B504460025084621606560FFF718F9EA
:100F10002573A06038BD38B505460C460131FFF792
:100F2000ECFF6C6038BD0023C0E901320123016091
:100F30000373704738B514460546FFF7DEFF024BD2
:100F40002560636038BD00BFA90E0108037B10B5A2
:100F5000044613B98068FFF71BF90023A36010BD96
:100F600038B505461020FFF7EBF804462946FFF791
:100F7000C4FF204638BD10B5044648B1037B13B901
:100F80008068FFF705F92046BDE81040FFF700B97B
:100F900010BD000038B5037B04460D461BB100218F
:100FA00006480BF04DFF016880682944FFF7E3F81D
:100FB0002368A0601D442560184438BDA88E05082C
:100FC00038B504460D46FFF753FFD4E901301D4400
:100FD0006560184438BDD0E900239A4210B5044634
:100FE00002D10121FFF7D6FFD4E901320021D1540B
:100FF000A06810BD10B50C460121FFF7E1FF047099
:1010000010BD7F29F8B50C46CEB204D80121FFF7F8
:10101000D7FF0670F8BD06F03F06B1F5006FC1F3CB
:10102000871546F0800607D20221FFF7C9FF65F059
:101030003F0505704670EDE705F03F05B1F5803FCF
:10104000C1F3073745F0800508D20321FFF7B8FF49
:1010500067F01F07077045708670DBE70421FFF714
:10106000AFFFA40C07F03F0764F00F0467F07F07A1
:10107000047047708570C670CCE738B505460846E1
:101080000C4630F0CEFC214602462846BDE83840EA
:10109000FFF70ABF10B51446FFF718FF047010BD24
:1010A00010B51446FFF712FF047010BD43688B4261
:1010B00034BF0021591A4160704738B504461546BF
:1010C000626808468A4203D929448A4201D860608E
:1010D00038BDA368521A1844194430F058FC6268AD
:1010E000521B6260F4E70846114630F0FFBA70B553
:1010F000054608460E4630F094FC044620B10246F0
:1011000031466B6828689847204670BD2DE9F74F37
:1011100091468A469DF830100D9A11F0DF0F8046F7
:10112000A2EB090559D030295AD1C3F34721002930
:1011300059D05F290CBF0527042792FBF7F107FB65
:1011400011212D4E06F1050008BF304609B90135C1
:10115000013292FBF7F107FB11227E1EB21A8618AC
:1011600013F0200241D005EBD573A5EB63045D10AD
:10117000002D3EDDAB465F453A46A8BF5A46314694
:10118000D8F80430D8F8000001929847019AABEBE8
:10119000020BBBF1000FEEDCB9F1000F07D04A469D
:1011A0005146D8F80430D8F8000098474D44002C38
:1011B0000FDD2544A742B946A8BFA14631464A469D
:1011C000D8F80430D8F80000A4EB09049847002CA4
:1011D000F0DC284603B0BDE8F08F084E1027BFE7CB
:1011E00001270CAEBCE7064EF8E713F00104BFD0B0
:1011F0002C460025D0E700BFC8710508D37105084B
:10120000BC7105082DE9F04F93B01E46DDE91E873D
:101210009DF8743081460793CB070C4692461C9D7F
:101220000BD4880703D109687C4B994205D020462E
:101230000DF0FCFC440044F0010415F0210306D13C
:10124000079A302A03D1B845B8BFB8461F46204692
:1012500010F049FF00280DF1280B18DBA90712D563
:101260002B238DF828300DF129012B07F6B21CD560
:10127000BAF1020F0DD130200B4603F8020B701C9F
:101280004870194611E06A0701D52023E9E759465D
:10129000EBE7BAF1080F5DD1302328060B7045BF8C
:1012A00006F10E034B70013102310EA800230B90A2
:1012B0001020012FA1EB0B020B70C5F34721C8BF13
:1012C0000543069215F01002CDE90C03CDE9026149
:1012D0008DF82730059247D0CDE900A30DAA23460B
:1012E0000CA90BA810F0C8FD037882462D2B06D15F
:1012F0008DF827300D9B00F1010A013B0D93012F62
:1013000040F385800D9C059BBC42B8BF3C462BB189
:101310009DF8273003B10134069B1C44A0452EDD07
:1013200015F00103A8EB04042AD126461C4625F03B
:1013300001054EB120230093002301961A4648462A
:101340003749FFF7E3FE0646059B002B5CD13023AF
:1013500007933AE0BAF1100FA7D130200B4603F8FB
:10136000020B06F117008BE70AABCDE900A30DAA2B
:1013700023460CA90BA810F07FFD8246BFE700248E
:101380000026D4E7002426469DF827305BB10023D1
:1013900001224846CDE900320DF12701FFF7B6FEE4
:1013A00008F1FF380644069B63B100230122594629
:1013B000CDE900324846069AFFF7A8FE069B064490
:1013C000A8EB0308012FD8BF4746079B514600935F
:1013D00048462B460D9A0197FFF798FE06444CB1FC
:1013E00020230093002348461A460D490194FFF735
:1013F0008DFE06440B980EAB984201D0FEF7C8FE56
:10140000304613B0BDE8F08F30230793BCE7059B4F
:10141000002BB7D11C461E464746D6E72493050845
:10142000853606082DE9F04107468CB00846990735
:101430001E46DDF84C8064D413F0040F0CBF00236B
:1014400020230193149B03A90093134621220AF041
:101450003FFCF20504461FD52E2103A830F033FBD4
:10146000D0B9652103A830F02EFBA8B96E2103A8DE
:1014700030F029FB80B92E2104F130026A4402F8D1
:10148000241C3022631C30336B44023403F8242CB8
:10149000A3186B4403F8240C73060ED504F1300234
:1014A000631C0DEB02042522002104F8242C1C46A9
:1014B00003F130026A4402F8241C16F0100522D011
:1014C0009DF80C302F2B4FF000031ED8012203A9EA
:1014D0003846CDE90032FFF719FE054608F1FF381E
:1014E000013C0DF10D019DF848302246009338462D
:1014F0003346CDF80480FFF709FE28440CB0BDE860
:10150000F0812B239DE703A9EDE71D4603A9EAE738
:101510002DE9F04F0746144600268DB00B461D46B8
:1015200013F8012B0AB1252AF9D1A94207D2A5EB5C
:10153000010842467B6838689847294646440B783C
:10154000002B00F080814FF0200A002301310A4671
:1015500012F8015B15B94FF00A0C18E02D2D03D1DC
:1015600043F001031146F2E72B2D02D143F00203B1
:10157000F8E7202D02D143F00403F3E7302D23D107
:10158000AA4643F01003EDE70CFB0525303D8846E5
:1015900011F8012BA2F130000928F5D92E2A3BD1F0
:1015A00098F801202A2A11D00A460A2000219046E4
:1015B00012F801BBABF1300CBCF1090F0AD800FBEB
:1015C00001BBABF13001F2E70025C4E754F8041B7E
:1015D00008F1020821EAE17B98F800206C2A08BF94
:1015E00008F1010898F80090B9F1000F00F02B8184
:1015F000B9F1780F09D8B9F1570F10D8B9F1470FE1
:1016000056D8B9F1440F00F20B81012241467B68A4
:101610003868984701368DE04FF0FF3BDCE7A9F1D1
:101620005802202AF1D801A151F822F0B71601087A
:101630000B1601080B1601080B1601080B16010802
:101640000B1601080B1601080B1601080B160108F2
:101650000B1601081F17010841170108B7160108EA
:101660002118010821180108211801080B1601088A
:101670000B1601080B1601080B1601080B160108C2
:101680000B1601080B1601080B160108B716010806
:10169000531701080B1601087B1701080B160108E8
:1016A000B71601080B1601080B160108B71601083A
:1016B000B9F1500FA9D154F8042BB9F1640F1146B8
:1016C0006DD0B9F1750F0CBF0A2010204FF0000C3F
:1016D000B9F1640F8DF81FC06AD1624561DA2D211E
:1016E0008DF81F10514229F00F0BABF10F0B5FFA71
:1016F0008BFB0DF13009ABF10A0BB1FBF0FC00FBE9
:101700001C12092A8CBF5A44303209F8012D08AA4C
:1017100091458E46614653D07045EED950E054F85D
:10172000042BCDE900A542B1042249493846FFF710
:10173000EDFC064408F10101F0E605224549F5E714
:1017400054F8042B08A98DF82020CDE900A501222A
:10175000ECE708A954F8040B0593FFF7E2FABBF194
:10176000FF3F0146059B04D0089A934538BFCDF84A
:1017700020B0CDE900A5089AD8E754F8049B05935A
:10178000484630F04EF9BBF1FF3F0246059B02D0C0
:10179000584528BF5A464946CDE900A5C6E70A2064
:1017A00094E713F0020F29D04FF02B0C8DF81FC0D7
:1017B000002A98D14FF030020DF12F098DF82F201B
:1017C00013F0100B9DF81F201ED03AB301223846AB
:1017D000CDE900A20DF11F010593FFF797FC8346A9
:1017E000059B013D0CAA49463846CDE900A5A2EB70
:1017F0000902FFF78BFC83445E449BE713F0040F60
:10180000D6D04FF0200CD1E7002AEBD008A98945AB
:10181000E8D909F8012C09F1FF39E3E79346E1E73C
:10182000073424F00704F4E80201059340F0DCF9E2
:101830004A460146CDE9015B3846059BCDF800A03C
:10184000FFF7F0FD75E730460DB0BDE8F08F00BF43
:10185000A8710508AD7105080EB403B503AA52F8C6
:10186000041B0192FFF754FE02B05DF804EB03B0D5
:101870007047034693F900200078002A0ADA4022D4
:1018800000F07F00104206D113F8012F02F0C001D2
:10189000802904D0704720EA02005208F2E702F0E3
:1018A0003F0242EA8010EFE7431C184602780133FA
:1018B00002F0C002802AF8D0704703460020994207
:1018C00000D8704711F8012D02F0C002802A18BF1D
:1018D0000130F4E703460144002099421A4600D83B
:1018E00070471278013302F0C002802A18BF01301D
:1018F000F3E700007F289DBF024B185CC0F3400057
:1019000000207047E37105087F289DBF024B185CDB
:10191000C0F3C00000207047E37105087F289DBF19
:10192000024B185CC0F3800000207047E37105088B
:101930007F289DBF024B185CC0F3801000207047C9
:10194000E37105087F2809D8064B1B5C13F00C0FC8
:1019500006D1A0F15F0358425841704700207047FC
:1019600001207047E37105087F289DBF024B185C7A
:10197000C0F3001000207047E37105087F289DBF69
:10198000024B185CC0F3401000207047E37105085B
:1019900008B50246FFF7E8FF00B12032104608BD47
:1019A00008B50246FFF7EAFF00B1203A104608BD2D
:1019B0003038092884BF20F02000073870470246DD
:1019C00010B50144E5240020914203D8B0FA80F01C
:1019D000400917E012F8013B30B103F0C003802B3F
:1019E00011D10138C0B2EFE7BF2B09D9F72B09D8C5
:1019F000D80800F0060044FA00F000F00300E3E726
:101A00001B06E1D510BD0020FCE7023981420B46E0
:101A100003D31A880239002AF8D00233181A40106A
:101A20007047B2EB131F70B505464FEA131615D970
:101A3000901B024603F00F0401EB46010E46012AFB
:101A400031F8023B18BF3368013A23FA04F39BB222
:101A500025F8023BF2D103B9013870BD0020FCE744
:101A6000F0B500242646059FD21BA74210D10024C2
:101A700000EB470C01EB4701A24214D10CEB4203EF
:101A80001EB1012102332CF81210181A4010F0BDBB
:101A900031F8145033F814C06544354420F814501C
:101AA0002E0C0134E1E731F8145035442CF8145071
:101AB0002E0C0134E0E7F0B400252C46049FD21B25
:101AC000AF420BD1002300EB470601EB47059A42DA
:101AD0000FD106EB4201F0BCFFF797BF31F815605C
:101AE000344433F81560A41B20F815402414013544
:101AF000E6E735F813100C4426F81340241401339C
:101B0000E5E72DE9F0438446DDE9087615464FF612
:101B1000FF78079CDDF828E00239A4EB020955B9EB
:101B200000EB42011FB10123023120F81230BDE861
:101B3000F043FFF76ABF31F8024F013D44442644A9
:101B400005EB0904AC428EBF4FF6FF7433F8024B2D
:101B50004444744486EA040E1FFA8EFE77442CF83F
:101B6000027B4FEA144E360C3F0CD8E7022938BFEF
:101B7000022138B5044680680D4618B12368B1EBE0
:101B8000930F07D96900FEF7F6FA2368A06065F3A2
:101B90009F03236038BD38B504460C20FEF7D0FA09
:101BA000054623682278C3F39D0002F0010223F06A
:101BB000030313432B60636840006B60FEF7C0FAB9
:101BC000A8602268A168C2F39D0252002FF0B7FE00
:101BD000284638BD994210B511D313D800EB410007
:101BE00002EB410209B9084610BD30F8023D32F857
:101BF000024D1B1B002B02DB04D10139F2E74FF031
:101C0000FF30F1E70120EFE710B5044638B18068F6
:101C1000FEF7BEFA2046BDE81040FEF7B9BA10BD87
:101C200038B50C4605460221FFF7A0FF002CB4BFD3
:101C3000012200222B78A8BF214662F300034FF057
:101C400001022B70AB68B8BF6142023B23F8021F50
:101C5000090C104602F10102F8D1686038BD00237A
:101C6000C0E900338360704728B103789B0702D432
:101C70008068FEF78DBA704738B505460C4649684E
:101C8000FFF774FF22782B78A86862F300032B70AB
:101C90006368A1686B606268BDE8384052002FF04D
:101CA0004EBE0A4629B90178426062F30001017014
:101CB0007047FFF7B5BF08B5FFF7D1FFBDE8084093
:101CC000FFF7EFBF920042F002020260002210B460
:101CD000C0E9012110BC1946FFF7E3BFF8B514466F
:101CE0001D469DF8187004210646FFF73FFF224667
:101CF0002B4627B1002D0CDA624265EB45033178A3
:101D000067F3000131700021716052EA030102D1D2
:101D1000F8BD0027F3E7D6E901104C1C746020F8E9
:101D20001120120C42EA03421B0CEEE70378CA0FA3
:101D300062F300032DE9F0410370C1F30F4313F484
:101D4000FF43074607D13B786FF300033B70002346
:101D50007B60BDE8F081B3F5FF4FF4D0C1F3C7530A
:101D6000A3F17F05002DEEDB04D1BDE8F041012198
:101D7000FFF756BFB3F16F0848BFA3F16008C1F386
:101D80001601162D4FEA281841F4000421DCC5F194
:101D90001705EC4000252E4641463846FFF7E6FE83
:101DA000C7F8048026B10021B86872002FF005FE44
:101DB00045B1BB6804FA05F2C5F1100523F81620F9
:101DC000EC400136B045C4D0BB6823F81640240C63
:101DD000F7E7B3F1960605F1090548BFA3F18706B9
:101DE00005F00F053611D7E72DE9F843044698466C
:101DF0000D468F18C2F35B02511C089EFFF7B6FE1A
:101E00002378294668F30003237000231FFA86FC19
:101E10006360B942084602D3401BBDE8F8830278EC
:101E20000131A2F13003092B05D9A2F14103192B8D
:101E300014D8A2F13703B342EED2D4E901E0F04660
:101E40008146B8F1000F10D100EB4E0213B120F81B
:101E50001E300232121A52106260DAE7A2F16103F8
:101E6000192BD9D8A2F15703E5E7B9F8002008F1FA
:101E7000FF3802FB0C3329F8023B1B0CE1E7F8B5F5
:101E8000044615461E46C1B14FF0FF37531E1E448F
:101E9000E9000F3109092046FFF768FE0021237889
:101EA00061606FF3000323704DB9D4E9011000EBBA
:101EB0004101FFF7AAFD6060F8BD0127E8E70023B4
:101EC0000F290ADC3278013D02FA01F243EA0203EB
:101ED0009BB201F108013E44F2D162681039501CF6
:101EE0006060A06820F81230DEE738B50B7805781E
:101EF000044603F0010305F00100181A08D1D1E9E6
:101F00000132D4E90110FFF765FEEB0748BF4042FC
:101F100038BD884210B5044601D0FFF7ADFE2378E6
:101F20006FF30003237010BD884210B5044601D042
:101F3000FFF7A2FE63683BB12378C3F30002C2F14E
:101F4000010262F30003237010BD88421FB50446EE
:101F500001D0FFF791FE626862B901212046FFF7C8
:101F600005FE0123A26813806360237843F0010318
:101F7000237010E02378D9070FD56FF30003237087
:101F80000123A168ADF80E30009308460DF10E0351
:101F9000FFF791FD606004B010BD2046511CFFF7B3
:101FA000E5FDD4E9012101230846ADF80E30009388
:101FB0000DF10E03FFF754FD6060D6E72DE9F843FD
:101FC0004B6805460E46144603B12AB931462846E9
:101FD000BDE8F843FFF750BE02F10F014FEA1118B8
:101FE00003EB1111FFF7C2FDD6E9013108EB03073E
:101FF000A86807F1004214F00F0402F1FF3208BF95
:10200000102400EB420001EB430E814619464FF0CD
:10201000000CC4F11004E9B96FF0010253432CFA2B
:1020200004F4C218C452C8F1010302EB430308F1DF
:10203000FF32184652002FF0C0FC831E17B133F850
:1020400017209AB16F6032782B7862F300032B70FF
:10205000BDE8F8833EF8022D013942EA0C0C2CFA57
:1020600004F229F802294FEA0C4CD4E7013FE5E7D6
:10207000F0B50E4649680546144685B001B132B93F
:102080003146284605B0BDE8F040FFF7F5BDFFF743
:102090006DFDD6E901212346A868FFF7C2FC686000
:1020A00031782B78024661F300032B70DB072DD5C6
:1020B000002370682109ADF80E30984201D08B42A0
:1020C0000FD1884222D9B36804F00F0433F81110FD
:1020D000012303FA04F4013C214213D0ADF80E3081
:1020E00008E0B76837F8137057B101238842ADF89C
:1020F0000E30E8D80123A96852B90B806B6005E067
:102100000133DAE7BDF80E30002BF3D105B0F0BD96
:10211000009308460DF10E03FFF7A2FC6860F5E797
:1021200073B50C461646D2E901320546D4E90110D2
:10213000FFF750FD0028BEBF234634461E462378D5
:10214000327861685340DB071BD428460131FFF722
:102150000DFD7368A8680093B368D4E90121FFF707
:102160007FFC686023786A68C3F30003002A0CBF11
:10217000002303F001032A7863F300022A7002B0FF
:1021800070BD2846FFF7F2FC7368A8680093B36837
:10219000D4E90121FFF78FFCE3E7F7B50D461646BA
:1021A000D2E901320446D5E90110FFF713FD0028FA
:1021B000BEBF2B4635461E462B783278B8BF012766
:1021C00083EA0203A8BF0027DB07696814D520460D
:1021D0000131FFF7CBFC7368A0680093B368D5E9C1
:1021E0000121FFF73DFC60606268237882B962F3E9
:1021F0000003237003B0F0BD2046FFF7B7FC7368FF
:10220000A0680093B368D5E90121FFF754FCEAE721
:102210002A7802F00102002FE9D0C2F10102E6E7BC
:102220002DE9F04F15464A686B680E469A423EBF4C
:102230000B462E461D4633780446DB07716885B091
:1022400021D42B7813F001071DD1FFF78FFCD5E9BE
:10225000011C3B46A068B66899420BD100EB4101D6
:10226000FFF7D3FB237860606FF30003237005B0A2
:10227000BDE8F08F36F813203CF813502A4020F8C0
:1022800013200133E8E720460131FFF76FFC96F891
:1022900000902B7809F0010E89EA0307FF4307F04D
:1022A000010247F30007BFB249F3000902971FFA82
:1022B00089F70197B768D6F804C0A068023F009775
:1022C00082466746D5F804B003F00108ABEB0C0B6F
:1022D00043F30003A9689BB2CDF80CB0AFB900EB93
:1022E0004C011AB10123023120F81C30FFF78DFB9D
:1022F000606033782A78C3F30003C2F3000213400E
:10230000227863F300022270B1E7DDF80090013F0C
:1023100039F802BFCDF80090DDF804908BEA090B84
:10232000DDF80C90DE4409EB070BBB458CBF9B46E8
:1023300031F802BBDDF8089098BF8BEA030BD84454
:102340000EEA080B8BEA090B1FFA8BFB5A442AF89A
:10235000022B4FEA18484FEA1E4E120CBEE72DE939
:10236000F84F16464A6873680D469A423EBF0B46C0
:1023700035461E462B780446DB07696831D432782F
:1023800012F001072DD1FFF7F1FBD6E9013E3A46E5
:10239000A9686D68D4F808C0ED1A934212D10022E2
:1023A00001EB43010CEB4303954214D103EB4503CE
:1023B000A3EB0C035B10636023786FF300032370BF
:1023C000BDE8F88F31F812003EF8126030432CF867
:1023D00012000132E1E731F8120023F81200013255
:1023E000E2E720460131FFF7C1FBD6E9013795F856
:1023F00000C06968A068AD6832780CF0010E4CF33B
:1024000000068246A5F1020C4FF001090D4602F0CC
:10241000010842F30002B6B292B2A3EB010B45B938
:1024200000EB4101FFF7F1FA2378606043F001030C
:10243000C5E73CF8023F013D73409E440BEB0503AA
:10244000AB428EBF134637F8023B534098444EEAE6
:102450000803DB439BB24B442AF8023B4FEA18487F
:102460004FEA1E4E4FEA1349D9E7F0B516464A68BF
:1024700073680C469A423EBF0B4634461E46277888
:10248000337805465F4017F00107616885B03AD19F
:10249000FFF76CFB237813F0010328D1D6E9012C58
:1024A0006168A868A768891A9A4211D1002307EBCE
:1024B000420700EB4202994213D102EB4101FFF7C0
:1024C000A4FA2B7868606FF300032B7005B0F0BDA1
:1024D00037F813403CF81360744020F81340013380
:1024E000E2E737F8134022F813400133E3E7CDE980
:1024F000027701977368A8680093B368D4E9012153
:10250000FFF7FFFADDE70131FFF730FB3378A8680A
:10251000DB4303F0010303932378DB4303F0010360
:1025200002930123019373680093B368D4E90121F6
:10253000FFF7E7FA2B78686043F00103C5E72DE960
:10254000F04F4B6804460E46154685B00BB15368F4
:1025500043B923786FF3000323700023636005B051
:10256000BDE8F08F81422DD1FFF715FBA54206464D
:10257000074600D105466B68716820461944FFF78D
:10258000F5FA22680021C2F39D025200A0682FF0E4
:1025900014FA0022D4F808E01146F446B368D6F8DD
:1025A00004900193AB680EEB490802936B680393A8
:1025B000039B93422FD0019B49460093ACF102004C
:1025C000002318E0824204D1FFF7E5FA05460746EA
:1025D000D1E70027CFE730F802AF013953449B46DB
:1025E000009B33F802AB0093029B33F8123003FBDD
:1025F0000AB303801B0C0029EDD14146881C13B19E
:102600000146A8F80030A1EB0E01804649100CF1FC
:10261000020C0132CCE7384661602A7833785340A7
:10262000227863F30002227005B0BDE8F04FFFF797
:10263000EBBA4B6870B50546144613B11378DA0748
:1026400006D52B786FF300032B7000236B6070BDF1
:10265000636823B9BDE870400121FFF7E1BA08467D
:10266000FFF799FA06462046FFF795FA012104463E
:102670002846FFF7D5FA636883B1A3681B88DB0798
:1026800004D5324629462846FFF759FFD4E90121EF
:1026900001230846FFF7C5F9606038B93046FFF7F7
:1026A000B3FA2046BDE87040FFF7AEBA3246314675
:1026B0003046FFF744FFDEE72DE9F04F9046054630
:1026C00000260C4651688FB001310293FFF74EFA95
:1026D000D8F80420002101325200A8682FF06DF9CB
:1026E0002B786E606FF300032B70D8F8041020462F
:1026F0000131FFF73BFA41462046FFF7BDFA029B46
:10270000A768D3F808A05B68D4F804900193AB687D
:102710005246039349463846019BFFF75BFA00286F
:1027200032D10123039A606013806B602378616863
:10273000C3F3000200290CBF002202F0010262F381
:102740000003029A237098F8003012785340DB0798
:1027500017D56B682A78003B18BF012363F300028A
:102760002A7071B14FF0FF310BA8FFF7A4FA294688
:1027700028460BAAFFF7D4FC21462046029AFFF711
:10278000CFFC0FB0BDE8F08F01DA6E60CEE7019BA1
:1027900003F10042013A3AF812304FEA420E1804AF
:1027A00006F1010150D50021BC4609F1010327F8CB
:1027B000191005936360B3B207EB490BC3F1100026
:1027C0000BF102090490CC4542D33AF812209A400A
:1027D0000492019A012A09D90AEB0E0232F8022C5E
:1027E000C3F11001CA40049911430491019A05995B
:1027F000AAF1020A881A6860039A00F100400138C1
:1028000002EB400206920EF1020209926268059202
:102810000599019A8A4227D3002001F1004B0BF160
:10282000FF3B07EB4B0BC3F110065F4573D96FF00D
:1028300000416B682BB103985A1830F81220002A17
:1028400073D06FF0004175E05B000E469BB2A6E7C7
:10285000BCF8006006FA03F001432CF8021B04994F
:1028600026FA01F189B2AEE70021BBF800203BF85F
:10287000026C8E4646EA0246049AB6FBF2F6099AC4
:10288000ABEB02021046CDE9072A83450DD8BBF811
:1028900000201144C9BB069AABF1020B22F8026971
:1028A0000692059A013A6260B0E7DDF820C0B0F800
:1028B00000903CF8022F9A4042EA1E4E1FFA8EF218
:1028C0007243CDF820C01FFA81FCE1441FFA82FC5C
:1028D000120CA9EB0C0CC2EB214220F802CB02EB4C
:1028E0002C41D2E739F8020F984040EA1E4E1FFAF9
:1028F0008EF00244BCF8000002442CF8022B120CAB
:10290000E345EFD81144013EC4E70022D146964684
:10291000DDF81CC0F4E7BBF8002042FA03F10143E4
:10292000B2402BF8021990B27FE7013B6B6080E761
:10293000013B63606368002B3FF4F8AE5A1837F828
:102940001220002AF4D0F1E6F0B51F464B68044689
:102950000D46164685B04BB11378DA0706D47B686E
:10296000012B0BD1BB681B88012B07D123786FF398
:10297000000323700023636005B0F0BD01212046F1
:10298000FFF74EF97368002BF6D02846FFF703F9DE
:1029900005463046FFF7FFF8064601A8FFF75FF946
:1029A0007368B3B1B3681B88DB070AD52A46214692
:1029B0002046FFF7C4FD3B462246214601A8FFF70B
:1029C0007BFED6E9012101230846FFF72AF8706053
:1029D00048B901A8FFF748F92846FFF715F930462E
:1029E000FFF712F9C8E72A4629462846FFF7A7FD50
:1029F0003B462A46294601A8FFF75EFED0E7D0E90C
:102A000001210346002010B501EB4202914204D39C
:102A10001B78DB0748BF404210BD32F8024D44EA44
:102A20000040F3E7002330B5D0E9012404EB420273
:102A3000944206D302780120D20748BF5B420B6064
:102A400030BDB3F5004F04D232F8025D45EA0343CE
:102A5000EEE70020F4E72DE9F74FDDF830C00F4630
:102A6000019221B30CEB03050126D0E90189002175
:102A70001A46B2468E46B8F1000F1AD101990029C4
:102A80004AD0002A48D1002B46D0002F40D09CF8D5
:102A9000003046B1DE430378C6F3C01603F00103ED
:102AA000F61A18BF0126304603B0BDE8F08F654620
:102AB000DAE739F8024B0EF1100E44EA0141BEF19B
:102AC000070F02DC08F1FF38D5E790F800B08CB2B0
:102AD0001BF0010F06D0E443E4B2A2441FFA8AF4CB
:102AE000CAF3072A52B93EB1E6B2B6FA86F67609BB
:102AF000AEF1080E090AE2E71646F9E7E4B227B19B
:102B000005F8014C013D013AF2E705F8014BFAE7FF
:102B1000634413F8013CBCE7037813F0010F14BFC2
:102B2000FF210021002F14BF604628462EF045FFEC
:102B3000B9E72DE9F041D0E9015704464FF08F483D
:102B4000002007EB4505AF4206D32378DB0748BFDB
:102B500000F10040BDE8F08141463FF0A3F9064690
:102B600035F8020D3FF04AF931463FF093F8EAE7B5
:102B70000A292DE9F74F15460CBF032204224468A9
:102B8000804689469DF830A00D9E0092A4B98DB173
:102B90003346013D15F8011F184641B93023037033
:102BA000002300F8013F801B03B0BDE8F08F03F85D
:102BB000011BEFE73046F1E7640020460193FDF783
:102BC000BFFA22460746D8F808102EF0B8FEB346E2
:102BD0003046019B3A19A3F13A0C0023941EA742F8
:102BE000A64629D95C463033392B88BF634404F8A4
:102BF000013B3B469A429E4629D83846FDF7C8FA23
:102C00005DB128462EF00DFF2A1859461346AB42F7
:102C100030D8954288BF0020044498F80030DB0784
:102C200044BF2D2304F8013B3346621E9A4226D846
:102C30000023A01B2370B7E7BEF800E04EEA034371
:102C4000B3FBF9FE09FB1E3324F802E9C7E7BEF81F
:102C5000001002330029CDD0BAF1000F08D000993E
:102C6000231A8B4204D10BF1020420468BF801A0F9
:102C7000A346B2E713F8017D01F8017FC7E7197891
:102C8000107803F8010B02F80119CFE7D0E90232FE
:102C900093423DBF5A1C826018784FF0FF30704756
:102CA000036810B5013B0333044602D84068FDF7C2
:102CB0006FFA2046BDE81040FDF76ABAF8B5054640
:102CC00010200C461F461646FDF73AFA054BC0E9A0
:102CD000007484603444C4606B60034B2860AB6054
:102CE000F8BD00BF8D2C0108A12C0108026910B5A8
:102CF0000A2A044635D1836A013383620123A2691B
:102D0000E36263696261226F2361002A31D0616EE0
:102D10008A422FBF0022501CA16E206738BF8A5CF8
:102D2000A2613BB9E26963662261226A236762613C
:102D3000626AA26163690D2B08D10A22A3696261EC
:102D4000934203D1D4E901039847A061A3690133F9
:102D500006D163695A1C03D00A2B1CBF0A23A36146
:102D600010BDC36A092A04BF073323F007030133E8
:102D7000C5E7D4E901039847A061DBE70369272B86
:102D80002BD0222B29D0A3F1620113291ED8174A78
:102D9000CA40D2071AD54269272A1ED0222A1CD03F
:102DA000722B1CD1662A06D18269272A15D0222AC5
:102DB00013D0722B15D14369622B0CD1806927285F
:102DC0000BD0A0F12203584258417047662BF0D136
:102DD0004269722AE8D00020704701207047662BB4
:102DE000F6D0622BF7D14369722BE6E71100090098
:102DF00038B504460D462069431C02D100252846FB
:102E000038BD0A2807D115B1636B002BF7D02046D7
:102E1000FFF76CFFEFE7FEF76DFD0028F7D12369A0
:102E2000232B08D12046FFF761FF23695A1CE2D00B
:102E30000A2BF7D1DFE75C2BE0D163690A2BDDD1E8
:102E40002046FFF753FFE2E72DE9F04F436E0446BB
:102E500085B0A3B1036F93B929216030FEF7CAF89A
:102E60002369E36163692362A3696362A36E1A78CD
:102E700022615A7862619B78A36103232367002350
:102E8000012163652046FFF7B3FFA36A266B6364E5
:102E9000E36A002EA36407DA0723013684F84C3076
:102EA000266305B0BDE8F08F04D00623013E84F808
:102EB0004C30F5E7002837D031462046FFF798FF21
:102EC00005236FF0004284F84C30E56AD4E90F30F6
:102ED000991830F81110013D8D42E2D019D9A16B3B
:102EE0008B4207D308314900FDF745F9A36B2064F5
:102EF0000833A363D4E90F32591CE16322F813505D
:102F0000236B01332363CCE7013BE363236B013B7A
:102F10002363E36B991830F811108D42F4D3C0D0BD
:102F2000022384F84C30BCE725696B1C02D184F87D
:102F30004C00B6E72046FFF721FF8046002800F04E
:102F4000D78184F84C602369752B21D0622B06D180
:102F500063690025722B1FD1C14602271EE0722B28
:102F60000CD16369622B4FD0662B0CBF4546002500
:102F7000C14614BF012702270B2310E0662B45D161
:102F800063694546722B0CBFC1464FF00009F0E75C
:102F900000250127A946EFE7A94601270C2394F84D
:102FA0004C20002A36D184F84C303FB12046FFF740
:102FB0009DFE022F02D12046FFF798FE236920468E
:102FC000222B14BF272322230093FFF78FFE2369B0
:102FD000009A934221D163699A421ED12046FFF79D
:102FE00085FE2046FFF782FE4FF0030A35B1636E7F
:102FF00023B9B44904F16000FEF73FF8002304F15F
:10300000500704F1600B19E00025A5E700253746BD
:10301000A946B1E79A42C8D043E74FF0010AE5E775
:103020000099914236D1013338460193FDF7E9FF0B
:10303000019B20460193FFF759FE019B2269511C19
:1030400000F05081BAF1010F02D10A2A00F04A8142
:103050005345E5D3194604F15000FEF727F8012146
:103060002046FFF7C5FE2046FFF788FE00287FF4C4
:103070006AAF16E72046FFF739FE21697B2920D188
:103080003846FDF7B7FF2046FFF730FE7B21384674
:10309000FDF7B0FF21690DB17B29EBD05C2940F031
:1030A0001C8120460191FFF721FE23690199B9F1A6
:1030B000000F4DD001933846FDF7A3FF019B194641
:1030C000E3E028215846FDF795FF0022636E216951
:1030D000481C0FD032BB3A290CD07D290AD02129B7
:1030E00020D160697238012821D8A0693A2801D01E
:1030F0007D281CD1D4E91921881810F8010C3D282D
:1031000007D1D21A19443846FDF7CEFE636E013B53
:10311000636658462921FDF76DFF2C215846FDF7BF
:1031200069FFB3E721F020005B280CD1013258463B
:10313000C9B2CDE90132FDF75DFF2046FFF7D6FDAC
:10314000DDE90132C3E75D2808BF02F1FF32EEE797
:10315000782B06D85B2B0BD8222B75D054D80A2B92
:1031600050D0A3F13001072900F2B0800323A2E080
:10317000A3F15C021C2AF4D801A151F822F000BF8F
:1031800049320108633101086331010863310108E4
:1031900063310108F531010821320108633101086A
:1031A00063310108633101083132010863310108DC
:1031B000633101086331010863310108633101089B
:1031C00063310108633101082932010863310108C4
:1031D00063310108633101081D32010863310108C0
:1031E00025320108353201082D320108633101080A
:1031F0009D320108072194F84C300B2B69D13846D9
:10320000FDF7FFFE002314E7552B13D0A9D8272B79
:103210001AD04E2BA5D12C480AF030FE0D21EAE73A
:103220000821E8E70921E6E70A21E4E70B21E2E7C4
:103230000C21E0E794F84C200C2A07D15C21384699
:103240000193FDF7DEFE019B1946D4E7752B0CBFF9
:1032500004230823002116E0204603930191FFF781
:1032600045FD226910460292FEF762FB002800F03D
:103270004F810199029A090110460191FEF798FBCE
:103280000199039B0144013BE6D2481CBAD0B1F539
:10329000881FB0D3012384F84C30B3E70223D9E769
:1032A0002046CDE90113FFF721FD22690199303A4B
:1032B000029B02EBC1016269303A072AE5D8013B63
:1032C000EED1E2E7A8720508B17205085C2101930E
:1032D000F1E6FF29DED80C2BDCD13846C9B2FDF768
:1032E00089FE8FE753453CBF032284F84C20B1E6AA
:1032F0002846FEF709FB054620691DB95F2801D065
:103300007F283ED9082304F1500584F84C30C1B21F
:103310002846FDF76FFE2046FFF7E8FC2069421CB7
:103320001BD12846FDF757FE002506467B4F304649
:1033300057F8041B2EF07CFB00281CD10E35EDB293
:10334000112D84F84C507FF4ACAD754BD3F8B031EF
:10335000002B0CBF10230E23E3E5FEF7D5FA40B98E
:1033600020695F2805D07F2803D8FEF7D7FA002808
:10337000D7D0217CCCE7FFF694AD0135242DD6D1F2
:103380008FE5FEF7CBFA68B321692E2935D10A23E0
:1033900084F84C3004F150063046FDF732FE2046EA
:1033A000FFF7A4FC0A272069431C3FF47AAD002DE7
:1033B00039D120F02003452B35D16521304684F8E2
:1033C0004C70FDF71EFE2046FFF790FC21692B296B
:1033D00001D02D29E7D13046FDF713FE2046FFF737
:1033E00085FCE0E723692E2B04D16069FEF796FA8D
:1033F0000028C9D100264B4D35E00923302984F837
:103400004C30C7D1656945F02005A5F16203162B44
:1034100097BF454D0125DD40ED4398BF05F00105FF
:1034200085F00105B6E7FEF76FFA28B121692E296C
:103430000DD184F84C70CEE72069FEF76FFA0028B2
:10344000F4D123692E2BF1D05F2BC7D029E521F0D1
:1034500020034A2BBFD1ECE7652F01D0632F00D1A9
:103460000135013601352F7817B12369BB42F3D1FD
:103470002046FFF73BFC0FB9012352E5212F07D16E
:1034800023693D2BF8D12046FFF730FC392348E56E
:103490002E2F0FD123692E2B02D163692E2B01D041
:1034A0005C233EE52046FFF721FC2046FFF71EFC8B
:1034B0000D2336E53346033515F8027C632F0FD014
:1034C000652F0DD0194AD35C03F0FD02542A84F80D
:1034D0004C3001D0582B13D1636B01336363E0E4AC
:1034E00015F8012C21690136914207D12046FFF7DA
:1034F000FDFB3346652FE5D00235DDE7632FFAE7A4
:10350000552A02D0592B7FF4CCAC636B013BE5E725
:103510000123014684F84C306DE600BF7473050842
:1035200070030020637205080120400048730508FD
:103530007FB5064601AD742085E80E00FCF700FE5D
:10354000034643F8046B044695E8070083E8070048
:1035500001236FF001020025C4E90A320A22142077
:10356000C4E90E23C4E90C55FCF7EAFD20212064D0
:1035700004F15000FDF7C1FC294604F16000FDF79D
:10358000BCFC236C204625671D80C4E905552561D8
:10359000FFF7ACFB2046FFF7A9FB2046FFF7A6FB91
:1035A0002046FFF751FCA36C012B06D094F84C3059
:1035B000052B1CBF062384F84C30204604B070BD98
:1035C00030B5054685B001AC2046FFF777FB94E89F
:1035D0000E002846FFF7ACFF05B030BD30B50446FD
:1035E00085B001AD0146284621F018FF95E80E0090
:1035F0002046FFF79DFF05B030BD10B5044690B1E1
:10360000C3684068984704F15000FDF79FFC04F13F
:103610006000FDF79BFC206CFCF7BAFD2046BDE87E
:103620001040FCF7B5BD10BDD0E90432013B036189
:1036300052F823007047C94303691944436953F89A
:1036400021007047F8B5446A06460D46BCB1D4E97E
:1036500000132B448B4223D905F108030022204696
:103660001944FCF793FD0246B8B961682046083159
:10367000FCF78CFD63682360336A63603462102D4D
:103680002F4638BF102707F10800FCF759FD00232B
:10369000076043600446706202E023682B442360A5
:1036A00060680834054444F8045C2044F8BD38B52B
:1036B0000D460C211446FFF7C5FF4FF49D720560BF
:1036C000C0E9012438BD38B5D0E903329A42044636
:1036D0000D4608D3103399004069FCF74CFDE368B0
:1036E00060611033E360D4E90432591C216142F86F
:1036F000235038BDF8B504461D4609C883420F461D
:10370000164608D31030C100A068FCF734FD2368CA
:10371000A06010332360D4E90103421C626053F8B7
:10372000301003EBC00267F3170143F83010D67076
:103730005560F8BD10B48469CAB20023616C10BC36
:10374000FFF7D8BF10F00102034604D040F0010398
:103750000B6001207047A8B110F0030013D11A7953
:103760003A2A11D19B6813F001000B60F1D19A073E
:103770000AD11868054B9842EBD0054BC31A584242
:103780005841704770471046704700BF24930508A2
:103790005490050810F001021CD110F003030CD066
:1037A00000F00F03062B15D00A2B11D100090D389C
:1037B00003288CBF00200120704770B102793A2A9B
:1037C00008D02D2A08D18068B0FA80F040097047EF
:1037D000104670470120704718467047C20702D54F
:1037E00040F001007047830710D0030900F00F007C
:1037F000062803D1D80040F002007047A3F10E0064
:10380000022809D8064B53F82000704730B10379DD
:103810003A2B03D1806870470248704702487047CE
:1038200060740508E89A0508C0A1050838B5054682
:103830000C46FFF7AFFF38B12846FFF7CFFF0BF07C
:103840003DFB031B5842584138BD0000F0B58DB018
:10385000044668460E4617461D46FCF73DFC10B16F
:1038600000200DB0F0BD3A46314620460AF040F93E
:103870000446FCF707FCA30703D12268024B9A42D7
:10388000EED001202C60ECE7248905082DE9F041F9
:1038900005460F461446164696B93146204612F0A4
:1038A0002DFF014600F10808ACB90A462846394602
:1038B000FFF7FDFE01462846FFF705FF012008E05F
:1038C000013E31462846FFF7B6FEFFF763FF0028AA
:1038D000E2D1BDE8F0812846FFF7A6FE0646FFF7D5
:1038E0007DFF013C48F82400002EDDD0B307DBD17A
:1038F000686A00F108039E42D6D3426813449E4290
:10390000D2D273681B0A0233A2EB83034360CBE776
:10391000F7B58669054696F84C200F46082A1FD150
:10392000D6E91510FDF72AF9902F04460ED1C100F3
:10393000002241F0020105F128000AF069FE28B1D9
:103940004268D30720D542F0010002E0200140F098
:1039500002000146284603B0BDE8F040FFF7B3BEC1
:10396000092A07D1D6E915100022334608F0E8FBF2
:103970000246E6E70A2A0CD100960023D6E9151084
:10398000012208F027FD02462846716CFFF78FFEE2
:10399000DFE70B2A13D1D6E915100A2906D8FDF75F
:1039A000EDF830B1000140F00600D2E7FDF798F8DD
:1039B000F7E7D6E91521074810F063FFE3E70C2A83
:1039C00004D1D6E9151011F051F8DCE7120142F0EC
:1039D0000A00BEE774A0050810B5FFF7B3FE50B1AA
:1039E0000B6813F0010007D19A0704D11868034B44
:1039F000C31A5842584110BD0120FCE72493050822
:103A00000021FFF713BF0121FFF710BF2DE9F04F91
:103A10002D2A1D4687B000F1280304468846164625
:103A200001930BD10021FFF706FEB8B1820702D146
:103A30000379922B12D007B0BDE8F08F922A20D1E3
:103A40000021FFF7F8FD014640B1830706D1037955
:103A5000952B0AD12046FFF7E7FD013DA6F11E0395
:103A6000012B6ED8A9462F461AE0962BF6D1204698
:103A7000FFF7DAFD4B6823F0FF0343F092034B603E
:103A8000D9E7962A08BF0135E8E71E2E4CD1FFF78B
:103A9000BAFFC8B95046FFF7B3FF002808BF5F461A
:103AA00007F1FF3BB9F1000F0ED009F1FF3949468C
:103AB0002046FFF7C0FD22696169D21B824641F8AA
:103AC0002200B9F1000FE0D10021594534D16D1A1F
:103AD000012DB0D0A6F12303022B01D92A2E67D1E4
:103AE000691E2046FFF7A7FD03A9FFF72BFE00285C
:103AF00000F06981232E40D0242E41D0252E0CBF0A
:103B00004FF018094FF02209AF1E002F3BDA002DAD
:103B100040F04E81039AD30740F14F8142F00101FA
:103B20002046FFF7D0FD86E7FFF76AFF0028CBD1DC
:103B30005046FFF768FFB0E72046FFF775FD0131FB
:103B4000C3E7202EC6D100212046FFF774FD0746AB
:103B5000FFF756FF70B93846FFF755FF0028B9D078
:103B6000EA212046FFF760FD204607B0BDE8F04F90
:103B7000FFF7A9BD4FF48571F3E74FF01609C3E7CE
:103B80004FF01709C0E739462046FFF754FD04A956
:103B9000FFF7D8FD002800F02181DDE90312484637
:103BA00003ABFFF753FE002800F01881013FACE79C
:103BB000A6F12603022B27D8691E2046FFF73BFDFE
:103BC00003A9FFF7BFFD002800F03A81AF1E002FC8
:103BD0009DDD791E2046FFF72EFD04A9FFF7B2FDFB
:103BE000002800F09E8039462046FFF724FDDDE9DD
:103BF00003120009243803ABC0B2FFF727FE0028E8
:103C000000F08F80023FE2E7292E22D100212046DA
:103C1000FFF711FD03A9FFF795FD002800F0818053
:103C200001212046FFF707FDC0F307103328039951
:103C300009D1CF0705D4880773D10A68814B9A420E
:103C40006FD1022001E03F38C0B209F053F9039070
:103C50005DE7052E73D100212046FFF7ECFC0746F7
:103C600000285ED010F0030B04D1436803F0FE037C
:103C7000562B56D001212046FFF7DDFC00F00F0344
:103C8000022B4ED1BBF1000F4BD13B792C2B48D1ED
:103C9000BB6803F00F02022A43D11B09482B40D115
:103CA000FB68002B3DD09A073BD11A79302A38D1D6
:103CB000D3F808A04FEA10195046FFF76BFD68B91A
:103CC000614962480DF0A2F80546A1695B463A6871
:103CD00009680DF052F92846FCF710FA5046FFF734
:103CE0007DFD4FEAC9010122074641F0020101981A
:103CF0000AF08EFC47604846FDF707F80278204638
:103D00005F2A08D10025FFF78FFC2046FFF78CFCC7
:103D1000A8460826A2E6FFF787FC51462046FFF793
:103D2000D2FCA91C89002046FFF78CFC46EA05233B
:103D30000746C0F80080436000F1080174E02C2EB3
:103D400041D101212046FFF776FC00F00F03022B42
:103D50000246E6D100212046FFF76DFC0028E0D0A6
:103D60008707DED10379322BDBD11109C9008768BF
:103D70000022374841F002010AF04AFC0028D0D066
:103D8000406804AA390908F0F7FF049B002BC8D04B
:103D9000D90708D49A07C4D11A682A498A4202D09E
:103DA0002C498A42BDD1059A002ABAD10393AEE6C6
:103DB0002046FFF739FC013DA9E629462046FFF7DA
:103DC00076FC0146ACE6922E08D1D4E9012303EB40
:103DD000C20313F8053C2D2BA3D116E0962E12D169
:103DE000D4E9012303EBC20313F8153C2D2B98D122
:103DF0002A4641462046FFF749FD002891D06368D6
:103E0000023B636017E6062E18D12A46414620463B
:103E1000FFF73CFD00287FF40EAE82E72046FFF757
:103E200003FC013D41F82500002DF7D1962E03D16A
:103E300039462046FFF747FC394695E6362EE4D052
:103E4000332EC9E72493050804740508148F050868
:103E50006C740508549005080346006830B508B92D
:103E6000106030BD840702D001201360F9E7446878
:103E7000E5B28D42F8D108301060200AF1E7000069
:103E80002DE9F04FAD4B97B0CDE907310D460290CB
:103E9000AB4905A800240192FCF7FCF840234FF43D
:103EA0000070CDE90934FCF74BF920230B908020FA
:103EB000CDE90C34FCF744F92146CDE90E0513A8F1
:103EC000CDE911440AF06EFB019B002B4DD0022B73
:103ED0000CBF3F2222460023696C09A8FFF70AFCA9
:103EE0000027DFF860A20A9C002C00F061810B998A
:103EF000013C01EBC40393F803B051F83410924A2B
:103F0000C1F3170912F80B209049009211F80B1019
:103F1000009ABBF1630F8E4E88BF41F4807106EBAF
:103F2000410602F0300110295B680A9402F00F0884
:103F30001DD020294BD0002F00F01081B8F1020FC6
:103F400040F0EE80012B17D00021009A581ED207B6
:103F500006D574880AEA0404B4F5805F08BF5808DF
:103F6000012800D161B10346D8E03D22B3E72BB967
:103F700006EB4306984505D80127B4E7002FF7D193
:103F80000027B0E7374636F8021B01EA0A00B0F511
:103F9000805F0DD195F84C00C1F30B01884214D11C
:103FA00009A85946FFF7B4FC2846FEF74DFFE7E79E
:103FB0000133434504D25A46494609A8FFF79AFB04
:103FC000398809A8FFF7B6FBDAE70133D2E77FB1FA
:103FD00003F10041013936F811100AEA0101B1F587
:103FE000405F1AD1002109A80393FFF76CFB039BE4
:103FF00006EB4304984524D8019B002B43D10024B1
:10400000274606EB480846455ED1012F7DD1009B2F
:1040100058067AD50026314671E0012BACD995F8C7
:104020004C30062B40F0F2804A494B480CF0EEFE33
:10403000044600236A6C29680CF09FFF2046FCF7B9
:104040005DF8274634F8021B01EA0A00B0F5805FEC
:1040500017D195F84C00C9B288420ED1082805D175
:10406000594609A80393FFF753FC039B2846039383
:10407000FEF7EAFE039B0133BCE7002B3FF47CAF65
:10408000CDE7013397E7BBF1050FB8D1002109A8AF
:10409000FFF7D1FA0028B2D1012109A8FFF7CBFA26
:1040A000840700F0BD8000F00F000228A7D009A807
:1040B000FFF7BAFA09A8FFF7B7FA00230822494622
:1040C00009A8FFF7A3FC5BE738F8023D03EA0A0101
:1040D000B1F5805F05D1DBB2082B94D101340137F3
:1040E00091E7214609A8FFF7A6FA00B1013701348C
:1040F00089E7FFF799FA002818BF01460136A64262
:1041000009A8F6D1FFF7DFFA3AE7009B190604D5B4
:10411000002109A8FFF7D7FA013423465A46CEE713
:10412000012B3FF429AF13F001013FF40EAFB8F1BA
:10413000030F7FF474AF012107E700BFFB350108CF
:104140007BCC010800F0FFFF98740508D0780508C3
:104150004875050810740508408D050808EA030134
:1041600001F0010136F8114004EA0A00B0F5805F61
:1041700013D195F84C00C4F30B04A04203F10104E1
:1041800009D119B9594609A8FFF7C2FB2846FEF71D
:104190005BFE2346E2E72346D0E6494609A85A4695
:1041A0000133FFF7A7FA214609A8FFF7C3FA9AE6F9
:1041B00013A80AF00BFA129850B141682246083150
:1041C000FBF7E4FF129B5A681A60119A5A60119328
:1041D00095F84C30002B7FF422AF0D9B002B3FF461
:1041E0001EAF0E9B0B981B681093FBF7D1FF0E9828
:1041F000FBF7CEFF0120FBF755FFDDE91001029B25
:1042000083E80300184617B0BDE8F08F022B01D1F8
:1042100007490AE7042B0CBF06490749074805E789
:1042200000283FF4ECAE03793A2B3FF440AFE6E6CA
:1042300022740508497405085C740508148F050884
:1042400038B50446406808B9606038BD4568FBF77A
:104250009FFF2846F7E70000F8B5054630200E46D8
:104260001746FBF786FF072D04460570C66001D090
:10427000012D0FD1B368C3F30F13A38208F070F9B7
:10428000042320612783E3842020FBF759FFE062A9
:104290002046F8BD014B5B5DEFE700BF8079050864
:1042A00010B50446C06AFBF773FF2046BDE8104016
:1042B000FBF76EBF30B500220446058D954201D84C
:1042C000002030BDE36A03EBC20043688B42F8D0A4
:1042D0000132F3E770B504460D461646FFF7EAFFD4
:1042E000C0B9E38C228D9A4208D30633D900E06A24
:1042F000FBF741FFE38CE0620633E384238DE26A3F
:10430000591C218502EBC30002F83360002345608D
:104310004370438070BD034618465B68002BFBD199
:10432000FFF7C8BFF8B544680E462CB9F8BD042B9A
:10433000FCD105230370F9E7254628466D68002D5A
:10434000F4D077683946FFF7B5FF0028F5D0037839
:10435000043B022BEAD80625357000223946204658
:10436000FFF7B8FF0378002BE1D105706468F4E72C
:10437000036A1B8B012B1EBFC3685B18C3607047A9
:1043800010B50446836A406A9B6F9847238B226A64
:104390000133918C9BB29942238338BF938410BD23
:1043A00010B50446038B013B0383836A406AD3F84C
:1043B000843098472046BDE810400121FFF7D8BF60
:1043C0002DE9F04107461E4661B111F0030511D1F8
:1043D0004B68D8B290420DD14FEA132801F108047E
:1043E000454501DBBDE8F081384654F8041BB04771
:1043F0000135F5E738463346BDE8F04118472DE969
:10440000F74F04460D46174698461BB1CB8A43F03A
:104410000803CB82236AEF83DA8A42F03002DA8221
:104420001B78002B46D1A36A3A46D3F8B4602946DC
:104430004346B446606A03B0BDE8F04F6047DB6AAC
:1044400003EBC60B13F83630053B012B1DD84FF09C
:10445000000917E0EB6A03EBC90213F83930062BA9
:104460000ED1DBF804105368994209D1A36ABBF856
:1044700002201B69606A9C460023E0470AF1010A9A
:1044800009F101092B8D4B45E4DC0136236A1A8DB5
:10449000B242D4DCBAF1000FC5D0A36ACDF80080D7
:1044A000D3F8B86052463B462946606AB04703B02D
:1044B000BDE8F08F0026B246E8E70000F8B50E46EA
:1044C00011461A4600230446857807698370036104
:1044D0000E4BFFF775FF6368BBB9618A51B1228A41
:1044E00042B9A36A606AD3F8A0309847A36A606AA9
:1044F0001B6C984731462046238A628AFFF77FFF6C
:10450000003D18BF01252761A570F8BD994E01082F
:104510009D22024B8968FFF753BF00BF156B01084E
:104520006B22024B8968FFF74BBF00BF0968010887
:1045300010B50446836A0021D3F88830406A984752
:10454000A36A606A0F211B6B9847A36A606A012106
:10455000D3F8CC3098472046BDE810400321FFF740
:1045600007BF38B50446836A00225B6C406A9847EF
:10457000A36A606AD3F8C05000231A461946A847B8
:104580002046BDE83840FFF7D3BF836A8968002220
:104590001B6D406A09091847836A8968DB6B406AAA
:1045A000184710B50446084611461A46FFF754FE50
:1045B000236A436000238360E3690BB9E06110BDA7
:1045C0001A469B68002BFBD19060F8E770B54378E2
:1045D0000546012B0C4606D1036A0A461B8B0221B5
:1045E000FFF7DFFF20612846A26821694C23BDE860
:1045F0007040FFF763BF70B5134642780546012A45
:104600000C4604D10A460721FFF7CBFFA061A6693B
:10461000284646233146E268FFF750FFB08A70BD56
:104620002DE9F04F85B005460C4600AF11B90121C8
:10463000116015E011F003081BD10B79682B07D12D
:10464000CB681B0913608C68002CF0D04FF0010878
:1046500004F00F03022B0FD12109B8F1000FE7D0AE
:10466000AB6A0022DB6A686A98471437BD46BDE82A
:10467000F08F4FF00008EBE7B8F1000F02D1A3680C
:104680001B09136004F1080AD1466668360A06F170
:10469000FF3B0AEB860659F8040B0009FCF72AFBDE
:1046A000B1458344F7D10BF1070323F00703ADEBCA
:1046B000030D6B4699465AF8040B07F10C010009EB
:1046C0003B60FCF72EFBFA68014648467A602DF005
:1046D00036F97A68B2453B68914418D15946184674
:1046E000FCF74CFAAB6A01460022DB6A686A98471D
:1046F000B8F1000FB9D00C34A642B6D054F8041B60
:10470000AB6A00221B6D686A09099847F4E74FF00D
:104710002E0209F8012BCEE731B1826801F00303C4
:10472000134304BF0B6883607047000038B54368CB
:104730000D46044611464BB905480CF067FB294667
:1047400060602046BDE83840FFF7E6BF38BD00BFD7
:10475000148F0508014AFFF7E9BF00BF87790508F4
:104760000B7970B5092B4FF6FF730CBF858AC58A8C
:1047700004469D4202D1064AFFF7D8FF218B628B87
:10478000A36A606A8A1A5B6F2946BDE870401847C1
:104790009479050870B5144605460E46127883B123
:1047A00032B1032A04D0104ABDE87040FFF7BEBF03
:1047B000032626706168286AFFF7ADFD00B1067018
:1047C00070BD62B9012323702146006AFFF7AAFD7C
:1047D0002378012BF4D131462846044AE4E7062A1F
:1047E000EED0034AE0E700BFAD790508BA790508C5
:1047F000C779050838B50446A9B101F00F03022BAB
:104800000DD10D09284609F045FD002806DA2A4693
:10481000064907480CF072FB6060002038BD054A6D
:10482000FFF784FFF9E70846F8E700BFCE790508EF
:10483000C88F0508D379050810B4044662780B4682
:10484000012A006A02D110BCFFF744BDA16A0246EA
:104850001031606A10BC02F047BE000070B505461A
:104860000C4600292ED0CA0706D5836A49105B6B17
:10487000686ABDE8704018478B0717D004F00F0432
:10488000022C4FEA11110AD0062C0CD0052919D0A0
:10489000BDE87040836AC9B21B6B406A1847BDE827
:1048A0007040FFF7C9BF836A9B6BE1E7836A0968C1
:1048B000DB68406A98472279034B2146284653F823
:1048C0002230D6E770BD00BF907B05082DE9F74F79
:1048D00005460C4616461F462046FFF791F840B1A4
:1048E0006EB93946AB6A9B6E686A03B0BDE8F04F9B
:1048F00018472046FFF787F820B1002EF1D103B00A
:10490000BDE8F08F002C48D0A30746D163684FEA7A
:10491000132BDBB21E2B18D1DEB1083404EB8B0B4A
:10492000A345ECD03B463246284654F8041BFFF71B
:10493000CDFFF5E7434628465AF8041B019209F1DA
:104940000109FFF7C3FF019A11E01F2B1FD1002EB1
:10495000E3D04FF00009D5F80C8004F1080A08F103
:104960000103EB600BF1FF33009386F00102009B23
:104970004B45DFDC0BF101013B4654F82110324678
:104980002846FFF7A3FFAB6A41469B6AACE7202BA2
:1049900003D1A46886F001069EE721462846FFF76A
:1049A0005DFF3A463146AB6A686ADB6E03B0BDE82C
:1049B000F04F184738B5026A044612780B46072AAA
:1049C00006D0022A04D0BDE83840144AFFF7AEBE34
:1049D0009D6885B9A36A0F211B6B606A9847A36A1B
:1049E000606A0021D3F8CC3098472046BDE83840B3
:1049F0000121FFF7BDBCAB070BD12B79AF2B08D141
:104A00002046A968FFF72AFF2046BDE83840FFF797
:104A10008FBD29462046FFF721FFE0E7E37905082F
:104A200070B543780446012B1546CE6806D1036A5B
:104A30000A461B8B2946FFF7B4FD70610023204610
:104A40001A467169FFF7DBFC2046F168FFF706FFA5
:104A5000062D05D1A36A0021D3F88830606A9847F3
:104A6000A36A606AD3F8BC500023AC46BDE870402E
:104A70001A460121604738B505460C46C968FFF75C
:104A8000EDFE2846A168BDE83840FFF7E7BE0B7988
:104A900070B5342B04460D4610D18968FFF7DEFE51
:104AA000ED68AD6885B9A36A0F211B6B606A9847F2
:104AB000A36A04220221D3F8A0301AE0836A0F21EE
:104AC0001B6B406A9847ECE7AB071FD12B799A2BF9
:104AD00013D1A36A0F211B6B606A9847A96800294C
:104AE000E6D02046FFF7BAFE04220321A36AD3F8DA
:104AF000A030606ABDE8704018479B2B06D1A968BA
:104B00002046FFF7ABFEEB689968E8E729462046A8
:104B1000FFF7A4FECCE710B504468968FFF79EFEB8
:104B2000A36A606A0021BDE81040DB6C18470000F2
:104B30002DE9F7438D68044616465DB9002A75D005
:104B400002222946836AD3F8A030606A03B0BDE828
:104B5000F043184715F0030740F08A802B79372B74
:104B600013D132B1836A02220121D3F8A030406A06
:104B7000984720462946FFF771FEA36A606AD3F87A
:104B8000A43003B0BDE8F04318479F2B70D1EB6809
:104B90001A79A12A5AD1A22101AA03F10800FFF72C
:104BA0005BF9A968804621B38B0722D10B79372B9B
:104BB0001FD136B1A36A411C0222D3F8A030606A2B
:104BC00098472046A968FFF749FEA36A606AD3F8B0
:104BD000A43098474FF00109474510D1B9F1000FB3
:104BE00024D1A36A0322D3F8A030606A791C9847C5
:104BF0001CE02046FFF732FE4FF00009ECE7019B76
:104C000053F82710A9B18E0713D10E79A6F13700FA
:104C1000464246412046FFF721FEB9F1000F11D070
:104C20004EB9184A29462046FFF780FD03B0BDE87B
:104C3000F0830026EEE7A36A606AD3F8A4309847B1
:104C40000137C9E7002EFBD00F4AEBE7AB685BB139
:104C50009A0709D11B79372B06D10422294603B0C4
:104C6000BDE8F043FFF7DCBE052229462046F6E703
:104C700029462046FFF7F2FDA36A03220121D3F85B
:104C8000A03062E7EE790508FF7905080122FFF7F9
:104C90004FBF70B50D460446C968FFF7DFFDA96830
:104CA000A36AC1F30711332918BF3F39606A08BFEF
:104CB0000221BDE87040D3F8983018BFC9B2184738
:104CC000F8B54F680C46896805460026FFF7C6FD13
:104CD0003F0A0C340236B74204F1080400DCF8BD88
:104CE000284654F8041CFFF7B9FD54F8081CAB6AB9
:104CF00009092439D3F89C30686AC9B29847E9E7B2
:104D00002DE9F0414E680C46896805460127FFF7FA
:104D1000A5FDA6F10D085FFA88F8360A0C34B742F3
:104D200001DBBDE8F081284654F8041BFFF796FD2F
:104D3000AB6A4146D3F89C30686A98470137EEE782
:104D40002DE9F04104464E680D46360A8968FFF7A2
:104D500085FD032E98BF4FF000084FF0010782BF7A
:104D6000D4F80C8008F10103E3607B1C9E4222DC36
:104D7000032E55DDE568606A6B1CE360A36A294673
:104D80009B6E9847A36A4146606A9B6A9847A36AEC
:104D90000121606A9B689847A36A606A1B6E984706
:104DA000A36A606ADB6D9847A36A2946606A9B6ABA
:104DB000BDE8F0411847204629690237FFF74EFD4C
:104DC000B74207DAA36A606A5B6D9847A36A606AB4
:104DD0005B6E9847E968A36A01F00F020A2AD3F8CC
:104DE0009C30606A11D1C1F3071125290EBF06213D
:104DF0003439C9B29847B74205DAA36A424600215E
:104E00001B6F606A98470835AFE70A79852A01D198
:104E10003221EFE78A680AB90721EBE73321E9E796
:104E2000BDE8F08110B504468968FFF717FDA36A55
:104E3000606A0321BDE81040D3F8983018472DE987
:104E4000F047044600274E68D0F80C805FFA86F9D8
:104E5000A9F11E03D3F1000949EB030908F101038D
:104E6000C360360A01F10805B74206DBA36A414672
:104E7000606A9B6ABDE8F0471847204655F8041B56
:104E80000137FFF7EBFCB742F0DAA36A4246494626
:104E90001B6F606A9847E7E701F00F03022B70B5BC
:104EA00004460FD00B79492B01D04F2B02D101239F
:104EB000A37070BD4A2BFCD0502BFAD0482B0DD1DB
:104EC0000D696DB9A378002BF3D1638A002BF0D064
:104ED0002046BDE870401C4AFFF728BCCD68F0E7CB
:104EE000A37843B3238A8E6801339BB2012B2382BC
:104EF0000ED1D4E90903618AD1B10022D3F8A030E0
:104F00009847A36A02220021D3F8A030606A98472C
:104F100029462046FFF7A2FCA36A606A9B6B310911
:104F20009847A36A606AD3F8A430BDE87040184778
:104F30001B6C9847E5E7638A294601332046638264
:104F4000BDE87040FFF78ABC0C7A05082DE9F041F6
:104F500004460E46C568D1F80C80AB1C0022D8F878
:104F60000810C3602B46FFF7B1FC2046B168FFF77D
:104F700075FCA36A6F1C3946606A9B6E9847A36AEA
:104F80002946606A9B6A9847A36A606A9B684FF0EB
:104F9000FF3198472046D8F80C10FFF75FFCA36A52
:104FA0003946606A9B6ABDE8F04118472DE9F04731
:104FB000C668D0F814A0B31CC360038B06F10108C7
:104FC000B0F81A9004468682A0F816804383886859
:104FD0000D46FEF715FDF8B9E768A8687B1CE3608D
:104FE000FEF711FD20B9A36A41469B6E606A98479F
:104FF000A36A39469B6A606A98472046E968FFF7CA
:105000002DFCA36A41469B6A606A98473B46012291
:105010002046A968FFF75AFC20462969C4F814A065
:10502000A4F81A90FFF71AFCA36A3146606A9B6ADB
:10503000BDE8F04718472DE9F347C6680446731CDE
:10504000C36088680D46FEF7DBFC0246E8B9E768F6
:1050500020467B1CA968E3603B46FFF737FC2046EF
:10506000E968FFF7FBFBA868FEF7CDFCD8B92B6910
:105070000BB96B6923B1A36A31469B6E606A98478E
:10508000A36A39469B6A606A9847712101AA05F1B3
:105090001000FEF7E1FE002781464F450BD1204668
:1050A0006969FFF7DBFBA36A31469B6A606A984730
:1050B00002B0BDE8F087019B53F82780D8F80800BC
:1050C000FEF79EFC0246F8B9D4F80CA020460AF17F
:1050D0000103D8F80810E3605346FFF7F7FB2046BA
:1050E000D8F80C10FFF7BAFBD8F80800FEF78BFCD5
:1050F0000028D8D1A36A31469B6E606A9847A36A9C
:1051000051469B6A606A98470137C6E770B58D685B
:1051100004463DB92946836AD3F8C830606ABDE8C1
:1051200070401847AB070ED12B795E2B0BD1A968C5
:10513000FFF794FBE9682046FFF790FBA36A022182
:10514000D3F8C830EAE729462046FFF787FBA36A71
:105150000121D3F8C830E1E710B504468968FFF7AC
:105160007DFBA36A606ADB6DBDE8104018472DE93E
:10517000F04105464E6801F10804360A04EB860743
:10518000BC4208D1AB6A3146686A0022BDE8F041F2
:10519000D3F8A0301847284654F8041BFFF75EFBED
:1051A000EEE78968034610B439B9826A406AD2F8DA
:1051B000A0400A46234610BC18474A68120A022A31
:1051C0000AD1CA6842B1940706D11279AC2A03D138
:1051D000062210BCFFF724BC184610BCFFF7C7BF5F
:1051E0002DE9F04105460E4600244B6801F1080800
:1051F0001F0ABC4201DBBDE8F081284658F8041BB9
:10520000FFF72CFB6B683BB10234284656F824109C
:10521000BDE8F041FFF780BA0134EAE710B5044673
:10522000FFF7DEFFA36A606A2221BDE81040D3F8D1
:105230009C30184770B58D68044645B9012229464F
:10524000836AD3F8A030606ABDE870401847A907A8
:105250001ED16B68DAB2922A1AD11B0A022B0CD12A
:10526000EB6853B19A0708D11B79AC2B05D12946BD
:10527000BDE870400322FFF7D3BB29462046FFF765
:10528000AFFF6968A36A0122D3F8A030090ADAE700
:1052900029462046FFF7E2FA0122A36A1146D3F815
:1052A000A030D0E7184B2DE9F041D3F8B071044697
:1052B0000D463FBBC6680122731CC3608968334634
:1052C000FFF704FBA36A1F2101225B69606A98470C
:1052D000E96851B12046FFF7C1FAA36A3A46D3F80C
:1052E000BC5001213B46606AA847A36A606A01215D
:1052F000D3F8C8309847A36A3146606A9B6ABDE814
:10530000F0411847BDE8F081700300202DE9F0411D
:10531000026A04461278072A04D0BDE8F0411A4A0E
:10532000FFF704BA8D685DB9836A0F211B6B406A71
:105330009847A36A606AD3F8C430BDE8F0411847C3
:1053400015F003021DD12B791B2B1AD1C668EF680B
:10535000731CC360B9683346FFF7B8FAA9682046E2
:10536000FFF77CFAA36A606AD3F8C4309847A36A4F
:1053700031469B6A606A9847F9682046FFF76EFAE3
:10538000D7E72946F9E700BF2A7A050810B4026A70
:10539000044640780B46012803D1104610BC02F0A9
:1053A00094B8A16A606A183110BC02F09DB8000080
:1053B0008B072DE9F14F04460D46164611D001F03A
:1053C0000F03022B16D1D7074FEA111104D401B0F5
:1053D000BDE8F04FFFF7DABF01B0BDE8F04FFFF7CF
:1053E0002BBA4968CBB22D2B7BD00BD8062B0DD016
:1053F0002C2B12D0294620464D4A01B0BDE8F04F73
:10540000FFF794B92E2B7FD09D2BF3D1002EF1D135
:1054100005F10802090A20467BE0022A02D0A968A9
:10542000FFF71CFAEF68002FE4D017F00309E1D171
:105430007B68B846DAB28E2A0DD1022E4FEA1328C5
:1054400005D007F1080A08F1FF3BD94511DB08F147
:10545000010857F8288098F80430312B24D1022E07
:105460000FD1A36A606A5B6E9847A36A0121DB6C67
:1054700015E020465AF8041BFFF7F0F909F101097D
:10548000E3E72046D8F80810FFF7E8F9012EA36AF1
:10549000ECD19B6D606A98470021A36ADB6C606A5F
:1054A00001B0BDE8F04F1847322BA3D1D4E909036E
:1054B000012E0CD15B6D98470022A36AD8F8081022
:1054C0001B6D606A090901B0BDE8F04F1847022E54
:1054D00001D11B6E9847A36A0122D8F808101B6DF2
:1054E000EFE7AA68002A85D0002E83D15168090A07
:1054F000022907D1D3682BB1980703D11B79AC2BB4
:105500003FF478AF083286E7002A7FF473AFA968CA
:1055100021B901B0BDE8F04F00F074B88E0703D197
:105520000B790A46922BE1D0012105F1080272E7BE
:10553000367A05082DE9F04704460D46C7681E4631
:10554000BB1CC360836A39469B6A406A9046984791
:10555000A36A07F101094946D3F88C30606A98477D
:10556000A96800222046FFF723FF2D69002D2DD1C9
:1055700041462046FFF772F9236AA06A1978062986
:105580001DD1D0F8CC302946606A984720460121C9
:10559000FEF7EEFEA36A606ADB6D9847A36A3946A0
:1055A000606A9B6E9847A36A606A49469B6A9847FF
:1055B000A36A606AD3F89030BDE8F0471847B2009C
:1055C000D0F8A8500532606AA847E7E72B79AD2BE1
:1055D00007D1A9683B4600222046FFF777F9ED681E
:1055E000C4E72046E968FFF739F9A36A606A012138
:1055F000D3F888309847424629462046731CFFF767
:1056000099FFCBE72DE9F84304460D469046002666
:105610004FF0FF3701F1FF39B9F1FF3F0CD17B1C8F
:1056200005D1A36A2946D3F8AC30606A98470026B2
:10563000AE421DD1BDE8F88358F8261071B18A0733
:105640000CD10B79222B09D101370BD1A36A4A4621
:105650003146D3F8B030606A98473746013609F1D1
:10566000FF39D9E72046BDE8F843074AFFF75EB89F
:1056700058F82610B7424FF00002204608BF89684C
:10568000FFF796FE0136D3E74A7A05082DE9F04781
:105690000446904699460F4621B9BDE8F0471946A1
:1056A000FFF7DCB8C668731CC360156835B315F026
:1056B000030A23D12B797B2B20D1A968FFF7CEF8E1
:1056C000524631462046FEF75BFE52462046E968C8
:1056D000FFF76EFE4B46204608F10402791EFFF7E5
:1056E000D5FFA36A3146606ADB6F984720460321E5
:1056F000FEF73EFEBDE8F047FEF752BE29462046C3
:10570000FFF7ACF8204600223146FEF739FEA36AC7
:10571000606ADB6D9847DDE737B50C46054601AAA0
:105720007A2104F10800FEF797FBE3680146019A2D
:105730002846FFF7ABFF03B030BD2DE9F04F8B6873
:10574000044603F00F03022B0E4689B040F0FF80A1
:10575000CB68002B00F0FB80980740F0F8801A79A6
:105760002C2A40F0F4809A6802F00F01022940F0E0
:10577000EE8012097C2A40F0EA80DB681A79302A30
:1057800040F0E5809B68A42107AA06A80693FEF7CF
:1057900063FB431E022B00F2DA80079901280A6896
:1057A00000F0C7800228D1F8049000F01F818D68B6
:1057B000E90740F1CC806B0800F0C98032B1930753
:1057C00004D11179A639022940F2C180B9F1000F44
:1057D00008D019F0030F05D199F80410A639022951
:1057E00040F2B580B368776901933369218B0293E6
:1057F0006369E6680493638B19F00108039361837E
:1058000006F1010306F10401059306F1020AA682DE
:10581000E38206F1030BE16005D14946204605927B
:10582000FFF71CF8059A11462046FFF717F8A26A01
:105830005946926E606A9047A26A5146926A606ABF
:105840009047A26A606A526D9047002220460199F3
:10585000FFF7AEFD20460299FFF700F8A26A606AE2
:10586000926A711C904729462046FEF7F7FFA26A0C
:105870000E21D2F89C20606A9047A26A5946926A2B
:10588000606A9047A26AB8F1000F56D1936D606AC2
:105890009847A36A606A1B6E9847A36A002DACBF45
:1058A00000210121D3F89C30606A9847A36A5246D0
:1058B000DB6E0121606A9847049B6361039B6383ED
:1058C000002F42D0A36A606ADB6D9847B8F1000FE1
:1058D00003D1A36A606ADB6D984739462046FEF71C
:1058E000BDFFE568606A6B1CE360A36A29469B6E96
:1058F0009847A36A88F001019B68606A0131984764
:10590000A36A606A9B6A31469847A36A606ADB6D46
:105910009847B8F1000F03D1A36A606ADB6D98471E
:1059200027B1A36A29469B6A606A984709B0BDE817
:10593000F08F91460325024648E7606A526D904712
:1059400049462046FEF78AFFA7E73D46D8E7E568C7
:10595000238BB4F81A9063836FEA45436FEA53438D
:10596000D4F814A06F1CA382EB1C2046F168E360FE
:10597000E782FEF773FFA36A606A0121D3F88830DB
:105980009847A36A3946606A9B6A9847A36A05F1FB
:105990000208D3F88C304146606A984700222046BE
:1059A000B168FFF705FD20463169FEF757FFA36A8E
:1059B0003946606A9B6E9847A36A4146606A9B6A53
:1059C0009847A36A606AD3F8903098472046716977
:1059D000C4F814A0A4F81A90FEF740FF2946A36A61
:1059E000606A9B6A09B0BDE8F04F18470325E5E6F9
:1059F0002DE9F74F0446174698460E4629B9194631
:105A000003B0BDE8F04FFEF729BFC5682B1DC3608A
:105A1000136805F1010A05F1020B05F10309002BDA
:105A200000F0D28013F0030240F0CE8019797B2978
:105A300040F0CA80996801920093FEF70FFFA16AB7
:105A4000606A496D884740F223212046FEF789FDB0
:105A5000DDE900322046D968FFF7AAFC0222294678
:105A60002046FEF78DFCA36A606A03219B68984775
:105A70003A1D43462046711EFFF7BAFFA36A606ACB
:105A80006FF002019B689847A36A2A465146D3F8F3
:105A90008060606A5B46B047A36A606A5B6D984746
:105AA000A36A606A5B6E9847A36A606A1B6E984738
:105AB000A36A00224FF40971606A5B6C9847A36A7D
:105AC000606A5B6E9847A36A606A5B6E9847A36AD8
:105AD000606A5B6D9847A36A00220A21606A1B6DA9
:105AE0009847A36A606A1B6E9847A36A606A0F2191
:105AF0001B6B9847A36A0321D3F8C0500023606A48
:105B00001A46A8472046FEF713FDA36A4A4600211D
:105B1000606ADB6E9847A36A606ADB6D9847A36A88
:105B2000606A0F211B6B9847A36A4946606A9B6EA7
:105B30009847A36A606A02219B689847A36A5946FE
:105B4000606A9B6A9847A36A606A5B6E9847A36A1B
:105B5000606A5B6E9847A36A5146606A9B6A984781
:105B6000A36A0022606A4FF409715B6C9847A36ACC
:105B70000F21606A1B6B9847A36A606A5B6D984748
:105B8000A36A606A5B6D9847A36A0321D3F8C0508B
:105B90000023606A1A46A8472046FEF7C9FCA36A9C
:105BA000606ADB6D9847A36A606A4FF0FF319B68BB
:105BB0009847A36A606A49469B6A9847204603B0A3
:105BC000BDE8F04FFEF7ECBB19462046FEF746FE57
:105BD000A36A606A5B6D9847204640F22321FEF776
:105BE000C0FCA36A606ADB6D984737E72DE9F04196
:105BF000CD6804460E463DBB0378C3B1036A1D78E9
:105C0000ADB940F23221FEF717FEB1682046FEF72B
:105C100025FEA36A2A46D3F8BC6001212B46606AA0
:105C2000B047A36A606ADB6DBDE8F0411847B16810
:105C3000880700F0BC8001F00F03022B40F0BE800B
:105C40002046FEF70BFEECE7A90740F0BB806B682F
:105C5000DAB25B2A14D1ED68002D40F0B180006A01
:105C60000378072B40F0AA80B16801F00F03022BE4
:105C700040F0A480BDE8F0410422D140FEF72ABBE9
:105C8000562A13D10122B168FFF792FB2046E9683A
:105C9000FEF7E4FDA968A36A09093E39D3F89C30F0
:105CA000606AC9B298470222B1687BE0572A40F087
:105CB00087801B0A5F1E013355F82310FEF7CEFDC7
:105CC000002F03DDA36A606A5B6D9847B16800220C
:105CD0002046FFF76DFB00260835BE426EDA01361E
:105CE000BE4203DAA36A606A5B6D984700222046D1
:105CF00055F8041BFFF75CFBEFE76B68DAB2062A86
:105D000060D1B768002F5DD0BA075BD17A68D1B295
:105D1000062957D11B0AB3EB122F4FEA122851D193
:105D2000A8F10203012B4DD8BB6823B1980702D11B
:105D30001B79222B46D0FB6823B1990702D11B792E
:105D4000222B3FD0B8F1020F06D03B6923B19A074E
:105D500002D11B79222B35D02046A968FEF77EFDA3
:105D60002046E968FEF77AFDB8F1030F07D1204617
:105D70002969FEF773FDA36A606A5B6E9847A36AA0
:105D8000606A1B6E984700222046B968FFF710FB37
:105D900000222046F968FFF70BFBB8F1030F0DD185
:105DA000002239692046BDE8F041FFF701BB002918
:105DB0003FF446AF0B793A2B7FF442AFBDE8F08158
:105DC000AB079AD029462046FEF748FD00226BE734
:105DD0000023032A2DE9F04104460D461646427081
:105DE0000162C36080F8342002D1C08E50BBA06332
:105DF0004FF00008A36A31461B68606A2A46A4F87F
:105E00003680984706212046FEF7B2FA6778EE689A
:105E1000012F04BFA5F82280A5F82480B6B1B207EF
:105E200014D133793F2B11D1B168FEF717FDA36A66
:105E3000606AD3F8C4309847A36A606A5B68BDE8BB
:105E4000F04118478000FAF794F9D0E72B784BB966
:105E500031462046FEF702FDA36A0F211B6B606AE4
:105E60009847E4E7072B16D1012F12D10023A37026
:105E70004622584B2046F168FEF7A2FA2B8B032BE3
:105E800007D120463169FEF7B5FCEB8A43EA80135F
:105E9000EB827169DDE7022B1BD1A36A3168DB68F5
:105EA000606A98476378012B07D10023A3704C22C6
:105EB0002046494BB168FEF783FA2046F168FEF7A9
:105EC000CDFCEB8ADB07B2D5A36A606ADB6D98472D
:105ED000C2E7033B032B4FD8012FD6F80C8005D126
:105EE00004223946206AFEF7F5F96F83A36A316808
:105EF000DB68606A98472B78032B24D10122A36AC0
:105F0000D3F8A0300021606A98472B78062B28D15F
:105F1000A36A606A1B6C984701212046FEF78CFC3F
:105F2000A36A606A1B6C9847A36A606A1B6C9847F7
:105F3000002341462046B268FFF7FCFA2B78062B77
:105F40007FF475AF88E7042B04D1A36A0222D3F84B
:105F5000A030D7E7052BD8D1A36A0322D3F8A0300D
:105F6000D0E720460121FEF767FCA36A0121D3F8A0
:105F70008830606A9847DBE7012F04D104220A21A8
:105F80002846FEF7A7F917212046FEF755FC1621F3
:105F90002046FFF7FBF9B168A36A606A9B6B0909A9
:105FA00098471A212046FFF7F1F920463169FEF79C
:105FB00055FC0A212846FEF77DF90378042BA36AD5
:105FC0003FF44BAF1D69428800230A21606AA8474D
:105FD0002DE700BF5D6D0108656D0108036A10B50E
:105FE0001A8B0446FEF707FB01462046BDE8104029
:105FF000FFF7CCB92DE9F04F8D6804462B7985B0B9
:10600000032B0AD12946FFF7E9FFAA69D38A43F097
:106010000103D38205B0BDE8F08F026AD28AD207AD
:1060200006D42946614A05B0BDE8F04FFEF77EBBB5
:10603000162B40F0AD80C668E968331DC360FEF7DB
:106040000DFCA36A606A002240F225215B6C984730
:10605000A36A606AD3F8C07000231A461946B8478D
:106060006369E7680193638B07F101080093BB1C28
:10607000E360238B41466383A36A606A9B6A06F1EF
:10608000010BA782A4F816809847012259462046A2
:10609000FEF776F9A36A606A5B6D9847204640F286
:1060A0002721FEF75EFA2046A9680022FFF780F953
:1060B000A36A06F1020900224946606AD3F89430C7
:1060C0009847A36A5946606A9B6A9847A36A606AC0
:1060D000D3F8D0309847A36A606A5B6D9847A36A8B
:1060E0000122606A4FF4FE715B699847A36A606A97
:1060F0000821D3F89C309847A36A06F1030A524658
:106100000021606ADB6E9847A36A606ADB6D98477E
:10611000A36A01223146606AD3F894309847A36A93
:106120005146606A9B6A9847A36A01219B68606A2E
:1061300098472046FEF734F9A36A606AD3F8D43052
:106140009847A36A49469B6A606A9847204629692E
:10615000FEF784FBA36A4146606A9B6E9847019BE9
:1061600031466361009B606A6383A36A9B6A9847B8
:1061700020466969FEF772FBA36A606A39469B6A2A
:106180009847A36A606ADB6D05B0BDE8F04F184719
:1061900003AA7A2105F10800FDF75EFEEB680146CF
:1061A000039A2046FFF724FC34E700BF517A050824
:1061B00001F00F03022B70B504460D46164602D0BF
:1061C0001E4AFEF7B3FA31462046FEF747FBA36AA4
:1061D000606A5B6D984763782E09012B0FD1226AA4
:1061E0001378033B032B0AD85068314601F06DF950
:1061F0000278032A09D13146206AFEF76BF831464E
:106200002046BDE87040FFF7C1B800223146206A41
:10621000FEF760F8236A02465B685B68002B0CBFE0
:106220000123002304D00178012904BF002101705B
:1062300029462046FEF7AEFAE1E700BF367A0508A8
:106240002DE9F04F002787B0CDE902210446A421B3
:1062500005AA03A81D46FDF7FFFDB9463E46B84610
:106260004FF0010B0190019B9F4211D126B1A36A0F
:1062700049465B6B606A9847D4E90903029A002A91
:1062800073D0D3F8C040334642462946A04713E0B6
:10629000059B53F827A0BAF1000F5BD01AF0030F4B
:1062A00058D19AF80420A62A19D1B00707D5304A48
:1062B00051462046FEF73AFA07B0BDE8F08F1D2F91
:1062C00001D92C4AF4E70BFA07F2DAF8081046F085
:1062D000010649EA02092046FEF7C0FA20E0A72A93
:1062E0000ED1A26A606A126C9047DAF8081046F084
:1062F00002062046FEF7B2FA08F101080137B2E7BC
:10630000A82A27D1DAF80C2072B191070CD11179A3
:10631000AA2907D120469268DAF80810FFF748FF4B
:106320000135EBE7AC290FD0DAF8081001F00F02C5
:10633000022A01D0104ABBE7A26A0909926B606A7F
:106340009047DAF80C10D4E7062251462046FEF7B3
:1063500067FBE5E7B30701D5084AA9E7B8F1000FE5
:1063600001D0074AA4E75146B5E7D3F8BC408AE715
:10637000687A05086F7A0508777A0508847A05082F
:106380008B7A050870B50D464178044601291346FD
:1063900003D12A46FEF705F96861A36A606A9B6C1F
:1063A000984700236E691A4631462046FEF727F8C3
:1063B000A36AB18A9B6B606A9847E96829B18B0729
:1063C00003D10B79A32B08BF002120460223002212
:1063D000FFF736FFB08A70BD002389681A46FFF7C1
:1063E0002FBF00002DE9F8430C4689680546FEF7EB
:1063F00035FAE668002E57D07768296AFBB209782B
:106400008E2BA36819BF012704F10C063F0A08363A
:10641000072903F00F024BD1022A47D11A099A2A01
:1064200048D132681179302944D19268002A41D18B
:106430000A212846FEF700FA2A6AD36A128D32B979
:10644000284631683F4ABDE8F843FEF76FB95978EE
:10645000C9070FD559682846FEF7EEF9022FAB6A37
:106460000BD8D3F8BC40002302211A46686AA04723
:10647000012417E0013A0833E1E772681179322903
:10648000EFD1B46821793029EBD191685B6C01229E
:10649000686A09099847A168002301222846FFF786
:1064A000CFFE0324A74225D8BDE8F8830024F9E7EE
:1064B000022AFBD11B09B3F5CF7FF7D133681A79D4
:1064C000302AF3D19C68002CECD014F00308EDD1F5
:1064D00023792F2BEAD1AB6A42464146D3F8BC4020
:1064E000686A4346A0473368424628469968FEF7E3
:1064F0001FFBBDE704F10108B84556F824104FEA28
:1065000084031AD20A79322A17D13344D3F804907B
:1065100099F80430302B10D18968AB6A00225B6C8B
:10652000686A09099847002301222846D9F808100B
:10653000FFF786FE08F10104B4E72846FEF78EF95E
:10654000A046F7E7927A050810B5026A0446127869
:106550000B46072A06D0022A04D0BDE81040064A9E
:10656000FEF7E4B820461946FFF73CFF2046BDE899
:106570001040FDF7DDBF00BFA57A0508CA6889682D
:10658000FFF716BE036A10B51A8B0446FFF7FAFE32
:1065900001462046BDE81040FEF7F8BE2DE9F04F59
:1065A00085B00191019B0446422103F1080002AA33
:1065B000FDF752FC00268346B146236ADFF808A1A6
:1065C0001D8B5E450AD1019BD9680B79032B51D1F4
:1065D0002A462046FEF70FF8054659E0029B6C213B
:1065E00053F8263003AA03F108000093FDF734FCAA
:1065F000039B074619680A09732A0DD02046FEF747
:106600002DF94FF00108B84528D3009BD96859B13E
:106610002046FEF723F907E0022807D0524620461D
:10662000FEF784F809F101090136CAE759680B0938
:10663000412B0DD040F2A73293420BD040F265427D
:10664000934209D040F25F229342E7D10425E9E763
:106650000125E7E70546E5E70325E3E7039B00227D
:1066600053F82810A36A606A1B6D0909984708F15E
:106670000108C8E7442B17D18E682A4631462046C8
:10668000FDF7B9FF0546B269D38A43F00103D3820F
:106690000026ABEB0909B1450BD829462046FEF789
:1066A00075FE05B0BDE8F08F2A462046FFF76AFE6A
:1066B00092E7A36A0121D3F8BC700023606A1A46EE
:1066C000B8470136E7E700BFB07A05082DE9F34186
:1066D0008D68044605F00F030A2B0E4606D0002DE8
:1066E00030D0AB072ED12B79652B1ED1009500251C
:1066F000652101AA6846FDF7AFFB002140F2CA52AE
:10670000019B03EB8000984215D140F21A43F268D6
:106710009A4237D1236A1F78B7B131462046394AA9
:1067200002B0BDE8F041FEF701B8622B0AD1AB68B8
:106730000093ED68DCE753F8047B97420CBF01310E
:106740000331E0E70021E0E7A36A606A5B6B9847EA
:10675000A36A05219B6B606A9847A36A3A46D3F8FF
:10676000A0300121606A98472946204601AAFDF71A
:1067700057FFA36A02223946DB6A606A984702B073
:10678000BDE8F081A36A606A5B6B984706F10C0074
:106790006A466A21FDF760FB00270646D4E9090333
:1067A000B74211D100223146D3F8A030984729468C
:1067B000204601AAFDF734FF0025D4E90903B542BC
:1067C0000BD1DB6D9847DAE7009A9B6B52F82720D4
:1067D0000137916809099847E0E7009ADB6A52F8A7
:1067E00025800122D8F808703F0939469847D8F823
:1067F0000C1029B939462046FEF7C8FD0135DCE703
:106800000909F8E7C87A050837B504460D46836AD2
:1068100000215B6B406A9847A36A606A1B6B0F217B
:1068200098472946204601AAFDF7FAFE204601991D
:10683000FEF7ACFD03B030BD10B4026A04464078E8
:106840000B46012803D1104610BC00F03EBEA16AE1
:10685000606A203110BC00F047BE00002DE9F04F07
:106860000F46044685B0C5681E460E9B2946039315
:10687000AB1CC36002920122FDF782FD394600275E
:106880002046FDF7EBFFA36A05F1010A00225146FD
:10689000D3F89430606A9847A36A29469B6A606A75
:1068A0009847A36A606AD3F8D0309847D4F80C8030
:1068B00008F10103E360029B9F4218DB2046FDF7CD
:1068C0006FFDA36A606AD3F8D4309847A36A514633
:1068D0009B6A606A984720460399FDF7BFFF4146CF
:1068E000A36A606A9B6A05B0BDE8F04F184733465B
:1068F000D4F80C901A680436019209F10102E260A2
:10690000019A0137D2F808B0BBF1000F50D1029ABA
:10691000BA4242D10025A36A606ADB6D9847AB4654
:10692000019B2046D968FDF799FF25B3A26A0F2184
:10693000126B606A9047A26A5946926A606A9047F1
:10694000A36A01219B68606A9847A36A0F211B6BA9
:10695000606A984729462046FEF718FD29462046DA
:10696000FFF76AFFA36A606A4FF0FF319B689847A0
:106970002046FDF715FDA36A01224146606AD3F85F
:1069800094309847A36A4946606A9B6A9847A36A0D
:1069900001219B68606A98478DE720461E4A196866
:1069A000FDF7C4FE204605B0BDE8F04FFDF7F8BC8A
:1069B0001BF003052DD19BF804205B46762A03D1FA
:1069C000DD68DBF808B02D09A36A606A5B6D984743
:1069D00059462046FDF742FFA36A0821D3F89C30B0
:1069E000606A9847A36A4A460021DB6E606A98474E
:1069F000002D8FD029462046FEF7C8FCD4F80CB0F5
:106A000020460BF10102E26059460222FDF7B8FC74
:106A100086E70025D8E700BFD47A05082DE9F347BB
:106A20001646DDE90AA9C76898467B1C0D46022276
:106A30003946C3600446FDF7A3FC002E2DD1A36A9E
:106A400003219B68606A984729462046FDF706FFA8
:106A5000A36A6FF002019B68606A9847A36A606A44
:106A60000F211B6B9847A36A3946606A9B6A984757
:106A7000A36A606A9B680121984749462046FDF752
:106A8000EDFEA36A606A4FF0FF319B68984720468D
:106A900002B0BDE8F047FDF783BC434632462946C5
:106AA0002046CDF800A0FFF7D9FED7E77FB5CD6827
:106AB00006462B790C46782B09D1AB68019300234D
:106AC0001A4600938968FFF7A9FF04B070BD742BC4
:106AD0004FF0770103AA16D105F10800FDF7BCF9C4
:106AE0002B6902463BB9EB6800933046039BA168D3
:106AF000FFF7B4FEE9E79B6830460193EB68A168B5
:106B00000093039BDFE704F10C00FDF7A5F90023D8
:106B10000246E9E701F00F03022B2DE9F047054695
:106B20000C4604D1BDE8F0470909FFF785BE0029EE
:106B300056D011F0030653D10B792C2B38D189682C
:106B4000FDF78CFEE668002E4AD016F0030847D108
:106B500077683346FAB28E2A09D13F0A06F108094E
:106B600007F1FF3AC24510DC013756F827301A7991
:106B7000312A12D128469968FDF770FEAB6A686A1F
:106B80000221BDE8F047DB6C1847284659F8041B82
:106B9000FDF764FE08F10108E4E7322A20D1996884
:106BA000AB6A686A0222BDE8F0471B6D0909184705
:106BB0002D2B15D18C689CB163681B0A022B07D062
:106BC00004F108076368B6EB132F10D3BDE8F08714
:106BD000E368002BF4D09A07F2D11B79AC2BEFD1EC
:106BE00021462846BDE8F047044AFDF79FBD2846E8
:106BF00057F8041BFFF78EFF0136E3E7EC7A050830
:106C00002DE9F34143780446012B0D461AD10B7947
:106C1000102B0CBF4FF001084FF0000808D0036A9A
:106C20001B782BB9114A02B0BDE8F041FDF77EBDDB
:106C30006D2101AA05F10800FDF70EF900260746AF
:106C4000B74202D102B0BDE8F081019B002253F8A7
:106C50002610206A0909FDF73DFB434602462946F6
:106C60002046FDF797FD0136EAE700BF007B0508E7
:106C70002DE9F8430646006A0F46C48A904614F090
:106C8000020506D0334A39463046BDE8F843FDF7E1
:106C90004DBD01F00F02022A17D1B37809097BB16B
:106CA000828B013282834FF0010900294FD00022EC
:106CB000FDF710FB03780446002B34D0264AE2E7A8
:106CC000428B1D4601324283EDE70A790D4642456B
:106CD0000BD18968B37809091BB1838B0133838396
:106CE000E1E7438B01334383DDE79A4213D1B57863
:106CF000002DC7D10123B370896841B301F00F02A1
:106D0000022A1CBF0D46A96844F004044FF0030991
:106D1000C4820909C9E7896844F002044FF00509F3
:106D20000909C482C1E7042380F801900370336A23
:106D30001B8B032B0BD1B8F1480F08D13DB1304666
:106D4000E968FDF757FD637843EA00136370BDE817
:106D5000F88300BF5C740508127B050849234822AC
:106D6000FFF786BF4F234E22FFF782BF2DE9F04F7A
:106D70000E46016200214270C16033780446072B41
:106D800015468DB005D08A4A0DB0BDE8F04FFDF72D
:106D9000CDBC012A05D0036B021D29461B68C06AC1
:106DA00098476378D6F80C90032B10D146210BAA94
:106DB00009F10C00FDF750F8236B01469B680B9A14
:106DC000E06A984763687083002B40F0B980D9F877
:106DD0001010C1B101F00F06022E10D10B09752B56
:106DE0003DD006D83E2B3CD05E2B0DD02046714ABC
:106DF000CAE740F252429342F8D1032604E020460B
:106E00006D4AFDF793FC0226D9F81430192109AA1E
:106E100008A80893FDF720F84FF0000A0590059B9D
:106E20009A4520D16378012B15D9236B31465B68D5
:106E3000E06A98476378042B0DD1206A0396438B50
:106E4000E26A02930023CDE900330521D2E9023240
:106E5000006905F095FB6368002B71D114E00026F2
:106E6000D2E70126D0E7099B4FEA8A0B53F82A1094
:106E70000B79082B02D10AF1010AD0E7052B06D0C5
:106E80004E4A2046FDF752FC0DB0BDE8F08F8B68EE
:106E9000002BF5D09807F3D1CA68002AF0D11A79EF
:106EA0002C2AEDD19F6807F00F02022AE8D1DB6897
:106EB0000493002BE4D09A07E2D11B79302BDFD169
:106EC000049BA42103F108000AAAFCF7C5FF40F2C5
:106ED0006A333F099F4280461BD1012805D10A9A97
:106EE000136803F00F03022B04D0354A099B53F8B3
:106EF0000B10C6E7E168012D01F10103E3601AD030
:106F00001268236BE06ADB681209984798B92D4A2A
:106F1000ECE740F256239F4216D1012803D10A9B89
:106F20001968CB0701D4284AE0E7012D03D0E06AB5
:106F3000491001F009F86368002B9CD0DDF810902F
:106F4000D9F80030A3609FE740F2CD239F4224D1BF
:106F5000012804D90A9B1B6813F0010701D11B4AC1
:106F6000C4E7012DE7D05B1006930A9B0BA953F8E9
:106F70002700FCF731FD08B9154AB7E7E36A0B981B
:106F800007930BF0BCF9DDE90613024601371846FA
:106F900000F0E1FFB845E8D1CDE7012DCBD0236B60
:106FA0000246D3F810B039460A9BE06AD847C2E7D8
:106FB0001C7B0508327B0508367B0508477B0508E6
:106FC000557B0508617B0508657B0508717B050815
:106FD000837B05082DE9F04F9BB01446CDE90101F4
:106FE0005822002104A803932AF0E7FC4FF0FF3356
:106FF000012113A88DF81040099307F0D3FA029BE2
:107000000122D90041F0020113A807F001FB01237E
:107010000021436016A80BF0ADFC019A944B0021AF
:1070200093F8B431126804A8FDF7BBFA054611A81D
:1070300000F02CFF4FF0000807468E4B0B9C0D9084
:107040000E930CB1059E26B30B9C14B1059B002B2F
:107050003ED000264146384600F01FFFDFF814926C
:107060000B9CDFF814A2DFF814B2059B002C00F093
:107070002F81002B00F0E1800C9B04A8D968FDF75C
:107080004BFB0C9B069A9B8A0299059809F075FFA9
:1070900021E1238B0122042B214604A807D1FFF70D
:1070A00065FE079BA468984538BF9846C9E7FEF778
:1070B0008FFE238DB342F4D9E36A03EBC60113F8C4
:1070C0003630012B02D12046FDF72CF90136F0E7CE
:1070D000E28A520711D5218D01390ED3E26A02EB03
:1070E000C1025078860720D53BB1D3E900C692E8AB
:1070F000030083E80300C2E900C64FF00003002646
:107100002384B4F828C0664515DB00239C454BD189
:10711000616841B100200346B1F828B0584553DBFF
:10712000002B40F08880A4688FE7002BD4D1012881
:1071300008BF1346D0E72378D4F82C90012B4FEAF0
:10714000C60B09EBC60A05D1DAF804300A2B12D1B6
:107150000136D6E719F836300DD9012B0BD14FF097
:10716000030309F80B30238B032B16D0E38A43F07B
:107170001003E38203E019F80B30032BF3D019F866
:107180000B30042B03D09AF80130DB07E0D5238CB9
:107190005A1C2284AAF80230DAE7DAF8040007F071
:1071A00079F80128EBDCE1E7E26A02EBC30112F8AF
:1071B0003320052A06D14A78D6075FBF228C4A8041
:1071C000013222840133A1E7CA6A02EBC00A12F835
:1071D0003020053A012A14D8002610E0E26A02EBBA
:1071E000C60912F83620062A08D1DAF804E0D9F8E0
:1071F0000420964504BFA9F8023001330136B44596
:10720000ECD101308AE7E06A00EBC20110F83200ED
:10721000062802D14878C00702D54888184448801B
:1072200001329445EFD1628B9BB21A446283228C67
:107230001344238477E70022F3E7238B042B1FD129
:107240000F9B1BB9404604F057FC0F90002303220C
:10725000214604A80D93CDF840B0FFF787FD059BAC
:1072600023B90422214604A8FFF780FDA468FCE6A8
:1072700070030020887C0508847E05088C80050842
:10728000023B012B21D836B9434607AA05A911A80C
:1072900003F07EFD0646CDE90D6A0222214604A8D0
:1072A000FEF796FD059B002BE0D10322214604A8A2
:1072B000FEF78EFD059B002BD8D10422214604A8A1
:1072C000FEF786FD0028F8D0D0E7CDE90D79E4E798
:1072D000002B7FF4D1AE2B69039ADDF81480536044
:1072E000B8F1000F16D0384600F0DFFD002E47D170
:1072F0000F9808B104F015FC0198FCF7A1FF28468F
:10730000AD68FCF7CDFF002DF9D1059800283BD0E2
:10731000F8F7F4FE139C1898C4F3DC0464000334FB
:10732000039B00EB94008000D3F80090F8F708FF6F
:1073300024F003040444C9F80C40DDE91441C9F801
:10734000080001F1040CA0450CD10023189A9342C7
:10735000C9D0199951F82300D9F80C1041F823002D
:107360000133F4E751F838203AB1042A1FBF5CF822
:107370003830D2085B1020F8132008F10108E2E74A
:10738000304603F027FDB3E71BB0BDE8F08F00BF28
:1073900073B5044610200D461646F8F7D1FE084B8B
:1073A00032461B692946009043606B462046FFF732
:1073B00011FEDDE90010002205F0F4F802B070BD06
:1073C000700300208842F8B505460C4601D1012023
:1073D000F8BD224B984201D10020F9E79942FBD039
:1073E00007F03CFB0646204607F038FB8642F3D107
:1073F0001B4B9E4214D16A6863689A42ECD1002606
:1074000005F1080708346B68B342E0D954F8041B4F
:1074100057F8040BFFF7D6FF0028DDD00136F2E75E
:107420002146284607F0EEFD0028D5D00D4B9E42A0
:10743000CDD1284609F0DAFE002105463AF0C6FE15
:107440000028C4D0204609F0D1FE05F0004500F028
:1074500000402B1A58425841BAE700BF4483050840
:10746000C8A1050854900508C90010B501220446BA
:1074700041F00201083007F0CBF843683BB9A3683C
:10748000C3F3DC03013B5B0043F00103436040684E
:10749000C0F34F0010BD70B505460E460024EB69E1
:1074A000A34208D8314605F114000BF023F9EC692A
:1074B000013C204670BD2B6A314653F82400FFF78B
:1074C00081FF0028F5D10134E9E710B50122044617
:1074D000FCF700FF0378012B05D12378012B8CBF2B
:1074E00004230223037010BD70B505460E461046F6
:1074F00019461C46FCF7DEFE03785A1E012A06D800
:107500000022736821462846BDE870401847032BC7
:1075100002D101227368F5E73668042B2146B44690
:10752000428808BF00232846BDE8704018BF0123E9
:1075300060474379012B07D0836819440369816050
:107540005A8C9142C8BF5984704700238371437994
:10755000012B1EBFC26A036A43F8212070476FF0F7
:107560000301FFF7E6BF0421FFF7E3BF6FF002015D
:10757000FFF7DFBF0346426A4079114403288ABF00
:10758000586B1846801859627047827903460AB1D1
:10759000184670475A79C06A032A014401D8D96253
:1075A000F6E79A6AD9620244586B1044704710B5E6
:1075B0000C460121FFF7E9FF047010BD10B5144619
:1075C000FFF7B7FF0121FFF7E0FF047010BD532262
:1075D0000121FFF7F3BF54220121FFF7EFBF57222C
:1075E0000121FFF7EBBF58220221FFF7E7BF592225
:1075F0004FF0FF31FFF7E2BF5A220021FFF7DEBF55
:107600005B220021FFF7DABF5D224FF0FF31FFF769
:10761000D5BF002915BF5F225E2203210021FFF79D
:10762000CDBFA1F13002D2B20021FFF7C7BF622265
:107630006FF00101FFF7C2BF10B563224FF0FF31B9
:107640000446FFF7BBFF0123A37110BD01F16402E3
:1076500010B5D2B249420446FFF7B0FF0123A3712F
:1076600010BD10B5044601F16702D2B24942FFF7DE
:10767000A5FF2269D38A43F00103D38210BD000025
:1076800038B504461D46FFF799FF2A462046BDE857
:107690003840014913F0ACBE8B75010870B5044643
:1076A0000D46C06819461646FFF7DEFE3246034611
:1076B00029462046BDE87040FFF7E2BF0B46102286
:1076C0000121FFF7EBBF11320B46D2B20121FFF7C8
:1076D000E5BF002A0B464FEA4201C1F1010114BF88
:1076E00015221422FFF7DABF16320B46D2B24FF042
:1076F000FF31FFF7D3BF19320B46D2B20021FFF79B
:10770000CDBF70B41D46C46826786388042E04BFBC
:10771000666846F823505D1C658070BCFFF7B0BFFB
:1077200003F128011346CAB20021FFF7A9BF022ABC
:1077300002F12A020B46D2B20CBF0121C1F10101B4
:10774000FFF79EBF03290AD004290BD00021022392
:107750000A4443EA8203C9432F22FFF791BF002165
:107760000B46F5E70121FBE70B4630220139FFF715
:1077700087BF10B4144641EA02232144312210BCD1
:10778000FFF77EBF012A10B40B46044607D0022A39
:107790000CD169224FF0FF3110BCFFF70FBF11462B
:1077A0001B322046D2B210BCFFF778BF4FF0FF313A
:1077B000F6E7F8B516461F46FFF7BBFE8479054687
:1077C00004BB4379022B25D9C46A036AC4F1FF24A0
:1077D00053F8273004F57F04FE34442E1C4412D89D
:1077E00014F1400F14DB3F2CD4BF00270127E41B0A
:1077F0002846B91CFFF7C9FE06706FB9442E98BF22
:1078000040344470F8BD7F2C94BF00270127EEE779
:107810000127ECE70127EBE76B79442E98BF04F5CD
:107820008044042B05D1B4F5004F24BF012385F813
:10783000383064F07F03E41143708470E2E70B4654
:1078400010B5422200210446FFF7B3FF0123A371C4
:1078500010BDF8B505460C46164621F40047CAB9D6
:107860000B040ED55921FFF7A2FE59212846FFF738
:107870009EFE59212846FFF79AFE59212846FFF718
:1078800096FE3B46422200212846FFF792FF012345
:10789000AB71F8BD3B4640220021FFF78AFF210A69
:1078A00021F07F0131432846C9B2FFF780FEEEE7A1
:1078B000002A02F147020B46D2B20CBF022100217E
:1078C000FFF777BF0B464B220121FFF772BF0B4634
:1078D00010B54A2200210446FFF76BFF0123A37174
:1078E00010BD0000264B2DE9F047D3F8B031044617
:1078F000022B89460ED88669B1420BD940F2FF7738
:10790000C56A43698E1BED1A56EA050304D1E36A82
:10791000C4E90539BDE8F087062E01D90F2D1AD923
:107920001F2DAA4628BF4FF01F0A554510D8032E19
:10793000B04628BF4FF0030801212046FFF71AFE8A
:107940004AEA48130370A5EB0A05A6EB0806DBE735
:107950004FF00008F0E7BE42B04628BFB84602210B
:107960002046FFF707FE4FEA181303F070032B437E
:1079700063F07F03AA46037080F80180E3E700BF4D
:107980007003002010B5044631B955224FF0FF3185
:10799000BDE81040FFF712BE022904D1FFF717FE21
:1079A0002046FFF72DFE56226FF002012046EFE73A
:1079B000134621B143224FF0FF31FFF7FABE4422B4
:1079C000F9E7134621B145224FF0FF31FFF7F1BE31
:1079D0004622F9E7322938B5044612D0332913D1AB
:1079E000012507212939CAB220464FF0FF31FFF7A0
:1079F000E5FD5DB12046BDE83840D3220021FFF708
:107A0000DDBD01250621EDE70025EBE738BD70B5AA
:107A10000D46044611462AB92B461322BDE8704094
:107A2000FFF73CBE022A04D1FFF7D1FD2046FFF745
:107A3000E3FD2B4618226FF001012046EEE710B45B
:107A400004463BB90F2A05D8503A012110BCD2B2E6
:107A5000FFF7B4BD03F124012046134610BCCAB29F
:107A60000121FFF70DBE10B4044643B90F2A06D812
:107A7000403A4FF0FF3110BCD2B2FFF79FBD03F187
:107A800026012046134610BCCAB24FF0FF31FFF763
:107A9000F7BD70B4D2B2DDE9036503EB460443EAF7
:107AA000062315B101320134D2B2091B70BCFFF7B5
:107AB000E7BD07B5CDE900230B4634220021FFF7CF
:107AC000E8FF03B05DF804FB07B5CDE900230B46E2
:107AD00036224FF0FF31FFF7DCFF03B05DF804FB07
:107AE00010B50446C068FFF7D6FC232203460121E7
:107AF0002046BDE81040FFF7C3BD01F110033F2B46
:107B000073B506460C4608D8A1F180020121D2B215
:107B100002B0BDE87040FFF751BD012122220DF1F6
:107B20000505FFF74BFD294604F07F00E3B2E411A1
:107B30002A4605F8010D601C0128F5D8013403F030
:107B4000400313D11BB97F2305F8013C951E491B47
:107B50003046FFF71AFD2B46014601ACA34209D17E
:107B60009DF804205B1BC25402B070BD002BEED008
:107B70000023E9E713F8012B62F07F0201F8012BE3
:107B8000ECE7F8B51F4614460546D6B2069A0B69CF
:107B90003A4313BFE143C4F1010120222122FFF740
:107BA000B0FD31462846BDE8F840FFF700BD10B4EF
:107BB0001C4622430B6907BF3222012133224FF0BA
:107BC000FF3110BCFFF79DBD0D2910B504460BD148
:107BD0000949C068FFF75FFC2322034601212046C4
:107BE000BDE81040FFF74CBD4231CAB2BDE81040BD
:107BF0000121FFF7E3BC00BFE89A050838B5044649
:107C00000D460F21FFF7E0FF20462946FFF79DFCB8
:107C100002215C22FFF7D2FC2046BDE838406FF01D
:107C20000301FFF786BCF8B504460F4616461D460D
:107C30000F21FFF7C9FF2046FFF7DEFC394620463B
:107C4000FFF7FDFD31462046FFF77FFCFFF7C7FC3D
:107C5000012220462121FFF736FD20460821FFF7AB
:107C6000B9FE2A462046BDE8F8400021FFF7A0BE35
:107C7000437970B5012B044601D1012034E0002581
:107C8000C26B436A05649B1AC3632069038D9D42DE
:107C90000BD36379032B1AD1606AE36AA062236372
:107CA0001844F8F766FA6063E7E7C36A03EBC502B6
:107CB00013F83530052B08D1012120469678FFF7BF
:107CC00059FC0670236C013323640135DDE7042B76
:107CD000D3D1D4E90A13626A8A4202D1216B994254
:107CE00003D00020A262236370BD94F838301BB12A
:107CF0000549064805F0A4F8E268C38A5268616B3A
:107D0000006904F034FCB8E77C7C0508A88E0508FF
:107D100000232DE9F74F1646C0E904230122378CD2
:107D200083608371C362436280F83830738C044689
:107D30001F44974238BF1746B6F82490B6F81A8009
:107D40004FEA8905013F826105F0040508F003024E
:107D50001543B6F816A0FA0002F07802B38BB6F815
:107D60001EB041710AF00F0A15433F094FEA590945
:107D70004FEA980847EA090242EA0A0242EA080280
:107D80001A4352EA0B0235D101212046FFF7F2FBDC
:107D900005706379022B18D9D4E90F787D0008F0BB
:107DA000010305F07E054FEA5808BF091D4358EA54
:107DB00007094FF00101204618BF45F08005FFF785
:107DC000D9FB0570B9F1000FE8D1636AB18AE363AA
:107DD000E068FFF749FB2C490246204613F008FBF8
:107DE0000025294F738BB28B1344AB4248DD002230
:107DF000318D41E0012120460193FFF7BBFB65F087
:107E00007F053A0105704FEA8A15019B02F03002A6
:107E100005F0400515430BF001021543DA0002F0AE
:107E2000080215434FEA880202F0040215434FEAA4
:107E3000490202F002021543BF084FEA59094FEA0E
:107E40005A0A4FEA58085B084FEA5B0B92E7F36A5D
:107E500003EBC2035878C0070DD55888A8420AD151
:107E60005968E068FFF700FB39460246204613F0E8
:107E7000BFFA0135B6E701329142E8DC0521F0E7AF
:107E800003B0BDE8F08F00BF7575010810B504465A
:107E90004420F8F76EF9C46010BD10B50446C16106
:107EA0008800F8F74DF9206210BD10B50446006A4D
:107EB000F8F76EF92046BDE81040F8F769B910B53B
:107EC000044601618800F8F73BF9606110BD10B508
:107ED000044611B1C068F8F75BF96069BDE810406D
:107EE000F8F756B9012938B504460D460BDC02698E
:107EF0004FF0FF314069920029F05FFD00232570AB
:107F00006370636038BD4068F8F71AF96368E06031
:107F1000A360F3E70246407810B548B91378546877
:107F2000022B08BFD368214408BF1819516010BD47
:107F30000020FCE7002343700378012B9EBF4268BA
:107F4000436943F82120704742684B1E134449425D
:107F500019404160704738B50C461546FFF7DAFF07
:107F600010B10444A04200D138BD00F8015B2D0AD5
:107F7000F8E710B50C460221FFF7CCFF10B10470F2
:107F8000240A447010BD38B50D4604211446FFF78D
:107F9000C1FF28B1057084702D0A240A4570C47091
:107FA00038BD0000032970B58DBFFE260024134B99
:107FB000023994BF5E5C21F0010446F43541054668
:107FC000FFF7D7FF44B17F2C09D844F4304128464D
:107FD00041F08001FFF7CDFFC5E9066470BDA30045
:107FE000A201DBB202F4E0421A434FF2AD2128466F
:107FF00042F45062FFF7C7FFEEE700BF727D05084D
:10800000C16910B5044629B17F290BD841F430412C
:10801000FFF7AFFFA1692046BDE8104041F43D41A4
:10802000FFF7A7BF8B008A01DBB202F4E0421A43DC
:108030004FF20D2142F45062FFF7A5FFEAE711432A
:1080400041EAC301FFF795BF072A85BF083AD2006E
:10805000D20042F04002072985BF0839114311437D
:1080600041F0800141F48C41FFF783BF30B4DCB2B2
:1080700044EA02225C101D0104F48064C3F303335C
:1080800005F4E04523432A43194330BCFFF77BBF87
:1080900038B50546436953F821404368E41A043C67
:1080A000C4F34A0141F46041FFF763FF2B78022BD0
:1080B0000AD124F4FF6020F0070028B110F5006F0A
:1080C00014BF0020012038BD0120FCE770B54469D1
:1080D000054654F8224042681E46A41A043C621029
:1080E000ABB9D2B242EA012141F45041FFF741FF5E
:1080F0002B78022B09D134F0FF0606D016F5807FCD
:1081000014BF00260126304670BD0126FBE763112F
:1081100003F40053A512C2F30A021A4305F4806562
:108120002312C4F3053403F400632C431A4344EAD6
:10813000811142F4004241F47041FFF724FFE2E76D
:1081400038B50546436953F821404368E41A043CB6
:10815000C4F34F02C4F30A3142F4784241F470414F
:10816000FFF711FF2B78022B08D1A00D800528B155
:1081700010F5800F14BF0020012038BD0120FCE75E
:10818000F8B504460D461646476813460A464FF2B0
:108190004021FFF76BFF20462A464FF2C021330CE7
:1081A000FFF764FF3846F8BD072910B4044609D824
:1081B00032F0FF0306D142EA012110BC41F4005124
:1081C000FFF7D7BE130C1B043BB9134620460A46E3
:1081D00010BC4FF24021FFF749BF204610BCFFF70B
:1081E000CFBF2DE9F843072906460C461546DDF8B2
:1081F00020904DD8072A4BD803FA09F7FF2F0CD847
:10820000914201D0FFF720FF47EA042141F4405199
:108210003046BDE8F843FFF7ACBE33F0FF024FEA4B
:10822000C10814D1A94218D043EA012343F40051F4
:10823000FFF79FFE44EA8911304641EA0801FFF743
:1082400098FE48EA8511214341F4C051E0E7A94274
:1082500003D03A46FFF7A8FFF3E7012584F00709AA
:1082600005FA09F5304645F43441FFF782FE3A46F7
:1082700049463046FFF798FF44EA891141EA080170
:1082800041F4C0513046FFF774FE45F43C41BFE76E
:10829000BDE8F88308B50378012B05D931F0FF0359
:1082A00002D0064805F0EAFDC9B241EA022141F4D4
:1082B0001041BDE80840FFF75CBE00BF607D0508C7
:1082C00008B50378012B05D932F0FF0302D0064828
:1082D00005F0D4FDD2B242EA012141F41841BDE8D3
:1082E0000840FFF746BE00BF607D0508D2B242EAF3
:1082F000012141F42841FFF73CBE38B50C46054644
:10830000436953F8223042689B1A43F001030A463E
:108310000A3B4FF24021FFF7A9FE2346284622469A
:108320004FF43241FFF78BFE210101F0800104F090
:108330000704214341F488412846BDE8384041F014
:108340007801FFF716BE000073B50C4633F01F012D
:108350000546069E12D1072C10D8072A0ED81B49B5
:1083600044EAC202895D41F0010142EAC12141EAC9
:10837000831102B0BDE87040FFF7FBBD03FA06F0C1
:1083800020F47F6121F00F0169B942EA461140EA09
:108390000432284641F4784141F0900102B0BDE832
:1083A0007040FFF7F0BD214628461F3B0096FFF7BF
:1083B00018FF064B2846995D41F0010144EAC121AE
:1083C00041EAC40141F4F861D3E700BF767D0508B6
:1083D0002DE9F7431D4635F01F0307460E461446A8
:1083E000DDF8288011D107290FD8072A0DD8224B94
:1083F00041EAC40113F8082041EAC22141EA85118B
:1084000003B0BDE8F043FFF7B4BD05FA08F222F46B
:108410007F6323F00F036BB9384644EA481141F4F7
:10842000784142EA063241F0800103B0BDE8F043F2
:10843000FFF7A9BD4FF0010909FA04F9384649F4DC
:108440003441FFF796FD224621463846A5F11F0329
:10845000CDF80080FFF7C5FE074B46EAC40113F8CC
:108460000820384641EAC22141F4F861FFF781FD56
:10847000384649F43C41C3E7767D0508436930B48A
:1084800053F8211043680446CB1A043B0131C3F36F
:108490004A020DD0D91C0BDA23F4FF6525F007053D
:1084A00015F5006F04D130BC42F46041FFF761BDA7
:1084B000C3F30A33204630BC42F4384243F47041DF
:1084C000FFF761BD436930B453F822404368054665
:1084D000E31A043B01344FEA63020ED0DC1C0CDAD1
:1084E00023F0FF0414F5807F07D130BCD2B242EAFA
:1084F000012141F45041FFF73CBD581100F40050F8
:108500009C12C2F30A02024304F480641812C3F3FB
:10851000053300F400602343024343EA81112846F7
:1085200030BC42F4004241F47041FFF72CBD37B536
:108530001446022205460B46009221460722FFF709
:1085400003FF2846E10041F48F4103B0BDE830400D
:10855000FFF70FBD07289ABF024B33F8100040F217
:1085600093107047727E0508C36C19440369C16497
:10857000012B04DD436D5A8C9142C8BF598470476A
:1085800070474FF0FF31FFF7EFBFFFF7FABF6FF013
:108590000301FFF7E9BF70470B46D0E90C2102F158
:1085A0008042013A01EB820210B50446D0786FF3A5
:1085B000C710D070043A91420BD892F903000028FA
:1085C000F8DA12880021A06DC2F30E02FFF795FEC3
:1085D00006E063B91A4644F24001A06DFFF72FFD93
:1085E000A06D0022BDE810400321FFF753BE10BD6F
:1085F00038B5C46C036A21449942054608D908314C
:1086000021F00304406AE100F7F7B5FDC5E9084031
:1086100038BD70B504460E4601211546FFF7E8FF48
:10862000E16C626A204602F8316002EBC10301216D
:1086300059705D60BDE87040FFF796BF10B5044605
:108640000121FFF7A9FFA06D01220021FFF738FEED
:1086500000222046BDE810401146FFF7DABF70B592
:1086600004460E4601211546FFF7C2FFE16C626A1F
:10867000204602F8316002EBC10302225A705D60AD
:108680000121BDE87040FFF76FBF00221146FFF7E0
:10869000E6BF0A460221FFF7E2BF38B50D1E0446C9
:1086A00014DDFFF7A5FF0020626AE16C02EBC10355
:1086B000294402EBC102012D18BF0021587008BFE8
:1086C00094F8281003F8081B9A42F4D12946204652
:1086D000BDE83840FFF748BFF8B5D0E90B53013388
:1086E000AB4204460E46174606D90435406BA90036
:1086F000F7F741FDE5626063D4E90C30C6F30E0183
:108700005A1C226341EAC73220F8232000EB83057C
:108710004FF6FF733246A06D00216B80FFF7EDFD31
:10872000A06D0022BDE8F8400321FFF7B3BD03466A
:10873000007D28B1C943DA6C5B6A114413F831003B
:10874000704737B50446646D0B46E48A1546E40766
:10875000806D07D50222294600920622FFF738FED7
:1087600003B030BD03B0BDE83040FFF793BD70B536
:10877000002405462646EB6CA34200DC70BD6B6A04
:1087800003EBC4035A78012A07D15E70B5F84A108A
:1087900028465A682144FFF7D4FF0134EBE7F8B5C7
:1087A00004461E4617460D46FFF7E1FF3A4631469E
:1087B000A06DFFF7F9FC2946A06D0322BDE8F84043
:1087C000FFF7B5BE38B504460D46FFF7D0FF294682
:1087D000A06D0322BDE83840FFF7A9BE10B50821FF
:1087E0000446FFF7EFFF00222046BDE81040114687
:1087F000FFF70FBFF8B5044617461E460D46FFF7B4
:10880000B6FF3A46A06D0021FFF7CEFC3246A06DC0
:108810000121FFF7C9FC2946A06D0322BDE8F840FD
:10882000FFF785BE2DE9F041002405460E46A0461F
:10883000C76CBF1AEB6CA34201DCBDE8F081BC42FF
:1088400011D06B6A03EBC4035A78012A0BD15A6822
:10885000B24208D183F80180B5F84A103246284662
:108860002144FFF76EFF0134E4E7002238B50C46DF
:1088700005461146FFF7D6FFE200A86D002142F041
:108880000202FFF791FC00222846BDE8384011465D
:10889000FFF7BFBE13B50446646D1346E48A806DCE
:1088A000E40706D5022200920622FFF74DFD02B032
:1088B00010BD02B0BDE81040FFF702BDF8B5C369B6
:1088C00004469E5C1546602E06D147680A4613484A
:1088D000134908F013FB3860022D0DD8636D9A8C94
:1088E00052B9DB8ADB0707D40E4B5A5D314620466E
:1088F000BDE8F840FFF78DBE0022ED43114620464B
:10890000FFF790FFB4F84A20636C00211A442A4410
:108910002046FFF7BFFF0022E8E700BFC88F050829
:10892000797D0508747F050873B5036804461A78D5
:108930005D88042A08BF5A684FF0020608BF42F853
:1089400025106A1C5A800021B0F84820FFF7A2FFCA
:10895000002233461146A06D0096FFF7F5FC002279
:108960002B461146A06D0096FFF7EEFC02B070BDDD
:10897000002273B504460D461146FFF753FF626DA2
:108980002946D38A206843F02003D382FEF783FD73
:10899000B4F84820054600212046FFF77BFF022659
:1089A0000022A06D114601230096FFF7CDFC0022A6
:1089B000A06D114603230096FFF7C6FC0022A06DB0
:1089C00011462B460096FFF7BFFC002220461146B9
:1089D00002B0BDE87040FFF71CBE00000D2902D1B7
:1089E0000749FFF7C5BF0F2903D100225421FFF724
:1089F00036BEB1F10E0218BF01220121F7E700BF18
:108A0000E89A0508F8B5C76C446A07F10053023BC1
:108A100004EBC3040546D4E9020184E80300667848
:108A200056B9B5F84A2031463A442846013AFFF78C
:108A300031FF0123666063702846BDE8F8404FF0BF
:108A4000FF31FFF791BDF8B504461E4617460D46A7
:108A5000FFF78DFE3A463146A06DFFF7A5FB29468C
:108A6000A06D0322BDE8F840FFF761BD10B402F12C
:108A7000290400230A46E1B210BCFFF7E4BF70B539
:108A800004460E46154662B1037D53B1084605F013
:108A900001FC021E05DD2046BDE870407021FFF795
:108AA000DEBD063532462046E9B20023FFF7CBFF94
:108AB00000222046BDE870401146FFF7AABD07B569
:108AC0001346022200920722FFF73EFC03B05DF836
:108AD00004FB000070B50E46154643B9037D33B163
:108AE0005268806DFFF760FB2C78204670BD2C78B3
:108AF0002CB931466A68806DFFF756FBF5E7012C0B
:108B000006D16A6801323146806DFFF7D8FF0AE06E
:108B1000A31E012B09D86A6831465200806D42F0CD
:108B20000102FFF741FB0024DFE7542C01D10022B2
:108B3000E9E7014805F0A2F98E7D0508F8B50024A3
:108B400005462746FFF713FEEB6CA34200DCF8BD99
:108B50006E6A06EBC4025378022B0ED101215770C6
:108B600000232846FFF7B6FF06F83400B5F84A1090
:108B7000012228462144FFF7E4FD0134E4E738B53B
:108B800004460D46FFF7DAFF2946A06DFFF776FC95
:108B90000122A36D5A7038BD38B50D460446114602
:108BA0007AB10022806D1146FFF7FEFA0022012102
:108BB000A06DFFF76FFB29462046BDE83840FFF760
:108BC000DEBFFFF7E9FCF6E72DE9F04104460E466B
:108BD000CAB3D0E90C51002305F18045013D01EBFA
:108BE000850528461746984690F901C0BCF1000F4C
:108BF00012DA90F903C0BCF1000F0DDAB8F1000FE2
:108C000008BF80463BB1B0F800E0B3F802C06EF395
:108C10000E0CA3F802C00346013FA0F10400E3D10B
:108C20006FF003004243A06D05EB020CCBB9614528
:108C300010D91A4644F24001FFF701FA002203213D
:108C4000A06DFFF727FB204626F40041BDE8F04168
:108C5000FFF795BFAA5A1946C2F30E02FFF74DFB64
:108C6000ECE747F6FE715A8861F30E025A803946E6
:108C700026F40042FFF741FB3A460D21A06DFFF7B5
:108C800009FB3A463946A06DFFF78EFA3A460121B4
:108C9000A06DFFF7FFFAB8F80060C6F30E06D2E742
:108CA000F8B504460E4617460A4619461D46FFF714
:108CB000B9FDE36C616A9B1B01EBC30211F8333011
:108CC0003B705378012B0DD0022B14D0CBB9B4F8E4
:108CD0004A20E36C29461A442046921BBDE8F8401E
:108CE000FFF7D8BD5268AA420BD02946A06DBDE857
:108CF000F840FFF7A9B9002329462046FFF7EAFE0E
:108D00003870F8BD10B5044613460A460121FFF736
:108D1000C7FF2046BDE810404FF0FF31FFF724BCED
:108D200070B504461D46049EFFF7ECFF3246294607
:108D30002046BDE87040FFF7E5BFF0B501250446C9
:108D400085B00DF10F030DF10E0100220095FFF724
:108D5000E7FF9DF80F709DF80E602A4639462046C1
:108D6000FFF757FC314620460022FFF752FC2A4607
:108D700039462046FFF74DFC002231462046FFF7DA
:108D800048FC05B0F0BD2DE9F0410446DDE906865A
:108D90001D46089FFFF7B6FF424629462046FFF7CB
:108DA000B1FF3A4631462046BDE8F041FFF7AABF81
:108DB0002DE9F04102260125044686B00DF1170386
:108DC00001930DF115010DF1160300220296009595
:108DD000FFF7D9FF9DF8178020469DF816709DF883
:108DE00015100022FFF715FC324641462046FFF7DA
:108DF00010FC2A4639462046FFF70BFC06B0BDE8BA
:108E0000F08130B587B00DF11703002501930223DF
:108E10000446012200930DF115010DF11603029590
:108E2000FFF7B1FF20461921FFF7CCFC2A4629465F
:108E30002046FFF7EEFB07B030BD73B504460E4683
:108E4000154672B901220DF10701FFF75BFF002300
:108E5000324620460C35E9B202B0BDE87040FFF75B
:108E6000F2BD0021FFF763FC8DF8070020B9012255
:108E700020460DF10701E8E720460DF10701002229
:108E8000FFF740FF20469DF8072001230421FFF74C
:108E900086FC00220121A06DFFF7D6F8D7E700007D
:108EA00037B500220DF107010446FFF72BFF9DF8AF
:108EB00007302BB107490848656808F01FF828609B
:108EC00022212046FFF77EFC0122A36D5A7003B0D9
:108ED00030BD00BF937D0508C88F0508022A7FB505
:108EE00004460E46154614D8436D9A8C8AB9DB8A1F
:108EF000DB070ED4184B0DF10F015A5DFFF702FF8F
:108F0000E3699DF80F10585D602813D1595504B0DE
:108F100070BD20460DF10F010022FFF7F3FE636CD8
:108F2000B4F84A1000221944EB4320461944FFF7D5
:108F300008FCE5E78842EAD0FFF70CFB024608464A
:108F4000FFF708FB05496468134600903246044861
:108F500007F0D4FF2060DAE7747F05089D7D0508DF
:108F6000C88F050873B5046B05460E46DCB1436B2C
:108F700004F18044013C03EB840292F90120002AB1
:108F800020DA33F82430C3F30E038B421AD10023C6
:108F900001210DF10702FFF783FE00220121A86DD8
:108FA000FFF778F901242846FFF7C8FD3146A86D80
:108FB000FEF7C0FF44B10021284602B0BDE8704072
:108FC000FFF7EABA0024EEE702B070BD03297FB5CF
:108FD0000446164612D101220DF10F01FFF792FE51
:108FE00018250023314620460DF10F02FFF758FEE9
:108FF00029462046FFF7E6FB04B070BD052906D1DF
:1090000001220DF10F01FFF77DFE1725E9E702238D
:10901000012200930DF10E010DF10F03FFF780FE09
:109020001925DEE77FB504460E46154682B90DF1D7
:109030000F01FFF767FE3246092120460123FFF7A3
:1090400002FD2A4629462046FFF7E3FA04B070BD28
:10905000012A35D11146FFF76AFB02468DF80F0051
:1090600078B90223204600930DF10E010DF10F0394
:10907000FFF756FE012332460E212046FFF7E3FCA0
:10908000E4E720460DF10F0200230221FFF708FE5E
:109090002B4620469DF80F200421FFF780FBA06D92
:1090A00000220221FEF7D0FF20460DF10E01002222
:1090B000FFF728FE4FF0FF312046FFF755FAD9E7BA
:1090C0000DF10F010022FFF71DFE022344F24001C3
:1090D0001A46A06DFEF7B3FFCCE7F0B504460E4686
:1090E000154685B0C2B90223077D0DF10E01027548
:1090F000012200930DF10F03FFF712FE2B463246BB
:10910000232127752046FFF79EFC002220461146AA
:10911000FFF77FFA05B0F0BD012A09D100232946E7
:109120000DF10F02FFF7BCFD2B4632462421E9E783
:109130000DF10F010022FFF7E5FD25212046FFF785
:1091400041FBE7E72DE9F3410E46002117460446AF
:109150001D46FFF7ECFA02468DF8070048BB204693
:109160000DF10701FFF7CEFD1DB901212046FFF7E4
:10917000FBF910212046FFF725FB1DB99DF80730AC
:1091800084F828302046FFF7D9FC4FF42051A06D19
:109190005EB3FEF7EEFE3A460121A06DFFF792F9AD
:1091A00025B94FF0FF312046FFF7DEF902B0BDE8E8
:1091B000F081002220460DF10701FFF7A3FD1DB944
:1091C00001212046FFF7D0F99DF80700431E022B2E
:1091D000D3D9FFF7BFF9074902460748D4F80480FE
:1091E00007F08CFEC8F80000C7E7FEF7C2FE3A465B
:1091F0003146D2E7AD7D0508C88F05080023FFF78B
:10920000A1BF0123FFF79EBF38B50446FFF7B9F9A8
:1092100001220021806DFFF753F822212046FFF73D
:10922000D1FAD4E90C3547F6FF72013B05EB830513
:1092300023636B88C3F30E03934228D00D220021D1
:10924000A06DFFF73DF84FF42051A06DFEF791FEA1
:10925000A36800211A68A06DFFF734F947F6FE7382
:109260006988C1F30E029A420BD14FF48E41A06D72
:10927000FEF77FFEA36820461968BDE83840FFF777
:1092800071BE2046C1F30E01FFF779FCF2E738BD4D
:1092900083682DE9F3411E68436D0446DD8A9B8C8B
:1092A00005F011021343C66000F0FD8015F00105C2
:1092B00006F1020721D14FF00208B0F848202946F4
:1092C000FFF7E8FA01232A462946A06DCDF8008071
:1092D000FFF73AF82A4601232946A06DCDF8008011
:1092E000FFF732F805212046FFF76CFAB4F8481072
:1092F0002A4620460131FFF724FAD4E915309A8C2A
:10930000002A67D1D98A11F0010508D14FF4205104
:10931000FEF72FFE3A462946A06DFFF7D3F800224C
:10932000A06D1146FEF7E2FF20212046FFF74AFA22
:109330004FF42051A06DFEF71CFE3A460021A06DAF
:10934000FFF7C0F8636DD98A11F0010100F0928037
:10935000022501220021A06DFEF7B2FF052306229F
:109360000021A06D0095FFF733F8A06D2A4600217B
:10937000FEF71AFFA06DFEF743FE39462046FFF7C1
:10938000F1FD636DDB8ADB0740F18D80B4F8482086
:10939000204601320021FFF77DFAA06D4FF48E4187
:1093A000FEF7E7FDA06D0E22436800212364FEF75F
:1093B00087FFA06D00220121FEF7F6FEA06D0122BD
:1093C0000E21FEF767FF2221204602B0BDE8F041E2
:1093D000FFF7F8B9002344F240011A46FEF72FFECA
:1093E00000220D21A06DFEF755FF00220121A06D86
:1093F000FEF750FF751C3A460421A06DFEF77DFF75
:1094000029462046FFF7AEFD0022A06D1146FEF76B
:109410006DFF20212046FFF7D5F903364FF4205188
:10942000A06DFEF7A6FD32460121A06DFFF74AF8B8
:10943000002344F240011A46A06DFEF700FE002210
:109440000321A06DFEF726FF44F22071A06DFEF708
:1094500090FD31462046FFF785FD03220421A06DD3
:10946000FEF72EFF4FF43051A06DFEF782FD2A4625
:10947000012164E7B4F8482020460132FFF70AFAD8
:1094800005212046FFF79EF9636DD98A11F001018D
:109490007FF45EAFA06D0122FEF712FF222120466D
:1094A000FFF790F969E702B0BDE8F08170B50546B5
:1094B000D0E91560F68A0C46F6070BD544EAC404D9
:1094C0009200FEF771FEA86D44F4CC51BDE87040E7
:1094D000FEF74FBDBDE87040FEF708BF2DE9F84F1D
:1094E000002504460F469146A846FFF740F94D4532
:1094F00010D10026B3464E452BD171422046FFF7CE
:1095000033F8B4F84A20E36C39461A44BDE8F84F02
:10951000FFF7CCBFE66CD4F824A0013E761B0AEB23
:10952000C6025378022B12D10123394682F80180FA
:109530002046FFF7CFFA0AF83600B4F84A10E36C79
:109540003A46194401392046491BFFF7FAF801351C
:10955000CDE7E36CD4F824A003F1FF38A8EB0608AC
:109560001AF83820BAB1B4F84A5000211D44013D20
:10957000AD1B2A462046FFF78DF901230421204622
:109580001AF83820FFF70BF9002229462046FFF78A
:10959000D8F80AF838B00136ADE7F8B516460446F3
:1095A0000D46520093B1CB1C1A440221FFF796FFDF
:1095B00001221D2145EA06232046FFF71BF9002260
:1095C0002046BDE8F8401146FFF723B88B1C1A442B
:1095D0000221FFF783FF33462A461C21ECE72DE9E1
:1095E000F7430F4616460121B0F848201D460446B1
:1095F000DDF828904FF00208FFF74CF90123A06D29
:109600001A461946CDF80080FEF79EFE55EA090578
:109610002DD12046FFF7ABF82A464146A06DFEF754
:10962000C3FD20463969FFF77FF903221A21A06D97
:10963000FEF77DFF32460121A06DFEF7B5FD3246F3
:1096400002212046FFF74AFF25B16FF001012046B5
:10965000FEF78AFFA06D03222B21FEF768FF002290
:109660002046114603B0BDE8F043FEF7D2BF06F135
:1096700002094A4641462046FFF730FF4946204648
:10968000FEF772FFFFF773F8CBE72DE9F3411546BC
:109690000F46B0F8482001211E4604464FF002084C
:1096A000FFF7F8F80123A06D1A461946CDF800809F
:1096B000FEF74AFE354318D12046FFF758F82A46F0
:1096C0004146A06DFEF770FD20463969FFF72CF981
:1096D000A06D03221A21FEF72AFF00222046114620
:1096E00002B0BDE8F041FEF794BF20464246414635
:1096F000FFF7F4FE2046FFF73AF8E5E770B5042AD5
:1097000004460E46154686B02AD102294FF00005C0
:1097100018D101220DF1170100950DF11603FFF785
:10972000FFFA2A463146A06DFFF7C9F926212046E7
:10973000FFF748F800222046114606B0BDE8704009
:10974000FEF767BF0DF11503019301230222009379
:1097500002950DF116030DF11701FFF714FBE5E774
:10976000012A01D9032A04D1324601212046FFF7FC
:10977000B5FE1335002332462046E9B2FFF70FF855
:10978000D8E70000037D37B504460D4613B15F48A6
:1097900004F074FB426DD38A43F00103D382FFF7D8
:1097A000CDF9012D0BD1A368204619680231FFF7CE
:1097B000E6F9A368204619680131FFF7D3FB0122BF
:1097C00000212046FFF78AFE002202212046FEF7F4
:1097D000B8FF01220021A06DFEF7E6FC00220C215B
:1097E000A06DFEF757FDA36800211A68A06DFEF773
:1097F00084FDB4F84810002220460131FEF7A1FF95
:10980000E168A06DFEF73AFEA368A06D1968FEF747
:1098100091FB236BBBB1626B03F18043013B02EB15
:1098200083039A420FD893F90310002926DA1A8885
:109830000021A06DC2F30E02FEF75FFD002203219E
:10984000A06DFEF727FD01212046FEF726FFBDB9DA
:109850002946A06D0E22FEF733FD2A46A06D012198
:10986000FEF7A2FCA06D01220E21FEF713FD2221BE
:10987000204603B0BDE83040FEF7A4BF043BD0E76C
:10988000A368204619680231FFF76CFBA06D0E2219
:109890000221FEF715FDA06D00220121FEF784FCD8
:1098A000A06D01220E21FEF7F5FC20460DF1070107
:1098B0000122FFF727FA002320460DF107020121BC
:1098C000FFF7EEF9204602220021FEF7A2FE012258
:1098D00020460221FFF702FE20463021FEF772FFEC
:1098E000A06D4FF42051FEF744FBA368A06D1A68E9
:1098F00001210132FEF7E6FD01212046FEF7CDFEF3
:109900002046FFF77FF803B030BD00BFC37D0508D8
:1099100038B504460D4604220021FFF7DFFD20463E
:109920000421FEF721FE1F21FEF74CFFA06D4FF42E
:109930002051FEF71EFB2A46A06D0021FEF7C2FD56
:1099400000222046BDE838401146FEF762BE37B51A
:1099500004460D460021FEF71FFE20464FF0FF3162
:10996000FEF702FEA36819680231FFF7FBFA2046F2
:1099700000225421FEF773FE204600225421FEF7F8
:109980006EFE204600225421FEF769FE2046052285
:109990000221FFF7A3FD0322204600231C21FEF72E
:1099A00029FFA36820461968FFF7E9F82946A06D4A
:1099B000FEF7C0FA20460121FEF7EEFD2046022107
:1099C000FEF76BFE0122A06D0021FEF779FCA06D71
:1099D0004FF42051FEF7CDFAA368A06D1A6800215C
:1099E0000232FEF76FFD02250023A06D1A46012109
:1099F0000095FEF7A9FC204601220021FEF709FE92
:109A0000002220461146FEF704FE20460022542183
:109A1000FEF725FE294620460522FFF75FFD0023BD
:109A2000032220461C21FEF7E5FE20461021FEF70A
:109A3000C9FEA06D4FF42051FEF79BFAA368A06DFC
:109A40001A6800210132FEF73DFDA368204619681F
:109A5000FFF788FA0022A06D1146FEF7A5FB002251
:109A6000A06D0121FEF716FCA3682046196801319C
:109A7000FFF778FA0121204603B0BDE83040FEF739
:109A800073BD0000436D73B5DD8A044615F0010611
:109A900013D001220021FFF721FD002202212046E0
:109AA000FEF74FFE0022A06D1146FEF77DFB00225F
:109AB0000C21A06DFEF7EEFB1BE0027D002A47D0D3
:109AC0003146FEF734FE5428C5F3871525D12046CC
:109AD000FEF757FDADB92A462946A06DFEF7EFFF08
:109AE000636D9A8C002AE2D1DB8A03F01103002B0C
:109AF000DDD12046226BE16802B0BDE87040FFF77F
:109B000063B832463146A06DFEF74EFB01232A466C
:109B100004212046FEF743FEE2E70DF1070132463D
:109B20002046FFF7EFF89DF80710A9420DD0284610
:109B3000FEF710FD02460846FEF70CFD07490346F6
:109B40000748666807F0DAF93060002DC8D0DDE715
:109B50000DF10701FFF7D6F8C2E700BFCB7D05087E
:109B6000C88F0508F8B51646044600250F46FEF7CF
:109B7000FEFD31462046FEF73BFD2A46E36CB5422A
:109B80000CD1B4F84A20394620461A44FFF78EFC1F
:109B900029462046BDE8F840FEF7E6BC616A581940
:109BA00021F830200135EAE773B5164604460D4624
:109BB00000220DF10701FFF7A5F8721C20462A4488
:109BC0000221FFF7CFFF01232821204645EA062284
:109BD000FEF7E5FD02B070BD37B504460D46002224
:109BE0000DF10701FFF78EF82A4620460221FFF704
:109BF000B9FF01232A4627212046FEF7D0FD03B0F6
:109C000030BD37B50D4600220DF107010446FFF7C0
:109C100079F855B1012120460422FFF7A3FF1E2148
:109C20002046FEF7CFFD03B030BD2A46A06D0121CE
:109C3000FEF7BAFA20461E21FEF7C4FD2A46294641
:109C40002046FEF7E6FCEEE737B504460D468AB13E
:109C500003220121FFF742FC204602220121FFF7E7
:109C600081FF00232A460B21204603B0BDE8304087
:109C7000FEF7E9BE0DF10701FFF744F80222204686
:109C80001146FFF76FFF01232A460A212046FEF7FF
:109C9000DAFE03B030BD7FB5012504460DF10F0398
:109CA0000DF10E0100220095FFF73AF89DF80F60C4
:109CB00020469DF80E100022FEF7ABFC2A463146E6
:109CC0002046FEF7A6FC04B070BD00002DE9F3416C
:109CD0000446138B0161D81E434243412375002380
:109CE0000E46E364118CA36915468B42626505D26A
:109CF000E069F6F740FA2B8CE061A361626D518B4D
:109D0000938BEA8A0B44510748BF013392074FF007
:109D10000002114648BF0133934249D1227D002AF7
:109D20005AD1A2699A4259D800236021226A9A42E4
:109D30005DD1042E0CBF02210121A06DFEF7D2F8E7
:109D40000023626DA4F84830938CD28A13B902F0D4
:109D5000110139B10D21D707A4F848104CD50F23B4
:109D6000A4F8483087492068FDF795FB277D804699
:109D70002B8C698C002F00F00981606D1944828C56
:109D80006164002A3CD1C08AC60707D4032BA8BF50
:109D900003231A466B8B032B00D9013A10F0110FE5
:109DA0002FD1E88AB4F84830800648BF01332BE051
:109DB000E06981540132AFE7C86A00EBC200417824
:109DC0000132CF0741BF4788E0690909C155616D7C
:109DD000088D9042F0DCA4E70022F8E7227D002AFB
:109DE00014BF60210021E269D154013399E7606A10
:109DF00020F8331001339AE7002BB3D00E23AFE7DE
:109E00000022B4F8483002330226A4F84A30B4F8ED
:109E10004A30A06D1944891AFEF7C4F801230022C4
:109E20000721A06D0096FEF78FFA07220323114643
:109E3000A06D0096FEF788FA072243461146A06DF2
:109E40000096FEF781FA636D9A8C1AB9DB8A03F0EB
:109E500030032BB10022B4F84810A06DFEF71AFAB7
:109E600001220021A06DFEF7EFF802220121A06D72
:109E7000FEF7EAF803220621A06DFEF7E5F84FF49D
:109E80002451A06DFEF775F8A36801211A68A06D32
:109E90000432FEF717FB6A8B0221A06DFEF784F9EE
:109EA000022300224FF48541A06DFEF7C8F8A36895
:109EB00000211A68A06D0532FEF704FBA368A06DAF
:109EC000196802260431FEF735F86B8B02215A001F
:109ED00042EA4342A06DFEF767F903222C21A06DF0
:109EE000FEF725FBA368A06D196800250531FEF774
:109EF00021F8254F636D5A8BAA4215DC032A0DD930
:109F00009A8C5AB9DB8ADB0708D4B4F84A20636C10
:109F100006211A44A06D033AFEF7D2F9204602B09A
:109F2000BDE8F041FFF7B4B92B4606220021A06D31
:109F30000096FEF709FAE3695A5D22B10123032175
:109F40002046FEF72CFC022D11DC636D9A8C72B951
:109F5000DA8AD2070BD4022D02D15B8B032B06D1F8
:109F60000022795DA06DFEF76FF80135C2E7B4F805
:109F70004A10636C0022194401392046491BFEF740
:109F8000E0FBF2E744830508747F05080B44636433
:109F90000421E26BA06DFDF7DEFF636DDE8A16F033
:109FA000010643D0226C0421A06DFDF7D4FFB4F864
:109FB0004810A06DFDF7F6FF4FF4A0230226A3641E
:109FC0003A460621A06DFEF73FF801220E21A06D52
:109FD000FEF760F906223946B4F84830A06D0096C5
:109FE000FEF7B2F901233A463946A06D0096FEF716
:109FF000ABF903233A463946A06D0096FEF7A4F963
:10A0000043463A460721A06D0096FEF79DF920468B
:10A01000FFF73EF9636D9A8C002A46D0002319465B
:10A020002A8D9A4258D802B0BDE8F0810227B4F8D0
:10A030004820616C053292B2A06DA4F84A20114408
:10A04000FDF7B0FF3246A06D012307210097FEF710
:10A050007BF90722A06D114603230097FEF774F9E0
:10A06000072243461146A06D0097FEF76DF9324670
:10A07000B4F84810A06DFEF70DF93146626CA06D82
:10A08000FEF792F8B4F84810324620460331FEF746
:10A0900058FB3146B4F84820A06DFEF727F904229A
:10A0A0002D21A06DFEF743FAB1E7DE8A16F0010616
:10A0B000B4D10F4F2B8CB342B0DDB4F84A20636C9F
:10A0C00017F8011B1A44013A921BA06D0136FEF7E6
:10A0D000F7F8032EEED1A1E7EA6A02EBC30012F80B
:10A0E00033200133052A02BF4288E069815497E793
:10A0F000747F050870B5164604460D461A464BB9DE
:10A100005421FEF7ACFA324629462046BDE870409D
:10A11000FEF7E4BE70BDF8B504460F4616460121B1
:10A120001D46FEF7BAFA2046FFF7B5FD002254217E
:10A130002046FEF794FA2046FFF7ADFD394620464B
:10A14000FEF71DFD20464FF0FF31FEF7A6FA31461F
:10A150002046FEF707FF2046FEF713FAA06D012206
:10A160000021FEF7ADF8002220461146FEF751FA15
:10A17000A06D4FF42051FDF7FCFE2A46A06D002192
:10A18000BDE8F840FEF79EB92DE9F74301EB420721
:10A190000D463946044616469846FEF7C8FA70281A
:10A1A0008DF8060033D1E26C636A002103EBC20331
:10A1B000204613F80C6CFEF7BAFA072805460DD8AE
:10A1C00088B12046FEF71EFCE36C626A03F100537F
:10A1D000013B02F8336003B0BDE8F0835428F0D0AF
:10A1E0001F4803F04BFE02460DF107012046FEF723
:10A1F00089FD2046FEF7C5F9324603210123FEF70B
:10A20000CEFA2A4631462046FEF703FAE3E745EA4E
:10A210000629B8F1000F0DD002212046BA1CFFF725
:10A220005DF94B4600221D212046FEF7E3FA00228D
:10A230001146E8E756EA050304D03A4602212046D3
:10A24000FFF74CF920460DF106010022FEF75AFDFA
:10A2500001234A461B212046FEF7A1FAE7E700BF8B
:10A26000D57D05082DE9F041C66CD0F824C0013E2B
:10A270000CEBC60715467A780446012ADDF81880EB
:10A2800013D1D7F804E09E450FD0C6450DD01CF879
:10A2900036300B7079682960FEF7C4FA2046BDE8B5
:10A2A000F0414FF0FF31FEF75FB90A462046012129
:10A2B0002B68FEF7F5FCF1E77FB5002303934FF021
:10A2C000FF330446009303AA0DF10B01FFF7CAFF09
:10A2D0009DF80B50039E294632462046FEF799F919
:10A2E000324629462046FEF794F904B070BD73B596
:10A2F00004460E461546002A56D1134601210DF19B
:10A300000702FEF7CDFC022220461146FFF72AFC89
:10A31000012320460D220A21FEF795FB20460DF170
:10A3200007010222FEF7EEFC20460DF10701012293
:10A33000FEF7E8FC2A4620460DF10701FEF7E2FC95
:10A3400020469DF807100122FEF763F920469DF88C
:10A3500007100222FEF75DF9022220461146FFF7A0
:10A3600001FC012320460C220A21FEF76CFB02228D
:10A3700020461146FFF7B2F82B462A4620461C21FC
:10A38000FEF738FA2A4629462046FEF742F92046CB
:10A39000FEF7D4FB012231462046FEF79DF9204608
:10A3A000FFF78AFF02B070BDFEF7C8FB31462046BA
:10A3B000AB1E5A425A4102B0BDE87040FEF78CB95C
:10A3C0007FB50E4600210446FEF7B1F9831E012B2E
:10A3D00005468DF80B0033D8BEB1012E17D10023EE
:10A3E00003AA00930DF10B0120460393FFF73AFFF8
:10A3F000039B44F240211A46A06DFDF720FE039A0C
:10A400009DF80B102046FEF704F904B070BD022E33
:10A410000DD1002303AA00930DF10B0120460393F5
:10A42000FFF720FF039B44F2C0311A46E4E70F4BCD
:10A4300064689A5D0E490F4806F060FD2060E4E70D
:10A4400070B9012220460DF10B01FEF75BFC32468C
:10A4500011212B462046FEF7A2F92A462946D1E7CC
:10A46000FEF778F8044902466468E4E732A3050879
:10A47000DD7D0508C88F0508E67D050870B5044632
:10A480000D46164686B023B906B0BDE87040FEF70B
:10A4900025BD00221146FEF7C5F920460022012104
:10A4A000FEF7C0F9324629462046FEF707FA002398
:10A4B00004934FF0FF3301252046009304AA0DF1C9
:10A4C0000F01FFF7CFFE049B2046009305AA0DF174
:10A4D0000F010595FFF7C6FEDDE904210223A06DFB
:10A4E00000932B46FDF774FF06B070BD7FB50446A0
:10A4F0000D46164623B904B0BDE87040FEF7DEB93C
:10A5000000221146FEF78EF9324629462046FEF714
:10A51000D5F94FF0FF3300252046009303AA0DF133
:10A520000B010395FFF79EFE02232946039AA06DB7
:10A5300000930123FDF708FF2A4629462046FEF72F
:10A5400068F804B070BD0000F0B50D4685B001217B
:10A550000446FEF7ECF806468DF80A000021204676
:10A56000FEF7E5F8B31E012B8DF80B0000F2CE804C
:10A57000861E012E00F2F480A5F109030C2B9CBF6E
:10A580000D35EDB21F2D01D0212D23D10023012245
:10A59000009320460DF10A030DF10B01FEF7C0FBFD
:10A5A0009DF80A30022B07D0784B79495A5D7948DB
:10A5B000666806F0A3FC30601F2D0CBF2E212F21F2
:10A5C0002046FEF7FFF8002202212046FEF721F880
:10A5D00005B0F0BD012602232046039303AA002301
:10A5E0000DF10B010096FFF73DFE324620460DF1BE
:10A5F0000A01FEF787FBA5F11903B34217D8192DFD
:10A60000A06D039B08D132464FF48141FDF717FD41
:10A6100001229DF80A10D8E79DF80A20032A08BFF6
:10A6200044F2C001324618BF4FF48241EEE7162DC6
:10A6300005D132464FF48641039BA06DE6E7172D06
:10A6400004D1324644F24001039BF6E7182D04D1B1
:10A6500032464FF48041039BEFE71B2D08D141F6B2
:10A6600009030399A06D43EA8111FDF782FCCFE74E
:10A670001C2D03D141F609230399F3E71D2D04D1C5
:10A68000324644F24031039BD7E7052D31D89DF87F
:10A690000A209DF80B309A4205D03F493D48666834
:10A6A00006F02CFC306000229DF80A301146032B86
:10A6B0000CBF002606262046FEF7B4F801224FF410
:10A6C0008541039BA06DFDF7BAFC344B354433F84C
:10A6D0001510A06DFDF74DFC42F20101A06DFDF7D4
:10A6E00048FC4FF40051A06DFDF743FC002201210E
:10A6F0006BE720460121FDF737FF244B28495A5DBF
:10A700002448646806F0FAFB206061E7064327D11D
:10A7100001270222204600970DF10A030DF10B01DB
:10A72000FEF7FEFA322D17D0332D17D1072500235F
:10A730002A4612212046FEF732F857B100220121A5
:10A74000A06DFDF781FC0023032211212046FEF7B6
:10A7500026F80022114638E70625E8E73746E6E7FF
:10A7600020464FF0FF31FDF7FFFE9DF80A00FDF790
:10A77000F1FE02469DF80B00FDF7ECFE0949034689
:10A780000448646806F0BAFBBEE700BF32A30508C0
:10A79000F67D0508C88F0508067E05085C7F05085C
:10A7A000197E0508277E05082DE9F0430446C16897
:10A7B00085B0FEF7D7FB636D9A8CD98A12B901F088
:10A7C000110373B311F0010117D1B4F848202046EA
:10A7D0000132FEF75FF8636D9D8C55B94FF420513F
:10A7E000A06DFDF7C6FBE2682946A06D0132FDF7BA
:10A7F00069FE05212046FDF7E5FF21212046FDF7F2
:10A80000E1FF636DDA8AD20706D49B8C23B9E16835
:10A8100020460131FEF7A6FB0C220021A06DFDF7BA
:10A820004FFDA06DFDF7ECFB237D002B5FD1A36DE9
:10A83000656C5B68013DA3632368EA005B8802F0F6
:10A840007802E363636D2D095E8BDF8AB3F81C9099
:10A85000B3F81E8006F0030307F00F071A43B6088B
:10A8600045EA0703334343EA090353EA0803A06DAB
:10A870006AD10121FDF76FFBB4F85060B4F8527053
:10A88000720007F0010302F07E027F08B60957EA62
:10A89000060542EA030218BF42F080020121A06DC2
:10A8A000FDF759FB002DEBD1636DA76D998A2068E8
:10A8B0007E68FCF7D9FD4C490246384610F098FDF9
:10A8C000494F626D538B918B108D0B44AB4279DCF9
:10A8D0000025A36D9F88BE1BA4F85060D4E91530F5
:10A8E0001A8DAA4270DC4368DB1BA4F8523023693E
:10A8F000042B25D1A36DD3E9027623685868237D04
:10A900005BB9A56BE16B354400296AD00131890040
:10A91000F5F731FCE36B40F823500021626D237D95
:10A920001569CDE90211002BD38A18BF0421CDE9A6
:10A93000000332463B4608BF0321284601F020FEB3
:10A94000012005B0BDE8F08342F080020121FDF74F
:10A9500002FBBA012B0103F0300302F040021A435C
:10A9600008F001031A434FEAC90303F008031A432E
:10A97000B30003F004031A43AD087F0876084FEADA
:10A9800059094FEA58086BE7D36A03EBC10393F800
:10A9900001C01CF0010F10D0B3F802C0AC450CD1BF
:10A9A00059682068D4F85880FCF75EFD39460246A5
:10A9B000404610F01DFD013583E701318142E3DBA4
:10A9C0000521EEE70021F9E7DB6A03EBC50213F886
:10A9D0003530052B03D101215288FDF7BCFA013532
:10A9E0007CE7284699E700BF157F01082DE9F04173
:10A9F00088B004460D4607AE002940F0C68001210C
:10AA0000FDF795FE07468DF8170088BB01462046E6
:10AA1000FDF78DFE8DF81C00C0B90122314620469D
:10AA2000FEF770F9002220460DF11701FEF76AF9D2
:10AA300004220F2102232046FDF7B1FE0022114619
:10AA40002046FDF7E6FD08B0BDE8F0813A46314604
:10AA50002046FEF757F920469DF81C2001230421CB
:10AA6000FDF79DFE3A460121A06DFDF7EDFAD9E70D
:10AA7000E36C626A013B02EBC30132F8332040F21F
:10AA800002239A422BD14FF0010820464F68FDF770
:10AA900078FD434632460DF11701CDF80080079549
:10AAA000FFF7E0FB20462A462946FDF7BBFE9DF84E
:10AAB000170006280DD007280ED005285BD1009579
:10AAC0003B462946079AA06DFDF73EFC0022022175
:10AAD000B6E7CDF80080F3E702230093F0E7012307
:10AAE00032462046079306A92B460095FFF7BAFB8E
:10AAF0002A4620460DF11701FEF704F920462A46A2
:10AB00002946FDF78FFE9DF81800831E012B08D9FA
:10AB1000FDF720FD984902469848656806F0EEF971
:10AB200028609DF8170006280BD0072816D00528A6
:10AB300021D10799890141F4B841A06DFDF719FAB7
:10AB4000C4E70799A06D41EAC10141F04001FDF75A
:10AB500010FA0799890141F4B441EEE70799A06D15
:10AB600041EAC10141F08001FDF703FA079989012B
:10AB700041F4B041E1E7FDF7EDFC814902467F4831
:10AB8000656806F0BBF92860A0E7012940F0E58080
:10AB9000FDF7CDFD07468DF8150048BB0146204660
:10ABA000FDF7C5FD022105468DF818002046FDF78A
:10ABB000BEFD55EA00038DF81C0008D0394620463A
:10ABC0000322FEF78BFC03212046FDF7CDFC022378
:10ABD000CDE9016300232046009306A901220DF16F
:10ABE0001503FEF7D0F80F212046FDF7EBFD2AE70D
:10ABF000E36C626A013B02EBC30132F8332040F29E
:10AC000002239A4239D120464F68FDF7BAFC02234D
:10AC100000220093CDE906230DF115012B4606AA6B
:10AC2000FFF720FB2046069B324600950DF11701E9
:10AC3000FFF718FB9DF81700431E022B08D9FDF7FC
:10AC400089FC504902464D48656806F057F928606E
:10AC50009DF8150006280CD007280CD0052872D1C5
:10AC60000023DDE906210093A06D3B46FDF7B0FB14
:10AC7000E9E60123F5E70223F3E7022320460793E1
:10AC8000009306AA00230DF116010695FFF7EAFAD4
:10AC9000204600220DF11501FEF734F89DF816004C
:10ACA000831E012B08D9FDF755FC3749024633486E
:10ACB000656806F023F92860069B2046009332461B
:10ACC00000230DF11701FFF7CDFA9DF81700431E81
:10ACD000022B08D9FDF73EFC2A4902462748656841
:10ACE00006F00CF928609DF8150006280DD00728FD
:10ACF0001AD0052827D1DDE9063141EA831141F454
:10AD0000A841A06DFDF735F99DE60699A06D41EAD1
:10AD1000C10141F04001FDF72CF9DDE9063141EABE
:10AD2000831141F4A441ECE70699A06D41EAC10109
:10AD300041F08001FDF71DF9DDE9063141EA83119B
:10AD400041F4A041DDE7FDF705FC104902460B4840
:10AD5000646806F0D3F8206075E60025334606A93E
:10AD600001220095FDF7DCFF02232A460F21204631
:10AD7000FDF715FD67E600BF4A7E0508C88F050888
:10AD8000417E0508547E0508677E05085D7E05083E
:10AD90002DE9F04180465C2016460F461D46F5F72A
:10ADA000E8F9866008260446C0E90087066240206C
:10ADB000F5F7C6F9E66260622020F5F7C1F9606335
:10ADC0002020F5F7D6F92946A065FDF778F820464A
:10ADD000BDE8F08110B504460021806DFDF777F8DD
:10ADE000A06DF5F7D5F9606BF5F7D2F9E069F5F7E5
:10ADF000CFF9606AF5F7CCF92046BDE81040F5F7C9
:10AE0000C7B9000070B50646B2B1900714D11079E9
:10AE10002E2811D194687CB1A2070DD16568EAB2E1
:10AE2000922A09D12D0A022D06D10120A2681A60AA
:10AE3000E268049B1A6070BD0A460448044906F0A3
:10AE40005DF8736A18600020F5E700BF148F0508ED
:10AE5000777F0508F0B585B005460E46104603A974
:10AE60001F46F8F7B9FD48B932460B490B4806F0C2
:10AE700045F86B6A1860002005B0F0BD039803F038
:10AE8000E1FE30EA0703F7D0034632460449009753
:10AE9000024806F033F8ECE78D7F0508148F0508AB
:10AEA000937F0508038C70B5032BC46A03D100237C
:10AEB000856A9D4205D144F82120FDF73BF8012029
:10AEC00070BD54F82360964201D00133F1E70020B1
:10AED000F6E7FDF795B838B58BB2032B04460D465F
:10AEE0000384426205D1826A0021C06A920026F082
:10AEF00064FD042D20460CBF02210121FCF7F2FF66
:10AF00002046BDE838400021FDF74CB802F00F03A1
:10AF1000022B10B5044608D00A460C490C4805F02F
:10AF2000EDFF636A1860002010BD836A00201209DB
:10AF3000984204D1238C042BF5D10649EEE7E16A4F
:10AF400051F820108A42EFD00130F1E7A97F0508BF
:10AF5000148F0508AF7F050800F00F03022B02D104
:10AF60000009F5F7D2BE0148704700BF85360608D4
:10AF700070B5054610460E46FFF7EEFF0378732BBB
:10AF800019D14378BBB103460A22002013F8014FC0
:10AF90005CB91F2808D91F2332460A490A4805F020
:10AFA000ADFF6B6A1860002070BD303C092C02D8E0
:10AFB00002FB0040EAE732460449034805F09EFFE1
:10AFC000EFE700BFBB7F0508148F0508C87F0508A1
:10AFD000F8B5054610460E461F46184CFFF7BCFF55
:10AFE0000022A446017863788B421BD190F801E0DF
:10AFF000A3789E4516D190F802E0E378734511D10D
:10B000006BB91CF82200B84208D93B4632460C49BD
:10B010000C4805F073FF6B6A18600020F8BDC37818
:10B02000002BEED00132152A04F10404DBD13246A4
:10B030000549044805F062FFEDE700BF04810508FB
:10B04000BB7F0508148F0508D17F05082DE9F3475C
:10B0500006460F46002A3CD093073AD113792F2B8E
:10B0600037D1926802F00F03022B08D10F23FFF7AC
:10B07000AFFF01248440204602B0BDE8F08742B310
:10B0800012F0030A25D113799F2B22D1D5682B7991
:10B09000A12B1ED10F239268FFF79AFF4FF00109F1
:10B0A000A22109FA00F401AA05F10800F8F7D4FE7C
:10B0B0008046C245DFDA019A0F2352F82A2039462A
:10B0C0003046FFF785FF09FA00F004430AF1010A50
:10B0D000EFE73A460349044805F010FF736A00247D
:10B0E0001860C8E7D77F0508148F050810B5044617
:10B0F000024805F08BFE206010BD00BF148F0508CC
:10B1000004292DE9F84380460C460DD83026151F3A
:10B1100001F13009B1450DD055F8040F00F00F03CF
:10B12000022B0AD00D4900E00D49D8F82400FFF7A2
:10B13000DDFF00242046BDE8F8830009F5F7E5FDB2
:10B14000074626F06EFC0228ECD13B78722BE9D141
:10B150007B78B342E6D10136DCE700BF0D800508FD
:10B16000E87F05082DE9F0470F4686B0044603A99D
:10B1700038461E469146F5F7D4FD03780546762BF2
:10B1800040F02A81B9F1020F40F0D58040F25E43D1
:10B190009F4232D14EF6B4684FF42C6906E04EF669
:10B1A000B168F9E74EF6B1684FF424692946326870
:10B1B0002046FFF7DDFE2946074672682046FFF766
:10B1C000D7FEFB02420102F0200203F47043134356
:10B1D000B90143EA0903C0F3430001F0400143EA27
:10B1E000000241EA08012046FCF7CDFE2CE24EF6B3
:10B1F000B868D1E74EF6BD68CEE740F26C439F4297
:10B20000CDD040F26A439F42CCD040F25F439F4290
:10B21000EDD0B7F58C6FEDD040F269439F421ED15F
:10B220003068FFF799FEAD4926F002FCA8B10F2364
:10B23000294620463268FFF7CBFE07467068FFF7C5
:10B240008BFEA74926F0F4FB002840F0BC803A03AF
:10B250004EF6F16142F42162C5E70F27EEE7B7F53C
:10B260008D6F2ED13068FFF777FE0378722B18D1DF
:10B270000F23294632682046FFF7AAFE294680465A
:10B2800072682046FFF774FE4EF610610746FA0119
:10B29000D2B242EA0832C7F3430742F4216239438B
:10B2A000A1E7294632682046FFF762FE2946074695
:10B2B0000F2320467268FFF78BFE4FF46E418046E5
:10B2C000E5E740F266439F422ED14EF6905829465C
:10B2D00032682046FFF74CFE05AB0093074629462F
:10B2E0002046726804ABFFF78DFD002800F0AC81AA
:10B2F00007232946049A2046FFF76AFE2946064698
:10B30000059A4FF47F732046FFF7A4FDFA02B901B6
:10B3100002F4704201F0400142EA900241EA080161
:10B3200042F4206231435EE740F26D439F424AD1CE
:10B330004EF68058CBE7B9F1030F44D10027DFF870
:10B34000A48100F1010A03224146504626F086FB03
:10B35000A0BB2B7993BB644B29463268204613F877
:10B360002780FFF705FE2946074672682046FFF74B
:10B37000FFFD29468146B2682046FFF7F9FDFA0233
:10B38000430102F4704203F0200313434FEAC91251
:10B39000D2B243EA50031343BF014FEA0812D2B2BC
:10B3A00007F0400708F0F00142F4206247EA59092B
:10B3B00041F46E411A4349EA010114E70137042FB1
:10B3C00008F10408BFD14B462A464849484805F0D1
:10B3D00095FD636A186037E1B9F1000F0FD1B7F539
:10B3E0006B7F05D14FF43F412046FCF7C2FD2BE1B6
:10B3F00040F271439F42E6D14BF63071F4E7B9F168
:10B40000010F40F00281B7F5197F10D10146326873
:10B410002046FFF77BFD01462046FCF739FE002859
:10B4200040F012813349606AFFF760FE0CE140F2A0
:10B430007522974209D1014632682046FFF766FD22
:10B4400001462046FCF77CFEE9E7B7F51F7F09D1EE
:10B4500001460F2320463268FFF7BAFDC10041F4D0
:10B460008E41C1E7622B49D1039B032B0CD0052BE6
:10B4700040F08E80C3785F2B40F08A8003796E2B7A
:10B4800002D0772B40F0848000224FF0FF3769789C
:10B49000194B5878884205D195F802C098788445B0
:10B4A00008BF1F7801320E2A03F10303F1D17B1C80
:10B4B00089D0326829462046FFF728FD039B0246C3
:10B4C000052B09D12B79A3F177056B426B413946E6
:10B4D0002046FCF7FBFDA2E70023F8E72B800508D8
:10B4E00035800508F5800508F480050848800508C2
:10B4F000148F05085580050860800508692B47D121
:10B500004378742B44D13068FFF726FDB74B0022F7
:10B510001F4601785E788E4227D190F801C09E7850
:10B52000B44522D1867806BBAE1C31460B4618784E
:10B5300001310028FAD1691D8B423FF644AF02EB7E
:10B540004202BA5C082112F0010F0CBF4FF0080C48
:10B550004FF0000CD00000F00800013BB3420AD2CB
:10B5600041EA021141F43F413EE701320E2A03F164
:10B570000303CFD127E713F801794908742F01D1CC
:10B580000143EBE7652F7FF41EAF4CEA0101E5E7CD
:10B5900040F2B5239F4202D14BF2726124E740F2A0
:10B5A000B6239F4202D14BF262611DE740F2D633CF
:10B5B0009F4213D1326829462046FFF747FD10F419
:10B5C0003F4F024607D150044ABFD1B242F4344142
:10B5D00041F4354108E74EF62D1104E6782F7FF44B
:10B5E000F2AE326829462046FFF730FD10F4FE4FD8
:10B5F000024607D101044ABFC1B240F43C4141F4C4
:10B600003D41F1E64EF6BD01EDE5B9F1020F40F026
:10B61000AC81736803F00F03022B40F09D80B7F5F7
:10B62000677F14D101460F2332682046FFF7D0FC14
:10B630002946074672680F232046FFF7C9FC3946A2
:10B6400002462046FCF700FD06B0BDE8F087B7F5DE
:10B65000297F1CD14FF6B0294FF280070F232946CE
:10B6600032682046FFF7B4FC2946804672680F23F3
:10B670002046FFF7ADFC47EA000242EA082249EA09
:10B680000001B0E54FF690294FF2A007E6E740F23F
:10B69000E3339F42F6D040F2A1339F422BD10146C3
:10B6A00032680C232046FFF793FC07467068FFF7CB
:10B6B00053FC064601464E4826F0BAF998B1314689
:10B6C0004C4826F0B5F9A0B12A464B494B4805F045
:10B6D00015FC0022636A186042EA07224FF2EF313C
:10B6E00042F400427FE50023454A03EBC303D25CEA
:10B6F000F2E70123F8E7B7F5167F15D14FF480473D
:10B700002946326807232046FFF762FC2946804617
:10B71000726807232046FFF75BFC42460346394622
:10B720002046FCF78CFC8FE70027DFF8D880032247
:10B730004146284626F092F940B9EB7833B9324BAE
:10B7400013F827703F0147F48047D9E701370F2FDF
:10B7500008F10408EBD136E6B7F5677F1CD14FF44A
:10B7600000570723294632682046FFF731FC294657
:10B770008046FF2320467268FFF76CFB47EA000112
:10B7800041EA082130E64FF42057EAE74FF44057EA
:10B79000E7E74FF46057E4E740F2A6239F42F2D078
:10B7A00040F251239F42F1D040F233439F42F0D008
:10B7B00040F29E339F4229D14FF240280F23294661
:10B7C00032682046FFF704FC4FF6FF730746294610
:10B7D00072682046FFF73EFB3A4603464146204644
:10B7E000FCF744FC30E74FF2C028E7E7608005082B
:10B7F00059810508628105083B800508148F0508FA
:10B8000058810508A1800508A080050840F29D33F5
:10B810009F42E8D040F29F339F421AD101460F2346
:10B8200032682046FFF7D4FB294607464FF0FF3326
:10B8300072682046FFF70EFB054683B23A464FF288
:10B8400040212046FCF712FC3A464FF2C0212B0C57
:10B85000C5E740F26E339F4228D101460F2332687C
:10B860002046FFF7B5FB05AB009307462946204667
:10B87000726804ABFFF7C6FA00283FF4E5AE0F2369
:10B880002946049A2046FFF7A3FB29460646059A57
:10B89000FF232046FFF7DEFA820842EA073246F429
:10B8A000684142F4706241F050019CE4B7F55B7F5F
:10B8B00040D040F26D339F423ED040F26F339F4202
:10B8C0003CD0972F3CD040F22F439F423AD040F2D9
:10B8D00031439F427FF477AD0523864A294632F8EB
:10B8E0002370204607233268FFF772FB05AB0093F5
:10B8F000804629462046726804ABFFF783FA002889
:10B900003FF461AD049A072329462046FFF760FB08
:10B91000FA04064618D51F2329462046059AFFF744
:10B9200099FA47EA0801800141EAC60100F4F8608B
:10B93000014359E50023D0E70123CEE70223CCE7FA
:10B940000323CAE70423C8E73B04059A06D53E2330
:10B9500029462046FFF77EFA4008E2E77C23294685
:10B960002046FFF777FA8008DBE7B9F1030F7FF491
:10B970002AAD40F27D339F4221D10027072329467B
:10B9800032682046FFF724FB072381462946726868
:10B990002046FFF71DFB294680461F232046B2683C
:10B9A000FFF758FA47EA090747EA801747EAC8014C
:10B9B0001AE54FF40067E1E74FF48057DEE740F205
:10B9C0007E339F42F5D0B7F5187FF5D040F2512372
:10B9D0009F422BD14FF4C058072329463268204696
:10B9E000FFF7F6FA07237268074629462046FFF755
:10B9F000EFFAB268814602F00F03022B0ED1072343
:10BA000029462046FFF7E4FA47EAC90141EA08015E
:10BA100041EA8011E8E44FF4D058DDE707232946D6
:10BA2000204648F48068FFF715FAEDE740F20A4334
:10BA30009F4222D14FF690380F2329463268204684
:10BA4000FFF7C6FA0F238146294672682046FFF7A2
:10BA5000BFFA29460746B2680F232046FFF7B8FA17
:10BA600040EA092242F4704242F0F00248EA07013B
:10BA7000FFF7B9BB4FF6B038DEE740F251439F42C3
:10BA8000F8D040F233439F42C5D0B7F5866F7FF4BC
:10BA90009AAC01460F2332682046FFF799FA0F232C
:10BAA0002946726807462046FFF792FA05AB0093D5
:10BAB000804629462046B26804ABFFF7A3F9002868
:10BAC0003FF4C2AD0F232946049A2046FFF780FABF
:10BAD00029460646059AFF232046FFF7BBF93F0299
:10BAE00047EA083746F4684147EA900241F04001CE
:10BAF000FFF779BBDC80050838B505463020F4F740
:10BB00001FFB04462022002125F057FF294620462E
:10BB1000FCF7D5F9A562A800F4F712FBE062204615
:10BB200038BD10B50446C06AF4F732FB2046002148
:10BB3000FCF7CDF92046BDE81040F4F729BB2DE90C
:10BB4000F84F8C46DDE90C84DDE90E1716460546F4
:10BB5000DDF828A058B1604509D3780759BF0A22FB
:10BB6000B5FBF2F50AF1010A013458BF013117F0B3
:10BB7000020933D0002931D00BDB0B9A91422DDA28
:10BB80000C44A24503DC0AF1FF38A4EB08080021AD
:10BB900024E00A1D22DB00224FF00A0EC1F1000B47
:10BBA000B5FBFEFC0EFB1C545018002C6FD0101A75
:10BBB0001C463021002800F1FF3BAAEB020AD8BF47
:10BBC0004FF0000B2E2204F8021B20465A705A46F2
:10BBD00025F0F3FE04EB0B030021FF240AF1FF3CE8
:10BBE00062464FF00A0E002A57DA621C524562DBA9
:10BBF000FE2CD4BF0025012503EB0A00B8F1000F8D
:10BC000007D02E233022A4EB0C04A4EB0808A04597
:10BC100056D1B9F1000F0AD04DB10346184610F8BD
:10BC2000012C013B302AF9D02E2A08BF184607F014
:10BC300001030B4326D07B0724D40029B4BF2D2356
:10BC40002B23044607F02007B8BF494247F04507B9
:10BC5000632904F8027B437005DD6423B1FBF3F331
:10BC60003033C41C83700A23B1FBF3F5B5FBF3F248
:10BC7000204603FB125203FB15133032303300F819
:10BC8000022B637000230370801BBDE8F88F013224
:10BC90005A45654684D1204689E7B5FBFEFB9442B0
:10BCA000A8BF10460EFB1B55B8BF501C30351D54A5
:10BCB000013A5D4697E72E22013301251A559BE78D
:10BCC00014B9012500F8013B00F8012B013C9EE767
:10BCD0002DE9F04F002899B0064617469946229C58
:10BCE0009DF88C800E912BDA014636F0A1FA38BB14
:10BCF0004FF02D0806F100460E9D013F05F8018B1F
:10BD000026F0004A5046664909F0200836F090FABD
:10BD1000D8B95046624936F06DFAB0B988F0490397
:10BD20002B7088F04E0388F046086B70E81C85F88D
:10BD30000280002303700E9BC01A19B0BDE8F08F7B
:10BD4000B8F1000FD8D10E9DDAE73146304636F013
:10BD50006FFA48B148F04E0388F041082B7085F81F
:10BD60000180E81CAB70E4E749F02009B9F1660FE7
:10BD70006AD148F00403002C0693A7F103096BDA9B
:10BD80000624A1454B46A8BF23460B93331E0993B7
:10BD900070D0C3F3C7507F3836F030F8414936F0E1
:10BDA00081F836F05BFAB6F17E5F34BF4FF00008E1
:10BDB0004FF00108834608EB00014FF07E5000F081
:10BDC00055FA099B4FF07E5AB3F17E5F2CBF0123D9
:10BDD0004FF0FF330793314636F00CFA003818BFA6
:10BDE000012040453ED0069B5A070ED5BBF1000FFF
:10BDF0000BDD04EB0B030233BB4206DD069B013473
:10BE000083F0040343F002030693069B13F004033C
:10BE10000F933AD0BB1EA342D8BF4C46BBF1000FD4
:10BE20002FDA022C29DD1BF1020F26DACBF10003F9
:10BE3000A342A8BF2346A3F1020AA4EB0A04092CDB
:10BE400034DC002303213AE0B9F1670F0CBF48F05E
:10BE5000020348F001038EE7632C92D110230924DA
:10BE60000B9393E7079B50469B4408EB0B0100F0B4
:10BE7000FDF9B0E7DDF824B0B5E701344FF0000A72
:10BE8000DDE70BF101031C44F8E7069B9B0700D597
:10BE900004B90134092C07DC002307219A460EE07F
:10BEA000FFFF7F7F9B209A3E4FF0000A0F9AA4F17C
:10BEB0000903002A4FF0090414BF032107213F1B87
:10BEC000791A9942A8BF1946062C27466FEA0B0338
:10BED000A8BF06273B4413910D93139B2344DB1B00
:10BEE0001193099B002B00F0BC800F9B002B00F0EE
:10BEF000B480BBF1000F07F1FF3180F2A980BAF1E5
:10BF0000000F00F0B3802B4630212E2203F8021BD5
:10BF100018466A70524625F050FD03465344079375
:10BF2000FF230AEB070108930A2201230A929F428A
:10BF300000F39F80062F40F3A580012940F3A280E3
:10BF4000072F00F09B80022900F098804FF06408D2
:10BF50000239304600F08AF94FF07C5135F09AFEF4
:10BF600036F0A2F9069B08FB00F8CDE904B3089B64
:10BF70002A460393119B0A9902930B9B4046CDE9F5
:10BF80000073079BFFF7DBFD17AA01460C902846BC
:10BF900000F098F93146179835F07AFE0C9B02466E
:10BFA0000146002800F08D804FF00109062FC2BF26
:10BFB00007EB4701123909FA01F90D21CDF830805C
:10BFC000109012911299013912917AD0069B002A91
:10BFD000CDE904B3089BB8BFC8440393119BA8BF25
:10BFE000A8EB090802930B9B2A46CDE900730A9936
:10BFF000079B4046FFF7A3FD17AA01461490284669
:10C0000000F060F93146179835F042FE149B024665
:10C01000002856D01593109B20F0004023F00041DB
:10C02000149235F035FEDDE91423002807DB4FF0CC
:10C030000A0CB8FBFCF10CFB1181014302D1CDF8D5
:10C0400030801092B9F1010F1FD94FEA5909B9E7B1
:10C050000D99CDF820B0079566E70F9B0D990893D1
:10C06000F9E7099B0795194608935DE7CDF820A0ED
:10C07000F1E70A98013350430A9058E74FF00A0855
:10C08000013966E74FF0010863E70D9AA74202F114
:10C0900001020D9201DA01371FE70C9A904510D08A
:10C0A000069B2A46CDE904B3089B0A990393119B8A
:10C0B0000C9802930B9BCDE90073079BFFF73FFDA4
:10C0C0000346E81837E600BF012910B5146822D9E5
:10C0D0000378302B1FD14178831C41F0200178294F
:10C0E00006D134F0100114D110211160181A10BDBE
:10C0F0006F2904D134F008010BD10821F5E762293A
:10C1000004D134F0020104D10221EEE70CB901237D
:10C1100013600346EAE7002CFBD10A23F8E700008E
:10C12000044608B531B1054B4A6C03600968002329
:10C1300004F023FF2046F3F7E1FF00BF148F05084A
:10C140002DE9F0418AB004461F46019246182AB1F3
:10C15000023A222A02D9424801F0C2FCB4422546E2
:10C1600050D214F8010BF5F7C5FB80460028F5D135
:10C170002B782B2B40D125462846711B01AAFFF7AF
:10C18000A3FF054428460024019BB04201463CD34E
:10C19000B8F1000F00D06442640044F00104A942E9
:10C1A0000AD08846B045434654D2187808F10108B1
:10C1B000F5F7A0FB0028F5D1322104AA06A8F4F770
:10C1C000B9FE019A2749012A08BF002204A8F5F701
:10C1D00043FB01232946721B04A808F02BF906A88B
:10C1E00008F088FB0121039000221F4803AB04F0F4
:10C1F000C5FC3946FFF794FF2D2B04BF25464FF0B1
:10C200000108B9E74FF00008B6E710F801CBACF130
:10C210003002092A0AD9BCF15F0FB6D04CF02002D7
:10C22000A2F1610CBCF1190FB2D8573A9342AFD9C1
:10C2300084FB0341B1EBE47F03D1144494EA44024C
:10C24000A3D5711B424606A8069506F040F806994C
:10C250000446A4E7B0D120460AB0BDE8F08100BF93
:10C260006A8105087F810508A48F050838B5044652
:10C270000D46B9B1002135F0A9FF98B9C4F3C753F1
:10C280002B4415F10A0F63F3DE540DD3684235F0E9
:10C29000B5FD01460A4822F0B7FF0146204635F0B9
:10C2A000B5FE0446204638BD284635F0A7FD0146B8
:10C2B000034822F0A9FF214635F0F4FDF1E700BF65
:10C2C0000000A0402DE9F74F0192002204460144EE
:10C2D0009446134617461046934615464FF00A08F3
:10C2E000DFF8E8E08C4254D2264616F8019BA9F10B
:10C2F000300ABAF1090F34D8022D06D1344CA742C6
:10C3000001DC08FB07A73446ECE7BAF1000F01D0C7
:10C3100070450CD90DB90133F5E70CF1010C01257D
:10C32000F1E7704594BF08FB00F00132013B002BA0
:10C33000F7D1634653B9704510D808FB00A0012D12
:10C3400008BF02F1FF324FF0000CDCE770459CBFE4
:10C3500008FB00F002F1FF32013BEBE77DBB01324D
:10C36000F1E78DB9B9F12E0FD9D049F0200ABAF111
:10C37000650F0BD1B14203D965782B2D19D1A61CBD
:10C380008E4220D00225BEE7022DEED1B9F15F0F1B
:10C39000B9D0BBF1000F14D113441F4435F02AFD6E
:10C3A0003946FFF763FF019B1860204603B0BDE8E4
:10C3B000F08F2D2DE6D14FF0010BA61CE0E79C4637
:10C3C000ADE77F42E8E70024EFE700BF97999919AE
:10C3D000646666062DE9F04F002604461F464FF0BE
:10C3E000000B4FF0FF494FF07E5A85B0DFF86481B3
:10C3F0000092451803962246AA42144672D212F8B9
:10C40000010B0192F5F776FA019A03460028F3D161
:10C4100021782B2961D11446A21C954274D9227827
:10C4200042F02002692A5FD1627842F020026E2A2F
:10C430006AD1A27842F02002662A65D1E21D9542B7
:10C4400004F10300CDF80C901AD9E27842F02002F2
:10C45000692A15D1227942F020026E2A10D1627920
:10C4600042F02002692A0BD1A27942F02002742AFC
:10C4700006D1E27942F02002792A01D104F10800C4
:10C48000009A6AB1A8420BD2027842F020026A2ACE
:10C4900006D1844208BFCDF80CA001304BF0020B4E
:10C4A0001BB1039B03F100430393844235D0034641
:10C4B000AB421C4638D2013320780193F5F71AFAC3
:10C4C000019B0028F4D147B3BBF1000F25D1002315
:10C4D000039E4FF0010B03938DE72D2904BF1446F3
:10C4E000012399E7002397E76E2A0DD1627842F085
:10C4F0002002612A08D1A27842F020026E2A03D1DC
:10C50000E01CCDF80C80BBE7204603AA291B019351
:10C51000FFF7D8FE019B0028B2D10F490F4804F065
:10C5200075FC0E99FFF7FCFDCDD1BBF1010FF4D0E6
:10C530000398BBF1000F06D00146304603F056FCCD
:10C5400005B0BDE8F08F0FB10021F7E704F0F0FD72
:10C55000F6E700BF0000C07FA9810508A48F050889
:10C5600008B51020F3F705FE0123837008BD10B550
:10C57000022403F00103C0E901128470C37010BDEE
:10C580009DF80430426003F00103C370009B039ADE
:10C590008360029B81700373C36862F31F23C360CF
:10C5A0007047000070B5044623880E461046C3B19C
:10C5B0000A460023214605F06BF923460022E44396
:10C5C00013F8011B090603EB040603D4D30724D593
:10C5D0001B4B18E013F8011BC1F38015B5402A432B
:10C5E000F0E7A3786568042B0FD0052B16D0032B3A
:10C5F0000A46A36829461DD105F04AF9114B03608C
:10C60000E37853B1104B036007E010200F49A46892
:10C6100002F018FAC0E90164C56070BD10200C4931
:10C62000267BE46802F00EFAC4F31724C0E9016522
:10C63000C460F2E705F02CF9E378002BEDD0C7E7F2
:10C6400064920508449105088092050864910508E4
:10C650009090050838B514461D4612F4807218BF34
:10C660001A46FFF79FFF620902F008022A44E1B26E
:10C67000BDE8384003F054BB09C8184770B50546FB
:10C680000C468E18B44200D170BDD5E9000398471E
:10C6900004F8010BF6E738B504460025D4E9000399
:10C6A000984700F07F0343EAC5150306F6D42846F1
:10C6B00038BD00002DE9F04186B00546FFF7DCFFEC
:10C6C00010F0FF0453D0012C53D0022C53D0032C74
:10C6D00053D0042C53D02846FFF7DDFF064648B957
:10C6E000062C07D12846FFF7C7FF264C204606B088
:10C6F000BDE8F0810A2C10D10021304609F0FEFF80
:10C700000027044600F10808B742EFD02846FFF79B
:10C71000D1FF013748F8040BF6E7314602A8F4F7D9
:10C72000FAFB324628460499FFF7A8FF631F012B46
:10C730000CD82846FFF7A0FF052C02A803D108F06B
:10C74000D9F80446D2E708F0DBF8FAE7072C4FF0F7
:10C750000003DDE9031003D10A22FFF7F1FCF0E743
:10C76000093C624200936241FFF734FEE9E7064C60
:10C77000BCE70624BAE70E24B8E71E24B6E7034C4C
:10C78000B4E700BFA09E050844830508E89A0508A1
:10C790002DE9F84305460E4617460024DFF8A08031
:10C7A0002868FFF769FF5FFA80F9B9F1FF0F01D13F
:10C7B000BDE8F883C2070CD52868FFF76CFF10F0BE
:10C7C000010F4FEA500416BFA86806EB840400EB83
:10C7D0008404B9F10B0F4FEA590311D8DB070DD5CB
:10C7E0002868FFF758FF5FEA990927D0B9F1010FD0
:10C7F0000CBFAB68EB68024621461AE00120F2E765
:10C80000062B03D16B689B680120F4E7072B02D14C
:10C810006B68DB68F8E7082B1BBF03F18043093B1B
:10C82000434658F82330EFE751F804CB9C4441F8D5
:10C8300004CC013AF8D204EB8004B1E73B46DAE7D6
:10C84000448305082DE9F04F8FB080460991FFF72A
:10C8500022FF00F003039A1C05924FEAD00900F072
:10C86000040204924846002B3DD14FF0000AF3F732
:10C8700067FC554657465646014604464A464046DA
:10C88000FFF7FCFECDE907AA049B002B00F0978080
:10C890004046FFF700FF059B0490032B08BF0130C3
:10C8A0008000F3F74DFC4FF0000B0690049B9B4576
:10C8B0007BD1FFF755FE059B8346022B40F0898014
:10C8C00022460023E64312F8011B090602EB060587
:10C8D00078D421465846069A9BB2FFF748FE584640
:10C8E0000FB0BDE8F08FF3F72BFC4A460146044633
:10C8F0004046FFF7C3FE059B4046032B19D1FFF7C7
:10C90000CAFE2318591C06460027DB43225C10068A
:10C9100001EB030506D44FF0000A55460023CDE98C
:10C920000733B1E711F8012BC2F38010A840074389
:10C93000EDE7FFF7B0FE059B0746052B09D1404602
:10C94000FFF7A9FE05464046FFF7A5FE00268246F2
:10C95000E4E710F0200521D04046FFF79CFE824618
:10C9600017F0400002D04046FFF795FE1AEB000694
:10C9700016D0033020F003060AEB0600F3F7F9FBAC
:10C9800003463344089007932DB15246194640465A
:10C99000FFF774FE0025AA462E4675E7AA46DFE794
:10C9A000B2463546CDE907666EE740460999FFF77E
:10C9B00049FF069B43F82B000BF1010B76E7049B24
:10C9C000069376E712F8011BC1F38010A8400343D9
:10C9D0007BE7099BCDF828800B93079B0C93089B62
:10C9E0000D93FB0613D5DFF85880D8F8B81021B99D
:10C9F000084606F063F8C8F8B8002146D8F8B80031
:10CA000005F078FE224621460AA8FFF7C1FE059BE5
:10CA1000032B06D1049B264483B1069B049A43F85A
:10CA20002260069BBFB2009322464B465846CDE992
:10CA3000025A05990197FFF7A3FD50E70696F0E724
:10CA4000700300202DE9F047836886B004930368E3
:10CA500005460E4602A841490593F3F71BFB042245
:10CA600028460DEB0201FFF709FE9DF806909DF8A0
:10CA700004204FEA99034D2A03F02F030CD19DF8AF
:10CA80000520062A08D11BB109F00302032A03D1AD
:10CA90009DF807201F2A02D9314801F021F823B15F
:10CAA000043B022B01D92F48F7E719F04009F3D1D5
:10CAB0002846FFF7F0FD80462846FFF7ECFD4FEAD9
:10CAC00048040334074600EB94008000D6F800A029
:10CAD000F3F736FB24F00304CAF808002044CAF830
:10CAE0000C00C1450DD10024BC4231682CD1284630
:10CAF000FFF7A8FE70600120F3F7D4FA06B0BDE896
:10CB0000F0872846FFF7C7FD10F0010F4FEA5004E9
:10CB100013D12046F3F714FB8246224601462846ED
:10CB2000FFF7ACFD2846FFF7A7FD21465046F4F776
:10CB300025F804465046F3F72BFB33689B6823F82F
:10CB4000194009F10109CCE72846D1F80C80FFF71C
:10CB5000B1FD48F824000134C6E700BF7BCC0108D2
:10CB6000AF810508BB8105081FB50C46014601A829
:10CB700018F054FC214601A8FFF764FF04B010BD73
:10CB80008268024B1A61C268DA6070477003002045
:10CB90008388024603F4C071B1F5C07F0FD0190637
:10CBA00004D5C07B02EB80021069704713F48070DB
:10CBB00006D0D07B02EB80021369586870470148A9
:10CBC000704700BF5D80020870B5F3F77DFF002558
:10CBD0000123244CE561A4F8B631D4F8B8310BB187
:10CBE000A4F8B651204B214EC4E90E35204B032149
:10CBF00020486364A4F8C0512564C4F8B05184F897
:10CC0000B45103F04BFE0121304603F047FEAA2247
:10CC1000BA21304603F04CFF00210846C4E9036600
:10CC2000C4E92B55C4E95955A566C4F8B850C4F8F1
:10CC3000B45005F043FF0A21C4F81C0105F05AFD69
:10CC400040F2E261D4F81C0105F054FD002106F128
:10CC5000440005F08FFE40F21A7240F2DA63C4E934
:10CC6000482370BD70030020AC8D0508C803002068
:10CC7000C0A10508B80300207047D0E9023018476A
:10CC800008B5074B986E08B9064808BD002241F266
:10CC90004A11043001F0BCFC0028F5D04068F4E7EC
:10CCA0007003002044A60508034BC0000A4640F06C
:10CCB0000201D86803F0FCBE70030020034BC100E2
:10CCC00041F00201D86803F001BF00BF70030020EB
:10CCD000034BC0000A4640F00201186903F0E8BEA9
:10CCE00070030020034BC10041F00201186903F0FA
:10CCF000EDBE00BF70030020F8B51C469307074641
:10CD00000E46154608D113689A88910615D5520625
:10CD100010D5B3889B0501D52560F8BD50B9114BDE
:10CD20009E4207D00C20104901F08CFEC0E901653D
:10CD30002060F2E7C4E90057EFE70C4A934202D1C2
:10CD40006B682360E9E70A4A9342E5D130B101F00C
:10CD500085FE084B834214BF06463E466B68C4E915
:10CD60000036DAE7509605082C8305088CA30508E1
:10CD700074A30508C4A3050800232DE9F0410E465D
:10CD8000C2E900330746144601F068FE0A2E054644
:10CD900002D12060BDE8F081192E07D1838803F409
:10CDA000C0731BB1144BC4E90037F3E76B7B5BB175
:10CDB00005EB83031B692246314638469847636872
:10CDC000042BE7D100236360EB7C002BE2D005EB62
:10CDD00083031869F100002241F00201043001F0E0
:10CDE00017FC0028D6D02346294642683846BDE8BD
:10CDF000F041FFF781BF00BF14A70508F0B58DB063
:10CE0000054668460E4617461C46F3F765F940B9D5
:10CE10003A4631462846FFF7AFFFF3F733F90DB036
:10CE2000F0BD002CFBD1019B044918680AF052FCAC
:10CE30000028F4D10198F3F761F900BF6C8C050864
:10CE400008B519B903F0DDFFF3F758F903F0DEFF79
:10CE5000FAE70EB403B503AA52F8041B019203F0DB
:10CE6000F9FFF3F74BF9000070B5124EC400054608
:10CE7000306944F0020400222146043001F0C8FB6E
:10CE80000246A0B9B06E30B12146043001F0C0FBBB
:10CE900008B1406870BD00222146074801F0B8FB88
:10CEA000024620B92A4605490548FFF7D2FF5068D7
:10CEB000F0E700BF7003002088A70508C7810508B8
:10CEC000188E05080A4B10B50446D3E903039842AF
:10CED00007D0E100002241F00201043001F098FB8C
:10CEE00020B92046BDE81040FFF7BEBF406810BD26
:10CEF00070030020032837B505460C4607D10846C5
:10CF000001F0DCFF00B30E24204603B030BDCA0799
:10CF10002FD54B1008282AD801A252F820F000BFC4
:10CF200009CF010851CF01086FCF01086FCF010869
:10CF300045CF01086FCF010809CF01084DCF010887
:10CF400009CF0108002BDED01E24DDE7002BDBDA41
:10CF5000B3F1404F06D14FF0804003B0BDE8304000
:10CF600005F090B95C42640044F00104CCE7DC4376
:10CF7000F9E7062825D101F00703022B10D08B0713
:10CF80001FD10B681A7BE2B103EB82031A691F4BB6
:10CF90009A4216D1486840B98B68C86801930CE082
:10CFA000CC082046F3F79AFE18B1400040F0010487
:10CFB000AAE7204601A9F3F7B4FE0199F3F774FD3F
:10CFC000F3E7204601F04AFDC37ABBB100EB8300D2
:10CFD000036921462846984798B9042DB4D0A5F195
:10CFE0000803022B0FD90A4B20465D5D01F042FD7C
:10CFF0002A46034607490848FFF72BFF062DECD1C8
:10D00000B1E7044680E700247EE700BF255102080F
:10D01000E8A30508D38105085C8F05082DE9F041D8
:10D0200005460E461746984601F018FD847A54B11D
:10D0300000EB8404246943463A4631462846A44618
:10D04000BDE8F0416047284601F014FD0249024660
:10D050000248FFF7FEFE00BFDC8105085C8F050873
:10D0600000231A461946FFF7D9BF000070B50546E0
:10D070000C46114986B008690490C868C1E90332BA
:10D0800005900E4902A8F3F705F82246294668469E
:10D090002E68F6F7F5FEB4FA84F231465209684676
:10D0A000FAF776F9FFF7DCFF04460120F2F7FAFF02
:10D0B000204606B070BD00BF7003002081CB010880
:10D0C00007B50022019101AB0121FFF7A7FF03B0D3
:10D0D0005DF804FB30B455681446003D18BF0125C7
:10D0E000C5F1020302EB83030A462918206830BC0D
:10D0F000FFF794BF10B5044603F00EFF30B10023D4
:10D1000020461A461946FFF789FF0446204603F0D9
:10D110001DFF28B9BDE810400249034803F076BE60
:10D12000204610BDE28105085C8F05087FB5114BD4
:10D13000C00040F00200019018690592029006209C
:10D14000CDE90301986E78B1002241F282110430DA
:10D1500001F05EFA40B100220521406801ABFFF703
:10D160005DFF07B05DF804FB01A905200BF0BEFBD5
:10D17000F7E700BF700300202DE9F0410446174691
:10D180001E460D4659B1186801F068FC626882427B
:10D1900005D0C388D28806490648FFF75AFE3346B1
:10D1A0003A462946A068BDE8F041FFF737BF00BF07
:10D1B000038205085C8F050873B5164604460D46C4
:10D1C000FFF7DAFD33683BBBA3071ED12368134A80
:10D1D000934205D12B46E28811491248FFF739FEE8
:10D1E000114A934211D120466A461721FFF7C4FD28
:10D1F000009800F00703022B05D107F0F1FE02466C
:10D200002B460A49E9E70122FAE7204601F032FC01
:10D210002B4602460649E0E702B070BDC4A30508EC
:10D220000D8205086C8C05081C96050816820508F9
:10D230001E82050807B56A46FFF7BEFFDDE900015B
:10D2400011B903B05DF804FB02F0ACFCF9E7000093
:10D250002DE9FF41174606460C461D4601F0FEFB30
:10D26000374A904208D12B463A462146304604B010
:10D27000BDE8F04104F0CABB818811F4C07814D035
:10D28000062C2DD100232F4F3B62FFF781FC034674
:10D29000304698472860E8B9396A19B1296004B066
:10D2A000BDE8F08108462C60F9E7062C18D1192159
:10D2B000304601AAFFF760FD019B6BB98A21304619
:10D2C00001AAFFF779FF03940021012001AAFFF7CB
:10D2D00001FF28600120E2E74146404601AAF6E747
:10D2E000002CEBD1384601F0B9FB17490AF0F2F9EE
:10D2F00001AA68B147213046FFF73EFD019B7BB193
:10D300002146204601AAFFF7E5FE28602046C6E731
:10D310009B213046FFF730FD019B0BB10397D3E70C
:10D3200038460A4903F019FE30B10949094803F0AB
:10D330006DFD28600220B2E73846FFF7DBFEF8E714
:10D340004492050870030020F88C0508F08E05084B
:10D3500026820508A88E05087FB545680646002286
:10D3600041F23211281D01F053F9044688B3694691
:10D37000406801AA01F0FCFC0024009BA34201D8F4
:10D3800004B070BD019B53F8240007F029FE054648
:10D39000014602AA3046FFF70FFF28460299FFF721
:10D3A00083FC0134E9E7EB68E60053F8340078B118
:10D3B00004280DD007F02CFE03785F2B08D0EB6813
:10D3C000985907F00DFEEB6833445968FFF76CFC81
:10D3D0000134AB68A342E6D8D2E7000073B5164625
:10D3E00005460C4601F03AFB427B5AB1042300EBA0
:10D3F0008202CDE900362146136928466A469847DD
:10D40000009B43B1284601F035FB23460246034901
:10D410000348FFF71EFD02B070BD00BF1E82050865
:10D420006C8C050873B50C46054601F017FB838824
:10D43000064619062ED403F4C073B3F5C07F29D075
:10D44000C37BB3B14CB900EB83031A69174B9A4203
:10D4500003D01020F2F774FE0446F37BB28806EB8B
:10D4600083031B69D20548BF1B682146284698479D
:10D4700078B96A460F212846FFF77EFC009B63B10E
:10D480001CB91020F2F75CFE04462146684604F001
:10D49000B7FB0546284602B070BD284601F0EAFAFF
:10D4A000034902460348FFF7D4FC00BF616B020842
:10D4B0003D8205085C8F050837B5044601F0CEFAB9
:10D4C000818811F4C0750AD00022104B1A62FFF750
:10D4D0005FFB0346204603B0BDE8304018476A466C
:10D4E00019212046FFF748FC009B3BB9204601F07C
:10D4F000C1FA074902460748FFF7ABFC6A462946CE
:10D500002846FFF7E7FD03B030BD00BF70030020E1
:10D510004A8205085C8F050830B505468FB000F0DB
:10D5200079FF284601F09AFA848814F4C0740AD06E
:10D5300000221B4B1A62FFF72BFB034628460FB055
:10D54000BDE8304018476A4619212846FFF714FC09
:10D55000009BE3B102A8F2F7BFFD014640B96A465D
:10D56000FFF7B8FD0446F2F78DFD20460FB030BD41
:10D57000039B0C4918680AF0ADF828B1039803F032
:10D5800011FC074B1862F0E70398F2F7B7FD284645
:10D5900001F070FA044902460448FFF75AFC00BF44
:10D5A00070030020F08E05084A8205085C8F05088C
:10D5B0002DE9F04F13688DB004460393002843D142
:10D5C00002F104095FFA81F8C1F3072708EB47036A
:10D5D00059F823604FEA830B76104BD1354609EB9F
:10D5E0008803009309EB0B034FF0000B954A02935D
:10D5F0004FEA880A09EB880302998B423ED1BB446B
:10D600004FEA4B03019308F10103002E49D1019A1F
:10D61000D518A800F2F794FD83460CB101260460EA
:10D62000524649460BEB860024F089F908EB0604C4
:10D63000019E2644AE4205D95846B100F2F79BFD43
:10D640003546834626468DE0546802F10809B9E75D
:10D6500026FA0AF3D80708D559F82A0001F008FC81
:10D6600018B101F0E3FA013805440AF1010AD04586
:10D67000EED1B4E74FF0000A5546F8E7196871B9E2
:10D68000586860B181070AD10168914207D10193BE
:10D6900003F00BFA0BF1FF3B6A4A019B834408330A
:10D6A000AAE71D44019B1D44A800F2F749FD8346EB
:10D6B0000CB10460012400271CE026FA07F2D2070F
:10D6C00059F8270036D5830717D102685E4B9A4276
:10D6D00002D05E4B9A4210D108AA07A901F048FB7C
:10D6E000079A0BEB84009200089924F028F9079A16
:10D6F00014440137B845E0D19AE708A9FFF792FE34
:10D700008246A8EB070304935046FFF705FF024645
:10D710000028EED0049B19198D4207D85846E9001D
:10D720000592F2F728FD8346059A6D004BF82420F8
:10D730000134E9E74BF824000134DAE7009BD3E930
:10D74000001A002975D11AF0030739D1DAF8002040
:10D750003C4B9A4234D1DAF80820974215D3009B0B
:10D7600008330093009B029A9342E7D1321B214673
:10D770005B4652080398FFF751FC04465846F2F7FF
:10D7800007FD20460DB0BDE8F08FDAF80C204FEA17
:10D79000C70852F8370088B104280FD000F00702FC
:10D7A000022A01D008F032FC4BF82600DAF80C20EF
:10D7B000B10042445268594402364A600137CAE710
:10D7C0006A21504608AAFFF7F7FC002108AA08467C
:10D7D000FFF780FC0021FFF725FE80464046FFF75B
:10D7E0009BFE07460028BAD0721CAA4207D35846AF
:10D7F000E900F2F7C0FC4FEA450983464D4607F0C1
:10D800000702022A03D0384608F000FC07460F2121
:10D81000504608AAFFF7D0FC08AA002101200A9769
:10D82000FFF758FCB2005A444BF82670023650609D
:10D83000D4E7B2005A444BF826100236C2F804A0CE
:10D840008DE700BF488B0508C8A105087894050836
:10D8500070B583070C46154686B01BD103681D4A78
:10D86000934202D01C4A934214D102AA01A901F0AA
:10D870007FFA019BA34228D31AD8029B043D03EBF5
:10D8800084049C4201D106B070BD54F8042D45F8C3
:10D89000042FF6E702A9FFF7C5FD00230646019312
:10D8A000019B3046A34206D3FFF736FE0028EAD09C
:10D8B00022460A490BE0FFF72FFE30B1019BDA4305
:10D8C000224445F822000133E9E7019A044905485A
:10D8D000FFF7BFFAC8A1050878940508718205080A
:10D8E00058820508A48F05082DE9FF4183071546D6
:10D8F000CFB2C1F3072437D103683A4A934202D02A
:10D90000394A934230D10290029803AA01A901F04A
:10D910002FFA01983B1983425ED80026039901EB48
:10D920008003A64216D1C01B01EB8701801B05F0C6
:10D93000C5F805EB860842460399BC0045F8260069
:10D940000B19994202F104020AD10023029304B098
:10D95000BDE8F08153F8042D45F826200136E0E7B4
:10D9600053F8040D1060ECE70021FFF75BFD002386
:10D9700080460193019BBB4219D30021084605F064
:10D980009DF806464046FFF7C7FD0146D0B9B1688D
:10D99000A14221D305EB810245F8246005EB840305
:10D9A000091BAB4212D1304605F0A3F8CFE7404641
:10D9B000FFF7B2FD80B1019BFA1A224445F822001C
:10D9C0000133D6E7304604F095FEDBE7F468D01A61
:10D9D000205843F8040DE4E7019A04490448FFF78E
:10D9E00038FA00BFC8A105087894050858820508D0
:10D9F000A48F05082DE9F04F85B000AF07F10802AC
:10DA000005460C46FFF7B8F9D7E9020129B102F043
:10DA1000C9F81437BD46BDE8F08F0028F9D140F2AF
:10DA20003121284607F10802FFF7A6F9BB6823B9A0
:10DA300022461F491F48FFF70CFA07F10802284643
:10DA40001721FFF799F9391DB86807F049FB82469D
:10DA50002046F3F74FF9D7F80490514609F1010633
:10DA60008519EB1D23F00703ADEB030D6B464A460A
:10DA700018464FEAD30B23F062FF2E23204609F805
:10DA80003B30F3F742F9E84681462046F3F732F996
:10DA9000464402464946304623F051FF2946404657
:10DAA000F3F76CF801221E21FFF740FBB1E700BF3E
:10DAB0008B8205081C8D050808B50446F2F7FCFBAF
:10DAC00018B104490448FFF7BBF92246034902484C
:10DAD000FFF7BFF991820508F48D0508B8820508A3
:10DAE000014608B50148FFF7ABF900BFA48F050850
:10DAF0002DE9F043072805460F46164687B004D1A6
:10DB000091421AD04FF00E0918E1022801D00528E1
:10DB100007D132463946284607B0BDE8F04301F048
:10DB2000F7B908282AD1104603F0F6F940B131467A
:10DB3000384603F012FA0028E4D04FF01E09FDE049
:10DB400016F0030440F025813268AF4B9A4240F052
:10DB5000208106F108097368A342D3D959F8048BD0
:10DB6000404603F0D9F9002800F076814146384656
:10DB700003F0F3F90028E0D10134ECE7C80740F1E5
:10DB800025814FEA6108D10740F1F2805410232D1E
:10DB900000F2FF80DFE815F0D600DA00FD00DE00BD
:10DBA000E200FD00FD00FD00FD0024002F0032001A
:10DBB00035005D00650068006B00FD0071007900B4
:10DBC0008C00940024002F00320035005D006500B9
:10DBD00068006B00FD00710079008C009400B800B3
:10DBE00048EA040090EA40034FEA400900F1BA8095
:10DBF00049F00109A2E088EA0400F3E708EA04001A
:10DC0000F0E7002C02DA8148FFF76AFF1F2C09DCDD
:10DC10006FF040432341434504DB4FF04043234131
:10DC2000434513DD4046C11704F01CFB0746384648
:10DC300000F014FF037B002B40F0CF80A5F1090317
:10DC40000C2B00F2D6800D35EDB2F0E708FA04F0A7
:10DC5000C8E7002CD7DB1F2CA8BF1F2448FA04F00C
:10DC6000C0E708EB0400BDE7A8EB0400BAE788FBB7
:10DC70000404B4EBE07FB5D0D4E7002C00F0EE80D4
:10DC8000214640460DF0F0FFACE7002C00F0E680A6
:10DC9000404634F0B3F80546204634F0AFF801466C
:10DCA000284634F0B3F907B0BDE8F04303F040BABA
:10DCB000002C00F0D380214640460DF0C7FF91E7CD
:10DCC000002C1EDA404634F099F8324601462846C8
:10DCD00007B0BDE8F04303F08BBAE20704D580FB40
:10DCE0000302B2EBE07F9DD1012C3FF47BAF83FBBD
:10DCF0000332B2EBE37F4FEA640493D1002CECD102
:10DD000070E743460120F9E7002C00F0A7800021CE
:10DD1000022008F0F3FC2146814640460DF0A4FFA6
:10DD2000400040F00100C9F80800214640460DF0CF
:10DD30008DFF400040F00100C9F80C00484607B0D4
:10DD4000BDE8F083A045FFF6F8AEDBE6A0453FF75F
:10DD5000F4AED7E6A0457FF7F0AED3E6A045BFF618
:10DD6000ECAECFE6C11707B0BDE8F04304F07ABAD5
:10DD700093072BD11368264A93421AD1404634F0B8
:10DD80003DF832460146284603F032FA8146002823
:10DD9000D4D1204B38465D5D00F06CFE0446304621
:10DDA00000F068FE234600902A461B491B48FFF7F7
:10DDB00050F81B4A934209D1404634F01FF83346CD
:10DDC00001460022284602F0CFF8DFE7062D01BF0A
:10DDD0003B46242537461E4629E700EB83000369AE
:10DDE0003246394628469847814600283FF426AFF8
:10DDF000A4E7A5F116030C2B14D83B460F35374684
:10DE0000EDB21E4613E700BFC8A10508E68205086B
:10DE10005490050832A30508FB8205085C8F0508AD
:10DE200024890508242D04D93B4637461E460F3D5C
:10DE3000EDB2242DADD1384602A9FFF7F3FA04461E
:10DE40002046FFF769FB00283FF45CAE314601F045
:10DE5000D9F80028F4D070E646469AE7014902480E
:10DE6000FEF7EEFF0E830508EC8F0508014608B5A6
:10DE70000148FEF7E5FF00BF5C8F0508014608B5C5
:10DE80000148FEF7DDFF00BF3C8E050807B5002204
:10DE9000019101AB012102F071FEF2F72FF90000B0
:10DEA000014608B5024809B9FEF7CAFFFFF7EEFFC1
:10DEB000F08E050808B500F0DDFD02490246024873
:10DEC000FEF7C7FF1A8305085C8F0508410008B5F7
:10DED000024841F00101FFF7D9FF00BF608E05083D
:10DEE00041F62A4108B50148FFF7D0FFA88E050882
:10DEF00030B58DB0044668460D46F2F7EDF848B9E6
:10DF000020462946FFF7DCF80446F2F7BBF8204626
:10DF10000DB030BD0199024800F0DAFD0024F6E7AB
:10DF2000B4710508054BD861B3F8B62112B2012AC5
:10DF300004BF0022A3F8B621704700BF7003002081
:10DF40000023024803643830FFF7ECBF7003002061
:10DF5000EFF3108172B6084AB2F8B6311B0451BF14
:10DF60004FF6FF73B2F8B63103F1FF331BB2A2F8DC
:10DF7000B63181F31088704770030020EFF31081F1
:10DF800072B60C4BB3F8B621013212B2A3F8B62127
:10DF900052B9DA692AB9D3F8B82112B993F8C02175
:10DFA0002AB10022A3F8B62181F31088704701221C
:10DFB000F8E700BF7003002070B5EFF3108572B66C
:10DFC0000F4B93F8C021042A18D0B3F8B641561C61
:10DFD00024B2012C04BF0024A3F8B64193F8C14138
:10DFE00083F8C061224402F00302243203EBC2032F
:10DFF000C3E90201012085F3108870BD0020FAE713
:10E000007003002030B5EFF3108572B60468C4B910
:10E010000D4BB3F8B62112B2012A4FF0000208BF2F
:10E02000A3F8B6414260D3F8BC2101603AB9C3F805
:10E03000B801C3F8BC01012085F3108830BD5060E1
:10E04000F7E70020F8E700BF70030020F8B50346AB
:10E050002C4C80B1E26972B1EFF3108272B6E069C4
:10E0600038B10021012BE16103D182F31088F2F76E
:10E0700045F882F31088B4F8B6311BB243B9EFF318
:10E08000108272B6B4F8B66136B216B182F3108857
:10E09000F8BD4FF6FF73D4F8BC71A4F8B63197B150
:10E0A000D4F8B8516B68C4F8B8310BB9C4F8BC31B6
:10E0B0002B682E6082F3108828469847EFF3108271
:10E0C00072B6AF42ECD194F8C051BDB194F8C131F1
:10E0D000013D03F12401013304EBC10103F003030B
:10E0E00084F8C13184F8C051D1E9020182F310886B
:10E0F000FFF7FEFEBDE8F840FFF740BF82F310884F
:10E10000F8E700BF700300200120FFF79FBFFFF773
:10E11000FBBF0120FFF79ABF38B1044A1369984248
:10E1200002D010611846704700207047700300202D
:10E1300001F00F0108290DD8DFE801F011050A0CE4
:10E140000C0C0C0C0E00002814BF1E200E20704773
:10E1500004F098B804F0B1B8C00040F00200704775
:10E1600008B500F0B3FD33F0E7FC08BD00F0AEBD2C
:10E1700008B533F039FDBDE8084002F0D9BF02F020
:10E18000D7BF0000F0B58DB0054668460F4614466F
:10E190001668F1F7A1FF78B9002E0CBF39460021AF
:10E1A000234632462846FFF753F80546F1F76AFF43
:10E1B000012D0BD1284611E0019B236010492068F6
:10E1C00002F0CBFE60B92068F1F798FF2368002DBC
:10E1D000F4D10BB9062323603EB900200DB0F0BD89
:10E1E000206802F0DFFD2060F6E73046054902F0C6
:10E1F000B4FE0028F1D03046FEF77CFFE4E700BF14
:10E20000F08E0508F88C0508036803B94068FFF72D
:10E2100083B91346C1F30722C9B2FEF7FFBE1FB58B
:10E2200001F00F03012B044613D011F00E0F08D19B
:10E230008BB10122204601A900F02CFF68B10198A2
:10E2400009E0023B012BF4D804B0BDE8104000F017
:10E25000F9BC00F033FE04B010BD204600F0F2FC23
:10E26000F9E708B528B1062803D0FEF743FFF1F718
:10E2700045FF08BD10B50C4619B9BDE81040FFF7C1
:10E28000D1B8FFF7CFF884421CBF0023C4E90030A7
:10E29000002010BD40F2D233984217D840F2CE335E
:10E2A000984209D85E281DD075281DD03E2814BF7D
:10E2B0004FF0FF3001207047A0F57470022803D89A
:10E2C000DFE800F00C0E14000420704740F25243C7
:10E2D000984214BF4FF0FF3003207047062070476C
:10E2E00007207047022070470020704705207047C4
:10E2F00038B5034615460C4609B92C460BE052B119
:10E3000011462046984758B1636833B9656044F0B8
:10E310000103A560EB60204638BDA368DD60F6E729
:10E320006B68E3606C60002BE7D145F00103AC60E3
:10E33000E360E2E7F8B5064631B1002511F00103CC
:10E3400004D000232946EB600846F8BDCC68CB60BA
:10E3500014F0010307D1E7682246E3603046FFF777
:10E36000C7FF3C4601460A4630462946FFF7C0FF34
:10E3700021460546E2E78A422DE9F04184460E46F1
:10E3800006D10023BDE8F04151685360FFF7D2BFCA
:10E39000D2F80C80B8F1000F12D01446E468E307FD
:10E3A000FCD524F0010463685168934208F001072A
:10E3B00016D1002339B99F4208BF41466160D3603E
:10E3C0003046BDE8F08160465360D360FFF7B2FF8E
:10E3D00005466060C5F80C80002FF1D0A560EFE71E
:10E3E0001D46DB689342FBD1002260465A60DA602A
:10E3F000FFF7A0FF0028EDD0E8600546EAE700003F
:10E40000034B82B0186801ABC01A02B0704700BF5E
:10E410007003002007B5064A01A9136852685B1A09
:10E420009A4201D8FFF75CFD03B05DF804FB00BF22
:10E4300070030020034610B5500C1446C2F34F027F
:10E4400021B1E10702D40C48FFF710FD904206D13C
:10E4500098420FD0024609490948FEF7FAFC984253
:10E4600004D9C21A07490648FEF7F3FC9A4201D2C2
:10E470000549F1E710BD00BFA0840508AA8405087E
:10E480005C8F0508BC840508C48405082DE9F74F96
:10E490000024DDE90CA706468B461546A046A1469A
:10E4A0000193019B9C4204D1B1453CD22248FFF725
:10E4B000DDFCB44210D2BAF802209205F6D45BF823
:10E4C000240009F101099AF80220012A24D100F060
:10E4D000F5FC07F8240017E0BAF800100022C90084
:10E4E000284641F0020100F093F888B9BAF80220FA
:10E4F000D30505D5BAF8002010491148FEF7A9FC4C
:10E50000DAF8042047F8242001340AF1080AC8E7A1
:10E51000406808F10108D6E7022A01D100F086FB25
:10E5200047F82400F0E72B68B8EBD30F01D2054879
:10E53000BDE703B0BDE8F08FE2840508DD8405087F
:10E540005C8F0508EC84050870B51E460446154628
:10E5500086B002EB800203A800F031F80B9B29463D
:10E5600001930A9B2046009303AA3346FFF78EFFD0
:10E5700006B070BD08B50148FFF780FCF6840508B9
:10E5800003460022064931F8020B984206D20132B6
:10E59000222AF8D103EB530343F00100704700BF78
:10E5A0001C85050810B50446416019B98160012336
:10E5B000236010BDC800F1F7DCFDA060F7E7416003
:10E5C000C90041F00701016082607047037810B50F
:10E5D0009B07044602D48068F1F7DAFD0022236825
:10E5E000626062F3DF03236010BD037810B59B0700
:10E5F000044602D48068F1F7CBFD236803F00403DE
:10E6000043F0010323600023C4E9013310BD00007F
:10E61000022A2DE9F74F04460E46174612D04268EB
:10E6200082B18D4BC1F386010B4493F8C231B3FB29
:10E63000F2F102FB1133826802EBC30552F833306A
:10E64000B34211D0237813F0010A12D006F007026A
:10E65000022A0ED016F0030203D130687F498842A7
:10E6600006D0012F05D00025284603B0BDE8F08F65
:10E6700092465B0768D52268A56822F0070205EB81
:10E680000208454530D3012FEDD1D4E90032B2EB79
:10E69000D30FC3F3DC0111D104316160A068C9005C
:10E6A000F1F769FDD4E90032A2EBD30223F00703AE
:10E6B000A0600021D200184423F07FF92368A168EC
:10E6C000C3F3DC02501C60F3DF03236001EBC205DF
:10E6D00041F83260002206F007066A60022EC3D0BD
:10E6E000237862F3000363E02868B04222D1022F4E
:10E6F00016D12368A8EB0502083B6F6805F10801F5
:10E7000028462360083A23F042F900212568A368CF
:10E71000C5F3DC0225F007051D4443F832106F6095
:10E720004D4BC6F386061E44A368EB1ADB1086F831
:10E73000C23199E7BAF1000F04D1314600F062FC12
:10E740000028D4D108359CE7636823B9012F8AD10A
:10E75000204600F085F806F0070BBBF1020F29D127
:10E76000F008F2F7BBFA814663680025B9FBF3F2C3
:10E7700003FB12939846A16851F8380001EBC802D8
:10E78000F8B9012F7FF46FAF002D08BF154623683D
:10E79000BBF1020FC3F3DC0101F1010161F3DF03FF
:10E7A0002360C5E900603FF45FAF237860F30003A6
:10E7B000237059E731460620FEF79CFB4FEA6009BB
:10E7C000D2E704281AD1002D08BF1546626808F167
:10E7D0000108B8FBF2F102FB11884345CBD1012FB0
:10E7E0007FF441AF002D33D000222368BBF1020F2C
:10E7F00003F1080323602E606A6070E7B04218D10D
:10E80000022F0ED123686168083B236008F10103E1
:10E81000B3FBF1F001FB1033A16851F83330ABB911
:10E8200013600D4BC6F386061E44154686F8C2815A
:10E830001AE7BAF1000FC9D13146CDE9003200F034
:10E84000E1FBDDE900320028C0D0D9E70423E7E787
:10E85000204600F005F887E77003002074A0050843
:10E860002DE9F04146680446701CFFF789FE054615
:10E87000C000A768F1F77DFC4FF0000823686560D1
:10E8800003F0060343F001032360A0603D1DB04583
:10E8900004D13846BDE8F041F1F77ABC55F8041CC4
:10E8A00039B1042905D001222046FFF7B1FE2B68BB
:10E8B000436008F101080835E9E7002310B5044674
:10E8C000016043608800F1F754FCA06010BD03684C
:10E8D0002DE9F74F04468B46914623B912F0010FFC
:10E8E00062D000F064F859460620FEF703FB236867
:10E8F0004710B7FBF3F603FB167609F0010300930C
:10E9000035460023A0684FEA850A50F8258000EBC1
:10E910008502B8F1000F0CD119F0010F44D0002B83
:10E9200008BF13466268D84601326260C3F800B07F
:10E9300034E0B8F1040F17D1002B08BF134622684A
:10E940000135B5FBF2F002FB1055AE42DAD1009A68
:10E9500052B3002BE6D1204600F029F82368B7FB1C
:10E96000F3F603FB1676CBE759464046019300F0D9
:10E9700049FB019B0028E2D019F0020F0ED022685B
:10E980000135B5FBF2F1636802FB1155013B636091
:10E99000A36853F825202AB943F80A20404603B05B
:10E9A000BDE8F08F0422F7E74FF00008F6E7F8B56E
:10E9B000076804468668781CFFF7E2FD00252060A2
:10E9C00065608000F1F7D5FBA060BD4204D1304600
:10E9D000BDE8F840F1F7DCBB56F8251029B1042951
:10E9E00003D001222046FFF772FF0135EDE7024612
:10E9F000002370B50168994201D1002014E09468A9
:10EA000054F8230004EB830601330028F3D00428D4
:10EA1000F1D05568013D5560B3FBF1F201FB1233B3
:10EA200054F823300BB9336070BD0423FBE710B5F5
:10EA300004468068F1F7ACFB0023C4E90033A3600F
:10EA400010BD704710B50C46F1F77AFB046010BD9D
:10EA500010B50C46F1F782FB046010BD830717BFA9
:10EA6000034B006800F00F0053F82000704700BF10
:10EA70004C86050808B5FFF7F1FFBDE80840C088DF
:10EA8000F2F743B970B50D4604461646FFF7C2FCCF
:10EA90002846FFF7E3FF437A43B100EB8303324696
:10EAA00029462046BDE870401B691847C2880349C3
:10EAB0002046BDE87040F2F7CFBE00BF6085050874
:10EAC0000A4601460148FFF7DDBF00BFA8B20508AE
:10EAD0002DE9F347044608460E4602F037FA98B18E
:10EAE0006946304601AA02F076FA009B63B12046DF
:10EAF0001949F2F7FCFA009D184FDFF86480DFF83F
:10EB00006490033D002D0BDA314620460222FFF7C8
:10EB1000B9FF2046134902B0BDE8F047F2F7E7BA63
:10EB2000019A394602EB85035B6852F8252020469E
:10EB3000F2F792FE019B4FEA850A53449A682AB97C
:10EB400049462046F2F7D3FA033DDBE7414620462B
:10EB5000F2F782FEF8E700BF65850508898505089C
:10EB60009E8505080CBA050808B50246FFF776FF32
:10EB7000837A53B100EB83031B6906498B4204D1AE
:10EB8000BDE80840104608F079BD181E18BF0120E6
:10EB900008BD00BFA1740208830713B5044603D162
:10EBA00002680D4B9A4208D021460820FEF7A2F9D0
:10EBB00010B92046FFF77EF9044614F0010103D096
:10EBC0006010E11702B010BD6B460822204603F02A
:10EBD0007FFADDE90001F5E7249305080E2838B532
:10EBE00003460D4603D100230B60012403E01E28D9
:10EBF00003D101240C60204638BD10F0010402D07E
:10EC000043100B60F7E7820707D10168064A91427B
:10EC100003D103F07BFB2860E7E719460820FEF7E5
:10EC200069F90028F5D1E6E72493050813B501A991
:10EC30000446FFF7D3FF10B92046FFF73BF90198D0
:10EC400002B010BDC20705D4830705D10268034B8B
:10EC50009A4201D103F053BBFFF7E8BF24930508A4
:10EC60000E2838B503460C4626D01E2826D010F0B4
:10EC7000010505D0401033F0C1F80125206019E0EE
:10EC800081070CD102680F498A4202D103F084FC4B
:10EC9000F3E70D498A4202D102F0A8FAEDE71946DE
:10ECA0000920FEF727F928B1820703D10268064B35
:10ECB0009A42F1D0284638BD0020DEE74FF07E5062
:10ECC000DBE700BF249305085490050813B501A99C
:10ECD0000446FFF7C5FF38B92046FFF7CBFE0449CD
:10ECE00002460448FEF7B5F8019802B010BD00BF17
:10ECF000A78505085C8F0508F8B505460F4616463A
:10ED0000FFF7AEFF044618B1002333602046F8BD7C
:10ED1000A9070AD12A680C4B9A4206D132463946D5
:10ED2000284601F01BF90124F0E729460A20FEF7E6
:10ED3000E1F80028EAD08207E8D10268024B9A4243
:10ED4000E4D132463946ECE72489050810B504467B
:10ED5000FFF7D2FF38B92046FFF78CFE0249024682
:10ED60000248FEF776F810BDB28505085C8F0508ED
:10ED700038B5840703460ED104680B4DAC4203D16D
:10ED8000BDE8384007F0C8BD084DAC4203D1BDE82E
:10ED9000384003F0A9BE1846FFF76CFE044902464E
:10EDA0000448FEF756F800BFC8A105087894050886
:10EDB000B98505085C8F050813B50C4601A9FFF756
:10EDC000D7FF019BA34204D0224603490348FEF724
:10EDD00040F802B010BD00BFC2850508A48F050829
:10EDE000F7B51F46D30706460D4614460FD55410F7
:10EDF0000194019A002ABCBF52190192019AD7B11D
:10EE0000002A14DA00230193019803B0F0BD1046E4
:10EE100001A9FFF7E3FE0028EBD12046F588FFF7B4
:10EE200029FE2A46034608490848FEF712F8AA4276
:10EE3000EAD90195E8E7002A01DBAA42E4D3F28887
:10EE400003490448FEF705F8D48505085C8F0508DA
:10EE5000EB850508648D0508820701D003F012BA1E
:10EE6000002801DA03F029BA400040F001007047A1
:10EE70008307014610B510D102680F4B9A420CD19E
:10EE800000F00703022B06D1C008F1F733FF400062
:10EE900040F0010010BD8068F9E70846FFF7DEFD8D
:10EEA000C37A33B1BDE8104000EB8300036905204D
:10EEB00018471846EEE700BF009F05080E2810B55A
:10EEC000044622D01E2801D1012010BD06281CD0E6
:10EED000C20703D5013818BF0120F6E7FFF7BEFDD2
:10EEE000C37A5BB100EB8300036921460420984795
:10EEF00020B1A0F11E0358425841E6E72046FFF733
:10EF0000B7FF0028E0D00138E5E70020DDE700008A
:10EF100005282DE9F04715BF1E260E264FF00E09D5
:10EF20004FF01E09914280460C46154607D1C8078E
:10EF300020D40846FFF792FD838859071AD504F0BC
:10EF40000703022B05D0A20717D122682C4B9A4247
:10EF500013D105F00703022B05D0AB0712D12A68A5
:10EF6000274B9A420ED12946204605F0F0FF002893
:10EF700008BF4E463046BDE8F08714F0010A06D0BF
:10EF8000EF0738D423464FF0010A2C461D46204691
:10EF9000FFF764FD027B07469AB18188080704D415
:10EFA0002846FFF75BFD87420BD1B8F1050F0FD064
:10EFB000387B2A4607EB8007214602203B699847A9
:10EFC00098B9BAF1000FDDD0AC4218BF4E46D1E778
:10EFD000CB06EDD507EB8202136921462A4640464F
:10EFE00098470028E4D00646C4E7B8F1020F04D0E1
:10EFF000FFF764FFBBE74E46BCE70646BAE700BF33
:10F0000074A0050808B50A4601460220FFF780FFF4
:10F01000BDE80840FFF752BF10B50446FFF728FFD0
:10F0200038B92046FFF726FD024902460248FDF79F
:10F0300010FF10BDF28505085C8F050838B5044641
:10F04000FFF70CFD837B15462BB100EB83000369B2
:10F0500020469847A0B9204635B9FFF70BFD024678
:10F0600008490948FDF7F5FE042D04D1FFF702FD1C
:10F0700006490246F5E7FFF7FDFC05490246F0E7C1
:10F0800038BD00BFFF8505085C8F0508128605089E
:10F090002486050838B50546FFF7E0FC037C1446D6
:10F0A0001BB914F004000BD138BD00EB83031B69BE
:10F0B000284602F0030298470028F2D10120F3E726
:10F0C0000148FEF7D3FE00BF2F860508042803D0B1
:10F0D000052807D0002070478B68002B14BF1E2026
:10F0E0000E2070478868400040F001007047000023
:10F0F0000346084A0846C1E900230022C1E902226A
:10F100001968054A914202BF5B68C3F31723836005
:10F11000704700BF68870508B4870508F8B50D4635
:10F120000179044601F07F0116464020002208F0D4
:10F13000A5FFA268E36842436A602279276802F06B
:10F140007F01A96008492B608F4209D1110601D4C3
:10F15000B20707D46268C2F3172200FB02332B60A8
:10F160000020F8BD0120FCE7B4870508F8B50022AF
:10F1700005460E460146402008F080FF0746102055
:10F18000F0F7DEFF094A0A4B0571012D18BF13463F
:10F190000360436804466FF31F23C0E9013606FB92
:10F1A00007F0F0F7CDFFE0602046F8BD3487050892
:10F1B000808705084268C368916830B48B420AD2E0
:10F1C0001479D16882685D1CC5601A4404F07F0020
:10F1D00030BC08F0B3BF002030BC7047F8B54668BB
:10F1E000044636F0FF060F461AD132460179402018
:10F1F00008F044FFA168054608314143E068F0F794
:10F20000BAFF08226368E06062F31F236360A368AB
:10F21000314603FB0553C5EBC502184422F0CDFB74
:10F22000D4E902213B46207909F0ECF9A3680620D5
:10F230000133A3606368A3F580736360F8BD0000C9
:10F24000F8B50E790546012E0C460ED11A49F1F794
:10F250004EFFD4E902213346284605F0EBF8284654
:10F26000BDE8F8401549F1F742BF32461449F2F7BC
:10F27000F3FAA368002BF2D028461249F1F737FFC2
:10F280000026114FA368B34204D828460F49F1F76E
:10F290002EFFE4E71EB139462846F1F728FF324633
:10F2A000E168207908F04AFF012201462846FFF76D
:10F2B000E9FB0136E6E700BF8C860508BD4C060871
:10F2C00098860508A3860508A78605085C2F06080A
:10F2D0002DE9F04F04460D46164689B00AB90025BF
:10F2E000DDE011F003078068DFF82CA240F0EC802D
:10F2F0000B688A4A934240F0E78002AA08F03EFB7E
:10F3000010B98748FEF7BAFD2179042E3A464FF02E
:10F31000400001F07F0100F0A38008F0AFFE16F07E
:10F320000302054662D131688B7B002B4FD001EB85
:10F33000830318697B4B984249D13179402001F011
:10F340007F0108F09BFEA84202D07748FEF7C8FB79
:10F350003368D6E9029B534545D17368C3F3172838
:10F3600005FB08F8DDE9020322681B1A5245E7682D
:10F37000A9EB03063CD194F90420002AAFDA002E51
:10F38000E3D16268C2F3172205FB027705FB09F29D
:10F390000BEB080105FB0070019322F0F8FA0399CA
:10F3A000A2680298521A48446A4305FB017105FBA2
:10F3B000007022F0ECFA019BA068A3EB0902304434
:10F3C00000216A4305FB007022F0F7FA3BE0574B3F
:10F3D00099420BD1012DB8D10522304605A9FFF77E
:10F3E00059FEDDE905B94FF00008BBE7504889E751
:10F3F000002ECBDD6368B6EB132F2FD9A1683846FA
:10F4000031446943F0F7B7FE8246BB4508BF8346E7
:10F410006368E06066F31F2363600298A268039943
:10F4200048443244121A6A4301FB05A105FB00A0BF
:10F4300022F0ADFA029805FB09F200FB05A00BEBE8
:10F44000080122F0A4FA6368C6EB132262F31F23BB
:10F450006360A3683344A360062520E0BA46DCE776
:10F4600008F00CFE236806465345029B1BD1B3F1FE
:10F47000807F03DB2F493048FDF7E2FC1020F0F7D6
:10F480005FFE054694E80F0085E80F00029A02EB44
:10F49000112363F31F216960039B9B1AAB6028460D
:10F4A00009B0BDE8F08F03992079C91AFFF75EFE15
:10F4B000DDE90232E168D21A0546724306FB031108
:10F4C000C06822F03CFAEAE700232A460146206899
:10F4D000FFF786FC23680246534511D16368042E6A
:10F4E00000EB13220ED094F90430002BBFF6F7AED8
:10F4F00020793346E16800F07F0009F083F8ABE73C
:10F50000042EF5D12079E16800F07F0009B0BDE854
:10F51000F04F08F013BE00BFB4870508289B05080C
:10F52000AA860508D1F20108CA860508009F0508C9
:10F53000DF860508FA860508848E05082DE9F04364
:10F54000012807460E4685B008D08B0724D10B68EA
:10F55000254A934202D0254A93421DD101223046CA
:10F5600001A9FFF797FDB8B100223946402008F005
:10F5700085FD029E0546B6FBF0F638463146FFF79C
:10F58000F5FD06FB05F204460199C06822F0D7F9A3
:10F59000204605B0BDE8F0833046FFF769FC05461C
:10F5A00000B1451029463846FFF7E0FD002104462A
:10F5B0003046FDF737FF4FF0000806463046FDF7AE
:10F5C000ABFF03460028E3D025B919462046FFF7D4
:10F5D00005FEF3E742463846E16808F1010909F003
:10F5E00011F8C846EAE700BF009F050880870508B4
:10F5F00038B50C461146204606221D46FEF71AFF76
:10F600002CB92146BDE838400120FFF7AFBD29687D
:10F61000CB0719D411F0030303D10868124A9042B2
:10F6200012D001F00702022A04D043B90A680F4B36
:10F630009A4204D1012C02D10D48FEF717FC01209B
:10F64000BDE83840FFF77ABF0846FFF7EFFA0546F6
:10F6500001460120FFF78AFD04462A460021C068C2
:10F6600022F0ABF9204638BD2493050874A00508A4
:10F670000F87050838B50D461C4611462846094A2D
:10F68000FEF7D8FE206805F0C3FC012D007804D1F8
:10F69000BDE838400021FFF769BD6168BDE838402A
:10F6A000FFF74CBF04000200F0B50F4685B001A97A
:10F6B000044601223846FFF7EDFC014678B938468A
:10F6C000FDF7B0FE05462846FDF726FF014610B9B6
:10F6D000062005B0F0BD2046FFF780FDF3E70022CD
:10F6E0004020217908F0CAFC029D6368B5FBF0F563
:10F6F000B5EB132F0646C3F317221ED9A168294480
:10F700004143E068F0F737FD6368BC426FF31F23A5
:10F71000E060636004D10522204601A9FFF7BAFC2E
:10F72000D4E9020305FB06F200FB0630019922F042
:10F7300006F9A3682B44A360CAE7521B62F31F2398
:10F740006360EDE770B51B2806460C4615468CB085
:10F7500026D005D804286BD90E2850D000244BE0C1
:10F760002428FBD10122284603A9FFF793FC002897
:10F770004ED0A1075AD12268474B9A4256D1012256
:10F7800009A92046FFF7CAFCDDE90901012300931E
:10F79000DDE9032304F024FF002847D01E242BE0DA
:10F7A0000A683E4B9A42D9D00122204606A9FFF7AB
:10F7B000B5FC0522284609A9FFF76CFC00229DF83C
:10F7C0002010402008F05AFC0A9EA168B6FBF0F613
:10F7D000054631449DF82000FFF7C8FCDDE906121C
:10F7E0000446C06822F0ABF8E068079B06FB05F210
:10F7F0000999184422F0A3F820460CB070BD0A689D
:10F80000264B9A42AAD029462046FFF74DFFF3E740
:10F81000EA0702D50020FEF731FBAB0706D12B68C3
:10F820001F4A9342F6D01F4A9342F3D00E24E3E7D7
:10F83000012206A92046FFF771FC0122284609A9EA
:10F84000FFF728FC0028F1D0089A012A1DD05A2A77
:10F850001DDC014620320B9B012B1AD05A2B01DCF8
:10F86000014620339342D5D123F00203642BD1D03B
:10F87000022E01D00029CDD0DDE906120A9B3046C8
:10F880000093099B08F0B9F886E74222E1E70021DE
:10F89000E1E74223E4E700BF80870508B487050855
:10F8A000249305085490050870B5064610201446A8
:10F8B0000D46F0F745FC054A067102604268C460D7
:10F8C0006FF31F22C0E9012570BD00BFB487050892
:10F8D0007FB51D46084611464FF00212FEF7AAFDFD
:10F8E000052201A92868FFF7D5FB9DF80C400022EE
:10F8F00021464020029E08F0C1FB019AB6FBF0F1C0
:10F900002046FFF7D1FF04462868FFF7A7F80D4B04
:10F91000834209D12A6861685368C3F3172363F3EC
:10F920001F216160D368E3600322286801A9FFF703
:10F93000B1FB18B1237963F07F032371204604B033
:10F9400070BD00BFB487050870B505460E46014678
:10F950000120FFF70BFC04462A463146C06821F01F
:10F96000EEFF204670BD000038B505460C4610205D
:10F970000349FFF767F80122C460C0E9012538BDDB
:10F9800080870508136870B56BB94468A51C50F8EA
:10F9900025509C4207D055F82360B14204D1023370
:10F9A00050F82330136070BD0133F2E72DE9F047C2
:10F9B00016460F46134904460025F1F798FBDFF879
:10F9C0004890DFF848A006F108087368AB4205D8F4
:10F9D0002046BDE8F0470E49F1F789BB1DB1494605
:10F9E0002046F1F784FB57F8252051462046F1F7D1
:10F9F00033FF0122204658F8041BFFF743F8013576
:10FA0000E3E700BF159B0508A7860508E4870508FE
:10FA1000BD4C06084B680A46023351F82310FFF725
:10FA2000C5BF0E3918BF0121490041F00101FEF7A1
:10FA30005FB8052807D00E3918BF0121490041F0F1
:10FA40000101FDF757BA002070470000032A05D1D5
:10FA50000E2914BF04490549F1F749BB0E2914BF0B
:10FA600003490449F8E700BFA8710508AD7105080E
:10FA7000C8720508C272050838B50C461146204602
:10FA800002221D46FEF7D6FC1CB12868FFF716FAC5
:10FA900008B90E2038BD1E20FCE702280AD188686C
:10FAA0009368984208D148685368984214BF0E2062
:10FAB0001E207047002070470E207047136813B94E
:10FAC0004068FDF759B9704738B504460D460A46F7
:10FAD0000B49F1F7C1FE01222046A968FEF7D2FFCB
:10FAE00020460849F1F703FB204669680122FEF72A
:10FAF000C9FF2046BDE838400349F1F7F8BA00BF16
:10FB000038880508A672050855A20508062801BF11
:10FB1000D1E901305840400040F0010018BF0020FA
:10FB200070472DE9F84F984602EB43035D1C042B08
:10FB300082468B46164600AF4FEA85051FD8EB1D5F
:10FB400023F00703ADEB030D6C464FF00009204690
:10FB5000B96A2A1F40F804BB21F0F1FE2346424651
:10FB60005046711CFDF75AFA0446B9F1000F02D055
:10FB70004846F0F70DFB2046BD46BDE8F88F284605
:10FB8000F0F7E9FA04460028D9D08146DFE707B547
:10FB9000009313460A4681684068FFF7C2FF03B02E
:10FBA0005DF804FB38B505460C460C200249FEF70B
:10FBB00049FFC0E9015438BD4C88050838B50D46E9
:10FBC0004A680A490446F1F747FE696849B9204680
:10FBD0000749F1F78CFA2046BDE838400549F1F7AE
:10FBE00086BA01222046FEF74DFFF4E77488050827
:10FBF0007E88050855A2050810B50349044608206B
:10FC0000FEF720FF446010BD848805082DE9F04F01
:10FC10000446866801EB420906EB010A0AEB420042
:10FC200005280F461546984687B004F10C0B4FEA9D
:10FC3000890916D8B6003246594601A821F07FFE40
:10FC400001AB4A464146981921F079FE60682A4680
:10FC5000514601ABFDF7E2F90446204607B0BDE886
:10FC6000F08F8000F0F76CFA0646A26859469200C1
:10FC700021F065FEA0684A46414606EB800021F06F
:10FC80005EFEA16833462A4660683944FDF7C6F92E
:10FC900004463046F0F77CFADFE700002DE9F84330
:10FCA0000D4604461749F1F722FA012220466968F9
:10FCB000FEF7E8FE2A462046AB681349F1F7CCFD73
:10FCC0000026DFF84880DFF8489005F10C07AB68A4
:10FCD000B34205D82046BDE8F8430E49F1F707BA0C
:10FCE00057F8041B49B941462046F1F700FA494646
:10FCF0002046F1F7FCF90136E9E701222046FEF73C
:10FD0000C1FEF4E79C880508A68805087E880508DA
:10FD1000902F060855A205084068FDF72DB8000091
:10FD20002DE9F041CD1CAD0080460E46284608491D
:10FD30001746FEF787FE0446C0E901863946A5F15D
:10FD40000C020C3021F0FBFD2046BDE8F08100BF25
:10FD5000BC8805087FB50D4604460021686832F06E
:10FD600035FA064620BB14492046F1F7C0F94FF09A
:10FD7000FF3363200096CDE90130672233462046E9
:10FD80006968F1F74FFB02230C4E4FF0FF326321FD
:10FD9000CDE901210022A968009220466722F1F7EF
:10FDA00041FB3146204604B0BDE87040F1F79FB9F1
:10FDB0000023034EE9E700BF159B0508F0880508FE
:10FDC000F3880508136810B514463BB940F2F233C6
:10FDD000994204D1406801F0ABF9206010BD40F2B7
:10FDE0004E339942FAD18068F5E7000038B50546F0
:10FDF0000C460C200249FEF725FE4560846038BDA4
:10FE00002489050838B50C46072805D8DFE800F036
:10FE1000052304040704162D0024204638BD0021C4
:10FE2000606832F0D3F9002833D0A068002132F0A6
:10FE3000CDF900280CBF1E240E24EEE7886832F0AE
:10FE40000DFA0546606832F009FA85EA000464009C
:10FE500044F00104E1E76068896800F1004001F1C5
:10FE60000041BDE83840FFF7C1BF4968A5680846B2
:10FE700032F018F829460446284632F013F80146B5
:10FE8000204631F007FF20F0FBFEBDE8384001F0CE
:10FE90004FB91E24C1E700007FB50C46114620462D
:10FEA00004221D46FEF7C6FAECB1012C286821D0C9
:10FEB000820744D10268274B9A4240D14468866841
:10FEC0006D68AB0740D12A68224B9A423CD120464C
:10FED000A96831F0DDFE04463046696831F0DAFE8B
:10FEE0000146204601E00021084604B0BDE870400C
:10FEF000FFF77CBF00F00702022A034605D0810706
:10FF000014D1026814498A420DD103A905F0E8F81A
:10FF100000230093012303991A46FCF75BFA03467A
:10FF2000184604B070BD0B498A42F9D002A903AA51
:10FF3000FEF70CFF03990298FFF758FFEFE7FEF773
:10FF4000C5FE00260446BBE72846FEF7BFFE314645
:10FF5000C4E700BF2489050874A0050843680B6046
:10FF600083681360704700002DE9F34105460E4693
:10FF700014466946184601AAFEF7BEFE002800F0A6
:10FF80000E81A81E202800F21081DFE810F0FB008F
:10FF90000E010E010E010E010E010E010E010E01E9
:10FFA0000E010E010E0121002B007A000E01360019
:10FFB00039000E0196000E010E010E010E010E0118
:10FFC00021002B007A000E01360039000E01960048
:10FFD0000099304631F05EFE05462046019931F029
:10FFE00059FE08E00099304631F052FE019905466D
:10FFF000204631F04DFE044685E06E48FDF736FFA1
:020000040802F0
:10000000019F0021384632F0E1F8DDF80080002140
:1000100088B1404632F0DAF818B167496748FCF712
:100020000FFF4146304631F0F1FF4146054620467C
:1000300031F0ECFFDFE7404632F0C8F840B1394616
:10004000204631F0E3FF3946054606F10040EFE770
:100050004146404631F026FF39460546384631F0E4
:1000600021FF0146284631F015FE0146054640466F
:1000700031F0CCFF2946009007F1004031F0C6FF77
:100080000190DDF800803146404631F00BFF019FC2
:1000900005462146384631F005FF0146284631F035
:1000A000F7FD21460546404631F0FCFE0446314648
:1000B000384631F0F7FE214691E73146304631F0BF
:1000C000F1FE21460546204631F0ECFE0146284669
:1000D00031F0E0FD20F0D4FD0021054632F076F845
:1000E000C0B10021019832F071F888B1009D002163
:1000F000284632F089F858B10021284632F066F8D7
:1001000000284FD1002521462846FFF76FFE46E024
:100110002B4983E728461FF0F7FD31460546204668
:100120001DF06AFB019F04462946384631F0BAFEAD
:10013000DDF8008006462146404631F0B3FE014618
:10014000304631F0A7FD29460646404631F0AAFE6A
:1001500021460546384631F0A5FE0146284631F0D5
:1001600097FD1FF0A7FB044630461FF0ADFF214668
:1001700031F098FE0546304620F0F6FC214631F07D
:1001800091FE38E73146009832F020F878B12146E8
:10019000019832F01BF8002814BF1E200E2002B078
:1001A000BDE8F0814FF07E55ADE70020F7E70E2067
:1001B000F5E700BFF58805080A890508EC8F0508F2
:1001C0001789050813468A684968FFF7CDBED0E94C
:1001D00002120346C86882420AD00869496850F88A
:1001E000220001328A42DA6003D10022DA607047CD
:1001F000002070470346084603499A680160034996
:10020000C260C0E901137047E4960508CF010208F7
:1002100070B5C568426846696B1C9A4208BF0023E6
:10022000F607846805D5A34203D108490848FCF7BE
:1002300007FE0669A34246F82510C36004D10133C6
:100240009A4208BF00238360062070BD18B00508DD
:10025000648D0508836810B55BB14469C268E40722
:1002600003F1FF3307D5934205D109490948FCF74B
:10027000E7FD4368F1E704699342836044F8231083
:1002800003D103B94368013BC360062010BD00BF22
:1002900018B00508648D050830B585B005460846D8
:1002A0006946FDF7BFF804462046FDF735F90146DB
:1002B00010B9062005B030BD2846FFF7A9FFF3E7C7
:1002C00070B504460E461546CAB1D4E90213591A50
:1002D00048BF6368324648BFC91800680023FEF76C
:1002E0007FFDA36818446368834298BFC01A2369DE
:1002F000042D1ABF43F82050062553F820502846F5
:1003000070BD0000F8B50F461E4611460446134A5C
:100310003846FEF78FF87068FEF788FC051E02DA93
:100320000020FDF7DDFB21461820FEF78BFB0023A4
:100330000446681C6060C4E902338000EFF719FFCF
:10034000022F206103D9B068FEF770FC606120467F
:100350003168FFF7A1FF2046F8BD00BF060004008A
:1003600008B5D0E902239A4203D107490748FCF7B0
:1003700067FD03B9436800210269013BC36052F87D
:10038000230042F8231008BD4C890508648D050838
:10039000042803D0052808D000207047D1E90203C3
:1003A000984214BF1E200E207047D1E90230C01AB7
:1003B00044BF4B68C018400040F001007047000087
:1003C000D0E902318B42024610B503D108490948F1
:1003D000FCF736FD0024016951F8230041F8234061
:1003E000516801338B4208BF2346936010BD00BFA4
:1003F0004C890508648D05080346054A08460A60CD
:100400001A7A0A715B688B600023CB60704700BF6B
:100410009C8B0508044B88600B6001230B71002343
:100420000846CB60704700BF9C8B050808B5037970
:100430009B0702D50020FDF719FD08BD10B5044942
:1004400004460C20FEF7FEFA02220272446010BD40
:10045000788B0508F8B506460D4614460F6812B1AC
:100460003846FFF7E3FF22466968381DFEF7D0F8EB
:10047000034608B1406870B9022E05D1022C08D19C
:1004800069680748FDF702FDA868012C00D1586093
:10049000F8BD0620F9E7022C04BF00225A60F7E7F6
:1004A000888D05080122FFF7D5BF0222FFF7D2BFD2
:1004B0000022FFF7CFBF10B50446FFF7B7FF201D9E
:1004C000FEF793F8062010BD042803D0052808D0B5
:1004D000002070474B6833F0070314BF1E200E2026
:1004E00070474868C0F3DC00400040F001007047EE
:1004F000062802D10B7A022B02D04968FFF7E4BF2D
:10050000490041F001007047024630B50B6885682C
:10051000AB4201D300200AE0D46804EBC30054F8D6
:1005200033400133002CF3D0042CF1D00B6030BDEC
:1005300013B5044600F10C018068FFF7E5FF60B1D8
:100540002379012B0BD0022B43680AD0026869463D
:100550000220CDE9002306F0D1F802B010BD0068FA
:10056000FBE71846F9E70000F0B504460D46164BC8
:100570000A7A85B053F82210F0F7B9FD20461349E6
:10058000F0F7B5FD124B012600932B7A114F8DF831
:1005900004306B680293002303936846FFF7C8FF9B
:1005A000054628B920460C49F0F7A1FD05B0F0BD7D
:1005B0001EB939462046F0F79AFD01222946204609
:1005C000FEF760FA0026E8E73C8B0508D8890508A5
:1005D0009C8B0508A7860508DB8905081FB504461E
:1005E000FFF724FF636833F0070203D11149124873
:1005F000FCF726FC0022019222792046510744BFD5
:10060000C3F3DC0303F1FF3301A948BF0193FFF7F4
:100610007BFF63680422083B6360036802A90293BE
:10062000436803930023C0E90023022006F066F824
:1006300004B010BDDE890508888D05082DE9F04F4E
:100640000B68DFF8DC80032A15460FBFD0E9029A59
:100650000125DFF8D0A0DFF8D090434504460F46CF
:1006600085B005D0032D03D0DA883049F1F7F4F8CE
:1006700020462F49F0F73BFD002303930123DFF8C9
:10068000B4B0384603A90193FFF73EFF019B06462D
:1006900078B920462849F0F72AFD3B68434505D044
:1006A000032D03D020462549F0F721FD05B0BDE814
:1006B000F08F1BB949462046F0F719FD032D2CD1C8
:1006C000326802F00703022B27D012F0030308D18F
:1006D0001268117B29B102EB8102126918498A4222
:1006E00004D059462046F0F702FD01232A46204651
:1006F00031680193FEF7C6F9019B1BB159462046AC
:10070000F0F7F5FC51462046F0F7F1FC2A4620466A
:100710007168FEF7B7F90023B3E70023E6E700BFEF
:10072000488B0508A6810508A7860508F7890508EE
:10073000FB890508FD890508E67F0508BD4C06080C
:100740002551020810B5044904460C20FEF77AF939
:1007500000220272446010BD788B050810B5044970
:1007600004460C20FEF76EF901220272446010BDAF
:10077000788B050810F003030CD10268117A31B1AF
:1007800002EB8102136904481A1A5342534103F0E1
:10079000010070470023FAE7C50802082DE9F34776
:1007A000164607460C680D462046FFF73FFE3168A7
:1007B0003846304AC908FDF73DFE022F12D16F6856
:1007C0003846FFF7D7FF0146B8B12B689F4209D0E2
:1007D000002304F104080193686801A9FFF794FE5F
:1007E000074610B9002504343CE001224046396830
:1007F000FDF70EFF7B684360EEE73846FCF712FE1C
:10080000814604F1040A4846FCF786FE0028E9D038
:100810000021FCF707FE8046FCF77EFE07464046B7
:10082000FCF77AFE05464046FCF776FE0FB105B1AF
:1008300010B11148FDF754F9012239465046FDF731
:10084000E7FE4560DFE7B36853F8351003EBC507F3
:1008500039B1042905D001222046FDF7D9FE7B6875
:10086000436001357368AB42EDD8062002B0BDE8A5
:10087000F08700BF05000200FF89050810B50022BF
:1008800004300C46FDF7C4FE18B921460248FDF7B6
:10089000FDFA406810BD00BF888D0508024B40F886
:1008A000043BFDF77FBE00BF488B050838B5054601
:1008B0001020EFF745FC04462946FFF7EFFF2046DE
:1008C00038BD00002DE9F041804686B000200D467D
:1008D00016461F46FFF7EAFF0F4B0446984508BF30
:1008E0000379C0F8008004BF43F00403037155EAA4
:1008F00006030DD03B683146019007EB850203A843
:100900000293FDF75CFE03AA01A9681CFFF746FFEE
:10091000204606B0BDE8F081B48B0508F8B50C465A
:10092000064600216068FCF77DFD022E05466068E2
:1009300094BF0626A668FEF79BFA50B9FFF7B6FFEC
:100940000446071D2846FCF7E7FD014618B9204676
:10095000F8BD4010F2E701223846FDF759FE466027
:10096000F0E738B504468068FFF7A0FF0546236826
:1009700062680360237922F0070203F00503134342
:100980004360A268E168D200C06820F0D8FF284622
:1009900038BD0000F0B516280C46154685B061D06C
:1009A00005D8022810D0092860D0002409E02428A6
:1009B000FBD100222946201DFDF72AFE002841D147
:1009C0000E24204605B0F0BD02F003038A0725D1AE
:1009D0000A682C498A4221D1002BF1D12968914221
:1009E0001ED1CDE9013301A92046FFF78DFD02A9F3
:1009F00007462846FFF788FD0646002F3ED0002810
:100A0000DED031683868FEF7FDFA0028D8D071686A
:100A10007868FEF7F7FA0028E5D1D1E7002BCFD1AF
:100A20002A68194B9A42CBD163686A68534033F005
:100A30000703C5D102930435204602A9FFF764FDE0
:100A4000064608B91E24BCE7002228463168FDF797
:100A5000DFFD0028B4D041687068FEF7D3FA0028A3
:100A6000EAD1ADE70846FFF77CFF0446074A02A932
:100A70000220CDE90245FFF791FEA2E700289FD1B1
:100A8000E0E700BFB48B0508488B0508308B0508EC
:100A900010B40C7A012C05D1242803D1496810BC6C
:100AA000FFF778BF002010BC70474068C00870474F
:100AB00070B504460E461546FFF7B8FC01223146D4
:100AC000201DFDF7A5FD4560204670BD022213B52F
:100AD0000446CDE9000169461046FFF7BBFC2046FD
:100AE00002B010BD38B50C461AB9FFF7EFFF06206B
:100AF0000BE0042A0AD100220430FDF789FD18B961
:100B000021460448FDF7C2F9406838BDFFF7D0FF21
:100B1000EDE700BF888D050813B504464068FCF773
:100B2000FBFC58B1A36869465A1C5B0043F0010303
:100B3000CDE90030A260022005F0E0FD02B010BD5A
:100B40001FB50446084611461A4602AB01930A4BEC
:100B500000930223FDF7F8FC21460C20FDF772FFFD
:100B6000002104460298FCF75DFC60602046039B70
:100B7000A36004B010BD00BFE88B05082DE9F0416B
:100B80000E46044611463046124A9846FDF752FC7E
:100B90001020EFF7E0FA104D0023002818BF05469B
:100BA0002C60AB6026B90D4C2846EC60BDE8F081A6
:100BB000B71CBF003846EFF7CEFA04460028F2D043
:100BC000074B4146C0E90036A7F10802083020F083
:100BD000B6FEE9E7FEFF010098030020C0A105086A
:100BE000C8A10508F8B5C36806465A68012A12D19B
:100BF0009C6814F003070ED12268114B9A420AD167
:100C0000E3681B78FF2B16D14A20EFF7A4FA0546BC
:100C100010B90C4BF360F8BDE168F0F7F1F8284625
:100C2000E56020F0FEFEC4E90170D4E90210EFF7A0
:100C30003BFF6060EFE76368002BECD1F5E700BF96
:100C400074A00508C0A10508F8B5164602F07F0794
:100C5000320605460C460AD47B1E012B07D80B68CA
:100C6000D888F0F752F801462846F0F740FA022FEC
:100C700003D128462249F0F73AFA2046FFF7B2FF9F
:100C800016F07D0734D1E3680BB15A682AB92846BB
:100C9000BDE8F8401B49F0F72ABA20681A49884293
:100CA0001FD1022A1DD89868C3071AD509F0FCFA8B
:100CB0000346B0B1E2682846926814495210F0F732
:100CC000CBFDE3685B68012B19D90D492846F0F785
:100CD0000EFA3A46E368D9682846BDE8F840FDF7C1
:100CE000D1BEE3685A68012A02D100229968F3E76D
:100CF00032462846E168BDE8F84005F085BCF8BDFD
:100D0000A681050885360608608E0508148C05083E
:100D1000F8B51546D0E901230F465919914204460A
:100D20000FD30178D9B105F11006164431460122DE
:100D3000C068EFF72BFA78B96568A268013D2070AA
:100D4000AD1A2A46D4E902303946184420F0F7FD9E
:100D5000A2682A44A260F8BD6660E060F1E7013A4B
:100D6000D51AEEE738B50546FDF778FE007A70B182
:100D70002846FDF773FE04462846FDF76FFE007A0D
:100D8000034B04EB80042069C31A5842584138BD14
:100D90007D0B020810B50446FFF7E4FF00B9246993
:100DA000204610BD10B5FFF7F5FFC36804465B6829
:100DB00023B1FFF717FFE368986810BD0620FCE732
:100DC00038B513680546144653B140F236239942AC
:100DD00005D15368062B02D10023C380236038BDA0
:100DE0003D2903D1FFF7FEFEEB68F7E7A22903D008
:100DF00040F2FB239942F2D12846FFF7D3FF20604F
:100E0000EDE700231A461946FFF7B8BE73B505464D
:100E100010200E46EFF79FF9044640B903460246FC
:100E20000146284602B0BDE87040FFF7A7BE084B58
:100E30000360304620F0F5FD0022C4E902060121DE
:100E40002846626001AB0194FFF798FE02B070BDC6
:100E500074A005082DE9F04306469BB010200D460E
:100E60009046EFF778F90446284620F0DAFD00F1C5
:100E7000010907464846EFF76EF944B92346224672
:100E8000214630461BB0BDE8F043FFF777BE70B98E
:100E9000C4E902750022174B6260236001213046CD
:100EA00007AB0794FFF76AFE1BB0BDE8F083012390
:100EB0008DF80C300023CDE9053003AB01930E4BC8
:100EC000CDF8109002932B78FF2B04D1294607A868
:100ED000EFF796FF07AD4246294601A8F0F718FB49
:100EE000DDE905320021D154059BA360069BE36038
:100EF000D0E700BF74A00508110D02080EB403B5B9
:100F000003AA52F8041B0192FFF7A4FF02B05DF898
:100F100004EB03B07047000083070BD10268084B55
:100F20009A4207D1037A2BB100EB83031A69054B70
:100F30009A4202D0044906F0CDBB0120704700BFA1
:100F4000C4A305087D0B0208908C050808B5FDF7C1
:100F500085FDBDE80840FFF7DFBF38B504460D4604
:100F6000FFF7F4FF18B12046FDF778FD0446294647
:100F70002046BDE8384006F0ADBB2DE9F04188467B
:100F800017461E46FFF706FF0446806890B90C20FE
:100F9000EFF7E1F8A06058B103236360E388A1682C
:100FA000D81C01EB8302E08041F82380C2E901767E
:100FB000BDE8F081E388A5880233AB42EEDB033560
:100FC0000122A900EFF7E2F80028F1D0A388A06081
:100FD0000333A380E2E738B50D461446FFF7DAFE87
:100FE000836813B92B60236038BDC2882A60FAE792
:100FF00037B50446A068FCF78FFA019068B16568C0
:10100000062D05D000220121284601ABFCF706F889
:10101000FDF754FF0028EDD0019803B030BD38B57E
:1010200004461D46084611464FF00412FDF702FA29
:1010300021460C20FDF706FD2B6804464360002185
:101040006868FCF7EFF9A060204638BD1FB54FF087
:10105000FF336322CDE901320023009367224FF46E
:1010600080734968F0F7DEF905B05DF804FB2DE9FF
:10107000F04780460F46006809681DF079FAD8F8F5
:1010800000A0D7F8009001460446504630F000FE1C
:10109000494630F0BBFF00210646204631F096F865
:1010A00098B14C466FF31E040021304631F08EF8A3
:1010B00040B34946504630F0A9FF05466FF31E0580
:1010C000C8F800503C60BDE8F0870021204631F0B0
:1010D00087F80021051E484618BF012531F080F829
:1010E000003818BF0120EDB28542DDD049462046C8
:1010F00030F0D0FD4FF07E510446304630F0C8FD50
:101100000646D1E730461EF06FFF014605463046E1
:1011100030F0BEFD4FF07C5131F080F80028CFD088
:1011200028464FF07E5130F0B5FD0546C8E7000077
:1011300010B504460820EFF703F8024A4460026045
:1011400010BD00BF5490050830B50D4687B011465C
:10115000284602221C46FDF76DF92DB9002007B084
:10116000BDE83040FFF7E4BF0122206803A9FDF786
:1011700091FF40B1DDE9030100231A460093FBF71C
:1011800029F907B030BD2068830703D10268044BFA
:101190009A42F6D0FDF79AFDFFF7CAFFF1E700BFCC
:1011A0005490050808B503464868072B05D8DFE8C2
:1011B00003F00517040407040F150021084608BDB5
:1011C000002131F003F800280CBF1E210E21F5E7A5
:1011D00031F044F8410041F00101EFE70028EDDA79
:1011E000BDE8084000F10040FFF7A2BF406870472B
:1011F000F0B587B004460191104603A91646FDF7E5
:101200002FFD002800F0B280232C00F2EA80DFE8F6
:1012100014F0CB00D400D900DE00E300E800E800C1
:10122000E800E800E800E800E800E800E800240042
:1012300029003200E8003700450051007C00E8003A
:10124000E800E800E800E800240029003200E80097
:101250003700450051007C00B4000399019830F03C
:1012600019FD03E00399019830F012FD01900198F7
:10127000FFF75EFF7AE00399019830F013FEF5E77F
:101280000021039830F0A2FF18B157495748FBF7E7
:10129000D7FD03A901A8FFF7EAFEE8E7039C0021B8
:1012A000204630F093FF0028EFD12146019830F01E
:1012B000ADFEDBE7039D0021284630F087FF0446A2
:1012C0000028E2D1294601981DF052F90021064676
:1012D000019030F07BFF039D18B164F31E0501956A
:1012E000C5E70021304630F07BFF0021041E284670
:1012F00018BF012430F074FF003818BF0120E4B299
:101300008442B4D029463046A9E7019D00212846F1
:10131000039C30F05BFF90B10021204630F060FF6D
:1013200068B124F000473846314930F081FF002889
:10133000ABD138462E4930F05DFF0028A5D1002101
:10134000284630F04DFF98B120461EF04DFE214654
:1013500030F03CFF60B92146204630F069FF38B9D3
:101360003346002229462220FEF7FEFD07B0F0BDDD
:10137000214628461DF048FF78E70021039830F009
:1013800025FF002881D103A901A8FFF770FE01986D
:10139000FFF7CEFE04900398FFF7CAFE04A905905C
:1013A000022005F0ABF9E1E70399019830F018FF4E
:1013B000002814BF1E200E20D8E70399019830F0B2
:1013C0002DFFF5E70399019830F000FFF0E703994E
:1013D000019830F00FFFEBE70399019830F014FF0C
:1013E000E6E70020C2E700BF0E830508EC8F050882
:1013F000FFFF7F7F30B494070346496808D1156822
:10140000054CA54204D1134630BC0022FEF7ACBD0A
:10141000184630BCFFF7ECBE2489050810B5044619
:10142000084611460022FDF705F86368BDE8104044
:10143000184770B51C460546084611464FF0021283
:10144000FCF7F8FF6B682068BDE87040184770B57E
:101450001C460546084611464FF00412FCF7EAFF09
:10146000D4E900016B68BDE87040184770B51C46B0
:101470000546084611464FF00612FCF7DBFFD4E99B
:1014800001126B682068BDE8704018472DE9F041F3
:1014900005460E4617469846FCF7BCFFEC684346E7
:1014A000043444F001043A4631462846A446BDE8D7
:1014B000F04160472DE9F04104460E461746984634
:1014C000FCF7A8FFE068434640F001053A46314684
:1014D0002046AC46BDE8F041604700002DE9F04FE2
:1014E000064683B000AF884691469A46FCF792FFC5
:1014F0000021F26812F8013BC3F3C30BC3F380046D
:101500001B0638D40BF1010B04EB44045C44A4002B
:101510002C2C04F114033CD8073323F00703ADEB64
:10152000030D6D4600244146DFF8888053464A4645
:1015300028462E60A5F80CB00AF048F9D8F810300B
:1015400000212B61736828465B68C8F8103008F0EA
:10155000D7FE2B690646C8F8103018BBAB68D3F825
:1015600000801CB12846EEF713FEFEB940460C374A
:10157000BD46BDE8F08F12F8013B4D0003F030008E
:10158000A8404BEA000B03F00200884004430131FD
:10159000B6E718467B60EEF7DEFD7B68054600285F
:1015A000C1D1B9E7D5F81480002CDBD14046EEF765
:1015B000A5FD00BF7003002070B51D46084611460A
:1015C0004FF00412FCF736FF2C68A30703D1226802
:1015D000104B9A4202D00020FCF748FC6D6815F0D1
:1015E0000306F8D12A680C4B9A42F4D11020EEF78A
:1015F000A7FD0346094AC0E9002500F10805324667
:10160000D4E9010185E80300E0681946BDE87040AF
:10161000FAF7C8BFDC880508488B05081C96050842
:101620001FB510F00103044602D0401004B010BDF5
:1016300006283FD00E283DD01E283DD010F00303D1
:1016400008D101681D4A914204D104B0BDE81040A0
:1016500000F055BE04F00702022A04D043B9226804
:10166000174B9A4204D1204601A903F039FDDDE76A
:101670002046FDF7F3F9134B984205D12046FFF7BA
:10168000B5FD30F0EBFDD1E70F4B984202D00F4B88
:10169000984206D16946204601AAFDF769FB0198E8
:1016A000C4E70122204601A9FDF7F4FC0028F6D189
:1016B0002046BBE71846B9E70120B7E724930508A1
:1016C00074A0050854900508C8A105087894050879
:1016D000F0B50C461746054642683946204685B0A7
:1016E0001E46FCF7A7FE6B68DB0706D43146204692
:1016F000AB6805B0BDE8F0401847394606EB8402F8
:1017000001A8FCF75CFF31462046AB6801AA984768
:1017100005B0F0BD2DE9F8430F4605461C46436869
:1017200011465A00384642EA4342FCF783FEAE684F
:1017300046F001062FB9B047E968BDE8F843FCF769
:10174000F7BC012F206803D1FFF76AFFB047F3E72A
:10175000022F09D1FFF764FF07466068FFF760FFBB
:1017600001463846B047E7E7032F0ED1FFF758FF91
:1017700007466068FFF754FF8046A068FFF750FFF8
:10178000414602463846B047D6E7FFF749FF0746CD
:101790006068FFF745FF8046A068FFF741FF81467C
:1017A000E068FFF73DFF4A46034641463846B047EA
:1017B000C2E700000268104910B58A420446C368B7
:1017C00002D00E498A4204D11A68A3680AB153F8BC
:1017D000223013F8012B51B20029184613F8012BBF
:1017E000F9DB10F9013B002BFBDB09F030FE6368ED
:1017F0009B6833F8100010BD4491050880920508DD
:10180000F8B514461268034682B9172906D1FFF7C6
:10181000D1FFC00040F00200206007E040F22F221C
:10182000914204D040F22A22914204D0F8BD43688C
:101830005B682360FAE702680A498A4202D00A49D3
:101840008A42F3D19A68002AF0D15A681020D2E96E
:1018500002760649DD68FDF7F5F8C0E90176C56056
:10186000DAE700BFA890050864920508DC8805083F
:1018700070B5054608460C46FFF79CFF2346024616
:1018800002492846BDE87040EFF7E6BF78900508AA
:101890002DE9F047884691469A460446F8B1076814
:1018A00007B37E6864680CB9304600E0701C0430F1
:1018B0000D498000FDF7C6F80546C0E9019AC0F859
:1018C0000C802FB1B20007F10801103020F037F87A
:1018D00014B1043645F826402846BDE8F08707468F
:1018E0000646E4E73E46DDE7A89005082DE9F84303
:1018F0000F46064600219046C268994612F8013B01
:10190000C3F3C305C3F380041B0616D4013504EBEF
:1019100044042C4407341049A000FDF793F8062333
:101920000446C0E9013685824B46424639460830B6
:1019300009F04CFF2046BDE8F88312F8013B4FEA5E
:10194000410C03F0300000FA0CF0054303F00200F4
:10195000884004430131D7E7449205082DE9F84354
:101960009946C36805461B680F46904684680BB1CC
:1019700054F82340002314F8010BC0F3C3060206F9
:101980001DD406F1080012498000FDF75BF806231C
:1019900001360446C0E9013586824B464246394647
:1019A000083009F01DFF4FF6FF73E382EB68204615
:1019B0005A68134443F00103E360BDE8F88314F868
:1019C000010B00F030029A4016430233D7E700BF04
:1019D0004492050808B50346406810B90248FCF770
:1019E0007FF8596008BD00BF7C91050870B50546B9
:1019F00088680C46FFF7DEFE234602460249284669
:101A0000BDE87040EFF728BF899105082DE9F04146
